:100000000C940A210C943B210C943B210C943B2131
:100010000C943B210C943B210C943B210C943B21F0
:100020000C943B210C943B210C943B210C943B21E0
:100030000C943B210C94A0D20C943B210C943B21BA
:100040000C943B210C94203C0C943B210C943B21C0
:100050000C943B210C943B210C9446370C944A2978
:100060000C943B210C941C370C94EC360C943B21E3
:100070000C943B210C943B210C943B210C943B2190
:100080000C943B210C943B210C943B210C943B2180
:100090000C943B210C943B210C943B210C943B2170
:1000A0000C943B210C943B210C943B210C943B2160
:1000B0000C943B210C943B210C943B210C943B2150
:1000C0000C943B210C943B210C943B210C943B2140
:1000D0000C943B210C943B210C943B210C943B2130
:1000E0000C943B21084AD73B3BCE016E84BCBFFD3C
:1000F000C12F3D6C74319ABD56833DDA3D00C77FF8
:1001000011BED9E4BB4C3E916BAAAABE0000008090
:100110003F05A84CCDB2D44EB93836A9020C50B91F
:10012000918688083CA6AAAA2ABE000000803F004B
:100130004E414E494E495459494E46CDCCCC3D0ACC
:10014000D7233C17B7D13877CC2B329595E6241FAF
:10015000B14F0A000020410000C84200401C462068
:10016000BCBE4CCA1B0E5AAEC59D742500F00F2CA8
:1001700000A00F3300500F3A00000F4300B00E4DA7
:1001800000600E5800100E6300C00D7000700D7EF0
:1001900000200D9000D00CA300800CB900300CD2D0
:1001A00000E00BF000900B1101400B3701F00A63E7
:1001B00001A00A9801500AD601000A1E02B0096F78
:1001C000026009D00210094003C008C1037008543E
:1001D000042008FC04D007B70580078C06300768A8
:1001E00007E006550890064E0940064B0AF0053216
:1001F0000BA005140C5005D80C00058C0DB004188C
:100200000E60048F0E1004F00EC0033A0F700373DB
:100210000F2003BD0F8002DC0F0802E90FB801F2C6
:100220000F6801F80F1801FC0FC800FF0F0000480D
:1002300000901A4800A00F5800000F6C00600E8458
:1002400000C00DA400200DD000800C1001E00B5860
:1002500001400BC001A00A4C02000A08036009F823
:1002600003C00828052008B00680075408E00618D7
:100270000A4006C80BA005300D0005400E6004FCC6
:100280000EC003740F2003BC0F8002E00FE001F4E6
:100290000FF000FB0FC800FC0FA0000400501D7CF5
:1002A00000D009A4001009CC008008F40010081C3C
:1002B00001B807440168076C0128079401E806BCEF
:1002C00001B806E40188060C026006340238065CB8
:1002D0000218068402F005AC02D805D402B805FC69
:1002E0000298052403800574035005C403280514EF
:1002F0000400056404D804B404B0042C058004A4EC
:100300000558041C062804940600040C07D803AC06
:1003100007A8034C087803EC0848038C092003A4C1
:100320000AD0021C0BA802AC0C2802FC0C0802C468
:100330000DB801140E9801B40E38012C0FE00054D2
:100340000FB8007C0F8800A40F4800F40F28FFFCB2
:100350000FC0F9000000008C030800AE035000D667
:1003600003A000F703F0001804400138049001597D
:1003700004E0017A0430029A048002BB04D002FC3B
:100380000470032605C003860630079709A00F7581
:100390000D201C520E401F1F0F6022FF0F803E04D5
:1003A00000081D900058091C01B007A801C80634B8
:1003B000023006C002C0054C036805D80318056466
:1003C00004D004F00498047C05600408063004940A
:1003D0000600042007D003AC07A80338088003C434
:1003E00008580350093003DC090803680AD802F4EE
:1003F0000AB002800B88020C0C6002980C300224B8
:100400000DF801B00DC0013C0E8001C80E30015442
:100410000FB800B40F2800E00F00000400401D904A
:100420000060091C01B007A801D00634023806C0DC
:1004300002C8054C036805D80318056404D804F005
:100440000498047C05600408063004940600042027
:1004500007D003AC07A80338088003C4085803502A
:10046000093003DC090803680AE002F40AB80280D4
:100470000B88020C0C6002980C3002240DF801B0BD
:100480000DC0013C0E8001C80E3001540FB800B4FD
:100490000F2800E00F000004000016D800C006ACD2
:1004A0000178058002C004540348042804E803FCD2
:1004B000049803D0055003A40618037807D8024C0B
:1004C00008A80220097002F4093802C80A08029C30
:1004D0000BD001700C9001440D5001180EF800EC87
:1004E0000E8800C00F00000400681D4C00500B94E3
:1004F000005809DC0050082401A8076C012807B443
:1005000001C006FC017006440228068C02F005D4E6
:1005100002B8051C03880564035805AC033005F4D4
:100520000310053C04E8048404C804CC04A80414A3
:100530000590045C057004A4055804EC05380434E7
:100540000620047C060804C406F0030C07D80354F4
:1005500007C8039C07B003E40798032C08800374C2
:10056000087003BC085803040948034C093003947D
:10057000091803DC090803240AF0026C0AE002B43B
:100580000AC802FC0AB002440BA0028C0B8802D4F9
:100590000B70021C0C5802640C4002AC0C2802F4D4
:1005A0000C10023C0DF001840DD801CC0DB80114E3
:1005B0000E98015C0E7001A40E4801EC0E18013477
:1005C0000FD8007C0F8800C40F0800FC0F0000004B
:1005D000000000000000000000000000000000001B
:1005E000000000000000000000000000000000000B
:1005F0000000000000401F450060094F0010095C2A
:1006000000C0086B0070087D0020089200D007AC85
:10061000008007CC003007F400E006230190065E5E
:10062000014006A601F005FF01A0056D025005F38B
:100630000200059603B0045A046004400510044803
:1006400006C0036E077003A8082003EB09D002233D
:100650000B8002410C3002390DE001040E9001A222
:100660000E4001170FF000690FA000A20F5000C646
:100670000F0000DD0FB0FFEB0F60FF0400700DD81E
:10068000004804AC0158038002D8025403800228B9
:10069000043802FC040002D005C801A406980178C1
:1006A0000770014C08480120091801F409F000C83E
:1006B0000AC8009C0BA000700C7000440D38001894
:1006C0000E0000EC0EA8FFC00FE8FE0400001B5453
:1006D000006009640010097400C008840070089C60
:1006E000002008B800D007D8008007000130072C90
:1006F00001E00668019006AC0140060002F00568C2
:1007000002A005E0025005740300052404B004F0C3
:10071000046004DC051004E406C003040870033020
:10072000092003780B8002600DE001A80E400168EB
:100730000FA000C00F0000E80F60FF0400801AD86F
:10074000009808AC012007800250065403C8052811
:10075000045805FC040005D005B004A4066804781C
:100760000728044C08E8032009B003F4097003C803
:100770000A38039C0BF802700CB002440D68021892
:100780000E0802EC0E8801C00F8800F00F00000078
:1007900000A00F5C006009690010097900C0088C96
:1007A000007008A2002008BD00D007DE0080070509
:1007B0000130073401E0066D019006B201400607E2
:1007C00002F0056D02A005E80250057B0300052B31
:1007D00004B004F8046004EB06C003350920037F6D
:1007E0000B8002650DE001B00E40011D0FF00048C6
:1007F0000FC8006C0FA000ED0F60FFFE0F48FE77E2
:1008000069656465722068657267657374656C6C90
:1008100074004B6F6E66696775726174696F6E0004
:10082000526573657420454550524F4D0025656AE9
:1008300020426C6F636B6164656EF5626572772E42
:10084000004D756C3A20256F6D2525252020202030
:100850004C61733A256F702057004D756C3A202516
:100860006F6D252525202020205370693A256F7053
:1008700052504D005A773A2578372020205A3A2591
:1008800078320059773A257836202020593A257851
:10089000310058773A257835202020583A2578308D
:1008A000005374617274205A2D50726F6265004D4E
:1008B00065737365202E2E2E005A2D4F6666736564
:1008C000743A25587A004162627275636800576510
:1008D00069746572004563687465205A20506F73AF
:1008E0002E3A2557306D6D0054656D702E202565AC
:1008F000632F2545630243004D6573732E205072AC
:100900006F62656E68EF6865004265642020202094
:100910003A20257062024300457874722E20363AE0
:1009200020257035024300457874722E20353A2018
:10093000257034024300457874722E20343A202505
:100940007033024300457874722E20333A202570AC
:1009500032024300457874722E20323A20257031DD
:10096000024300457874722E20313A2025703002FF
:100970004300566F726865697A74656D706572615F
:10098000747572656E00486F6D696E672E2E2E004D
:100990004175746F6C6576656C2042657474004BAC
:1009A000616C696272696572756E67736665686CA1
:1009B0006572004B616C696272696572652042659F
:1009C0006400202020203E3E3E204F6B203C3C3CDB
:1009D000004C6576656C696E67204665686C65726B
:1009E0000046696C616D656E74207275747363681E
:1009F00074004865697A656C656D2E20656E746B50
:100A00006F7070656C740054656D702E2D53656E3B
:100A1000736F7220646566656B74004D69747465EC
:100A2000696C756E673A006175662064656D204279
:100A30006574742073696E642E0064617373206B37
:100A400065696E65204F626A656B746500537465F5
:100A50006C6C656E20536965207369636865722CE0
:100A6000002A2A2A204269747465207761727465AD
:100A70006E202A2A2A0041626272756368004CF572
:100A80006674657220323A254653252525005A2D75
:100A90004B6F7272656B7475723A254465004D65D3
:100AA000737365205A2D5665727A657272756E671A
:100AB0000053657475700025506E00255070252513
:100AC00025004C617965722025506C2F25504C0013
:100AD000456E6453746F70202020203A25647000A6
:100AE0005A2D4F66667365743A2554326D6D005900
:100AF0002D4F66667365743A2554316D6D00582D1F
:100B00004F66667365743A2554306D6D0053657495
:100B1000207072696E74206F666673657473005A14
:100B20002D50726F62656E68EF68653A257A6800CD
:100B30002544332033204B6F7069656E00254432A5
:100B40002032204B6F7069656E00254431203120C2
:100B50004B6F70696500254430204B65696E6520D8
:100B60004B6F7069656E002558352057E1686C65DC
:100B700020457874722E2036002558342057E168BD
:100B80006C6520457874722E203500255833205727
:100B9000E1686C6520457874722E203400457874C5
:100BA00072756465722036204175730045787472E1
:100BB00075646572203520417573004578747275CF
:100BC0006465722034204175730054656D702E2069
:100BD00036203A2565352F25453502430054656D8D
:100BE000702E2035203A2565342F254534024300E8
:100BF00054656D702E2034203A2565332F254533FA
:100C0000024300202542436D6D0005256563020007
:100C1000052565632F254563020000256F730025B8
:100C20005566206D206765647275636B7400255589
:100C300066206D0025557400583A25783020593AC1
:100C4000257831004D756C3A20256F6D20202045A8
:100C50003A257834005A3A257832202042756620A9
:100C60003A20256F4200422565422F254562020049
:100C7000052565632F25456302422565422F2545DD
:100C8000620200256F73005075663A20256F42009E
:100C90004D756C3A20256F6D25252520FD202020DF
:100CA000453A202578346D00466C7573733AFD2003
:100CB000256F6625252520205A3A257832000E20FA
:100CC0002565622F254562B020593A257831000A02
:100CD000202565302F254530B020583A2578300042
:100CE0005370726163686500496E6469762E3A25B7
:100CF00042436D6D00496E646976696475656C6C1C
:100D0000004B6C6562657374696674004772F56EBA
:100D10006573205045542042616E6400426C6175D9
:100D20006573204B7265707062616E64004B617018
:100D3000746F6E004275696C6454616B00556E622D
:100D400065736368696368746574000042657474F0
:100D5000626573636869636874756E673A004265BB
:100D60007474626573636869636874756E67005351
:100D700074616E646279004578747275646572732B
:100D8000746175005A69656C74656D706572617423
:100D900075722E2E2E005761727465206175660083
:100DA0006465722045787472756465722E004B6CB0
:100DB00069636B65207A756D2041756677E1726DA8
:100DC000656E0049676E6F7269657265204D3130DE
:100DD000362025466900536572766F20506F732E5A
:100DE0003A20256F53004175746F6C6576656C3AD7
:100DF00020256C6C00576569746572206D697420DC
:100E00004B6C69636B004D656EF56B6E6F706620A1
:100E100064726568656E005A756D206D616E2E2076
:100E200066EF726465726E0046696C616D656E7422
:100E30007765636873656C3A0046696C616D656ED1
:100E4000747765636873656C005A204261627973D8
:100E50006368722E3A256F596D6D00447275636B2D
:100E60002061626272656368656E004C616E6773D3
:100E70002E424200546F747A6569740041545820C0
:100E80004E65747A7465696C20616E2F61757300AC
:100E90006765647275636B740046696C616D656E3D
:100EA00074206765647275636B74004765732E20E8
:100EB000447275636B7A65697400003A002054616E
:100EC00067652000447275636B65722062657265A8
:100ED00069742E005344204B617274652065696EFD
:100EE00067656C656774005344204B6172746520BC
:100EF000656E746665726E740052F5636B7A2E20AF
:100F0000756D3A255855206D6D0057617274657482
:100F1000656D702E2558540243004C6576656C2033
:100F200064656C7461004265726563686E65204C2F
:100F30006576656C696E67005365747A6520503319
:100F4000005365747A65205032005365747A6520C9
:100F50005031005A204B616C69622E005365747ADF
:100F600065205A3D30005265736574204D6573737A
:100F7000756E67005A65696765204D657373756E98
:100F80006700466C6F77204D756C2E3A256F66258D
:100F90002525004765736368772E4D756C3A256F7C
:100FA0006D2525250020423A2565622F25456202E0
:100FB000437E256F620045333A2565322F25453241
:100FC00002437E256F320045323A2565312F254593
:100FD0003102437E256F310045313A2565302F259A
:100FE000453002437E256F300020453A2565632F4A
:100FF00025456302437E256F430050756666657222
:101000003A256F4200486F63686C6164656E2E2EEE
:101010002E0067656C6164656E2E004B6F6E6669AD
:101020006775726174696F6E006765737065696377
:10103000686572742E004B6F6E66696775726174B5
:10104000696F6E004D6F746F72656E20417573002D
:10105000416E676568616C74656E004865697A65A4
:1010600020447275636B62657474004865697A65C3
:1010700020457874727564657200416B74696F6E97
:101080003A256C61005049440042616E6742616ECE
:101090006700592D4F66667365743A255879005874
:1010A0002D4F66667365743A255878005049442080
:1010B0004D61783A255844004472697665204D6147
:1010C000783A25584D004472697665204D696E3A2C
:1010D00025586D0050494420443A25586400504931
:1010E0004420493A25586900436F6E74726F6C6CE6
:1010F0002D50574D3A25584D00546F747A656974D8
:101100003A2558700050494420503A2558700052F2
:1011100065676C65723A25586800416476616E6354
:101120006520717561643A25586100416476616E8D
:101130006365206C696E3A25586C00537461622EA9
:101140005A6569743A2558770042657363686C2E56
:101150003A255841004D61782046523A25584600BC
:1011600053746172742046523A255866005363687E
:10117000722F4D4D3A25536500426175647261745A
:10118000653A256F6300416C6C67656D65696E003B
:101190005B6D696E5D20303D417573004175732054
:1011A0006E6163683A20256970004D61782E204990
:1011B0006E616B746976005B6D696E5D20303D41D8
:1011C000757300417573206E6163683A20256973F9
:1011D000004D6F746F7220496E616B746976004CBC
:1011E000F56674657220566F6C6C004CF56674651C
:1011F0007220617566203735252525004CF566740B
:10120000657220617566203530252525004CF56610
:1012100074657220617566203235252525004CF5F0
:101220006674657220417573004CF5667465723A98
:10123000254673252525004CF566746572004D69B9
:101240006E3A25737A204D61783A25735A005A3ADE
:10125000257832206D6D004D696E3A257379204DE9
:1012600061783A25735900593A257831206D6D001F
:101270004D696E3A257378204D61783A2573580090
:10128000583A257830206D6D004D696E3A25737A95
:10129000204D61783A25735A005A3A257832206DEC
:1012A0006D004D696E3A257379204D61783A25734A
:1012B0005900593A257831206D6D004D696E3A25F7
:1012C0007378204D61783A25735800583A25783064
:1012D000206D6D0031206B6C69636B203D203120E7
:1012E0006D6D00453A257833206D6D00004D6178B5
:1012F00020456E6473746F70703A25735A004D699F
:101300006E20456E6473746F70703A25737A005A5C
:101310003A257832206D6D00004D617820456E646D
:1013200073746F70703A257359004D696E20456E65
:101330006473746F70703A25737900593A25783167
:10134000206D6D00004D617820456E6473746F7080
:10135000703A257358004D696E20456E6473746F42
:1013600070703A25737800583A257830206D6D00FA
:10137000004D617820456E6473746F70703A257308
:101380005A004D696E20456E6473746F70703A2513
:10139000737A005A3A257832206D6D2025647A25BB
:1013A000645A00004D617820456E6473746F7070EC
:1013B0003A257359004D696E20456E6473746F70E1
:1013C000703A25737900593A257831206D6D2025C2
:1013D000647925645900004D617820456E6473740A
:1013E0006F70703A257358004D696E20456E6473B6
:1013F000746F70703A25737800583A257830206DF4
:101400006D2025647825645800486F6D653A25661F
:101410005A00486F6D65205A3A25665A00486F6D2C
:101420006520593A25665900486F6D6520583A2560
:101430006658004D61783A25667A004D6178205AE9
:101440003A25667A004D617820593A256679004D33
:10145000617820583A256678004665656472617443
:1014600065004461746569206CEF736368656E00A4
:101470004D6F756E74204B6172746500556E6D6FA3
:10148000756E74204B6172746500447275636B20D5
:10149000466F7274732E00447275636B20506175D1
:1014A00073696572656E00447275636B6520446193
:1014B00074656900416E7469204F6F7A65005374DA
:1014C000617274206E6163683A254F61004D696EE8
:1014D0002E416273742E203A254F64004261636B83
:1014E000736C2E2020203A254F620045696E66619C
:1014F0006872656E203A254F7200254F32204F509A
:1015000053205363686E656C6C00254F31204F503B
:1015100053204B6C6173736973636800254F3020EF
:101520004F5053204175730054726F636B656E6C3E
:101530006175663A256464004665686C65722020B2
:101540002020203A25646500496E666F2020202007
:101550002020203A256469004563686F2020202000
:101560002020203A25646F004C61646520766F6D01
:1015700020454550524F4D005369636865726520A0
:10158000454550524F4D0042657363686C65756EFA
:101590006967756E67005A2D5275636B2020203A7B
:1015A00025614A005275636B20202020203A256176
:1015B0006A004265776567653A25615A004265773A
:1015C000656765205A3A25615A0042657765676507
:1015D00020593A2561590042657765676520583A78
:1015E00025615800447275636B656E3A25617A0017
:1015F000447275636B656E205A3A25617A004472B5
:1016000075636B656E20593A256179004472756384
:101610006B656E20583A256178005365747A6520B1
:101620004E756C6C70756E6B74002558322057E1E6
:10163000686C6520457874722E203300255831205F
:1016400057E1686C6520457874722E203200255869
:10165000302057E1686C6520457874722E20310087
:101660004578747275646572203320417573004546
:101670007874727564657220322041757300457804
:101680007472756465722031204175730054656D04
:10169000702E2033203A2565322F25453202430033
:1016A00054656D702E2032203A2565312F25453145
:1016B00002430054656D702E2031203A2565302F8D
:1016C0002545300243004265642054656D703A251B
:1016D00065622F254562024300457874722E2050C2
:1016E0006F736974696F6E005A20506F732E2053A8
:1016F00063686E656C6C005A20506F736974696F13
:101700006E005920506F732E205363686E656C6CA9
:10171000005920506F736974696F6E005820506FC4
:10172000732E205363686E656C6C005820506F7385
:101730006974696F6E004D6F746F72656E204175CC
:10174000737363682E005365747A65204E756C6CF4
:1017500070756E6B740041626BF5686C656E004C61
:10176000616D70656E3A20256C6F00566F7268650A
:10177000697A656E20616C6C6500566F7268656988
:101780007A656E20457874722E203100486F6D6541
:10179000205A00486F6D65205900486F6D652058CC
:1017A00000486F6D6520416C6C6500486F6D652069
:1017B00044656C746100446562756767696E6700B3
:1017C0005344204B6172746500457874727564658A
:1017D0007200506F736974696F6E0045696E73743F
:1017E000656C6C756E67656E00256F65005374657A
:1017F000756572756E67005A7572F5636B2001002E
:101800002A2A2A2A204645484C4552202A2A2A2A92
:10181000004B65696E65205344204B61727465000E
:101820004C6565726C61756600447275636B656EBC
:1018300000447275636B652E2E2E004E65696E0036
:101840004A61006E760041757300416E004A184689
:1018500018431840183B183118291820181118007F
:1018600018F717ED17E917DB17D217C917C017B606
:1018700017AB17A1179A1793178C177A176B175F67
:10188000175617461736172B171C1711170217F77D
:1018900016E816D916C616B316A0168D167E166F44
:1018A0001660164E163C162A161A160C16FE15F061
:1018B00015E415D715CA15BD15B215A415961587CB
:1018C000157815681558154815381528151C150A6A
:1018D00015FA14EB14DC14CD14BE14B414A7149729
:1018E000148A147C147014621459144F1445143B58
:1018F00014331428141D1412140914F913E813D7FF
:1019000013D613C613B513A413A313931382137121
:1019100013701367135613451344133B132A1319FB
:101920001318130F13FE12ED12EC12E312D412CBA4
:1019300012BB12B212A2129912891280127012678F
:101940001257124E123E12371229121E120D12FC9D
:1019500011EB11DF11D111C311B711AA119C119014
:1019600011861179116D116011551149113B112B1F
:10197000111A110F110511F910E810DE10D410C65C
:1019800010B810AC109F109210891085107A106B4F
:10199000105B1050104410361029101B1012100547
:1019A00010FA0FE90FD80FC70FB60FA50F930F82CC
:1019B0000F740F660F5C0F530F4A0F410F380F263D
:1019C0000F1A0F0A0FF90EE70ED40EC40EBD0EBB90
:1019D0000EBA0EAB0E990E900E7C0E740E6B0E5B53
:1019E0000E490E390E280E170E060EF50DE60DD611
:1019F0000DC30DAE0DA00D960D840D770D6F0D5E10
:101A00000D4C0D4B0D3D0D340D2D0D1C0D0C0D0110
:101A10000DF50CE80CE00CCF0CBE0CA80C900C875C
:101A20000C830C700C660C550C440C380C340C2ECA
:101A30000C1F0C1B0C1A0C100C0A0C030CF00BDD09
:101A40000BCA0BBB0BAC0B9D0B8B0B790B670B56AF
:101A50000B4A0B3D0B300B1F0B0D0BFE0AEF0AE080
:101A60000AD00AC20ABB0AB70AB10A9E0A8E0A7EC7
:101A70000A760A610A4D0A3A0A270A1B0A070AF27D
:101A800009E109D109C209B3099F099009860972C0
:101A9000096309540945093609270918090909F88C
:101AA00008E808D508CE08C608B908AF08A108920A
:101AB00008830874085A0841082D0820081208FFF6
:101AC000074865617465722F73656E736F72206568
:101AD00072726F720044697361626C696E67206133
:101AE0006C6C206865617465727320647565207420
:101AF0006F2064657465637465642073656E736FCD
:101B000072206465666563742E00206465672E200C
:101B10004300206D656173757265642000457272C3
:101B20006F723A436F756C64206E6F7420686F6CCF
:101B3000642074656D706572617475726520002033
:101B40006D730020616674657220004572726F7259
:101B50003A54656D702E2072616973656420746FEC
:101B600020736C6F772E2052697365203D20004FE3
:101B70006E6520686561746572207365656D73209C
:101B80006465636F75706C65642066726F6D207438
:101B90006865726D6973746F72202D20646973615A
:101BA000626C696E6720616C6C20666F7220736175
:101BB00066657479210048656174657220646563A7
:101BC0006F75706C6564004865617465642062655A
:101BD00064206578636565646564206D6178207450
:101BE000656D7065726174757265210020453A00FB
:101BF000205A3A0020593A00583A002044303A001E
:101C000020403A002042403A0020524157002044F0
:101C1000423A0020423A00202F00543A00537065A7
:101C200065644D756C7469706C793A00466C6F77B9
:101C30004D756C7469706C793A00206D696E002086
:101C4000686F757273200020646179732000507290
:101C5000696E74696E672074696D653A006D200065
:101C60005072696E7465642066696C616D656E742E
:101C70003A00456E642066696C65206C6973740077
:101C8000426567696E2066696C65206C69737400D3
:101C90005344207072696E74696E6720627974654E
:101CA00020004E6F74205344207072696E74696E08
:101CB000670057726974696E6720746F2066696C7B
:101CC000653A20006F70656E206661696C65642CF2
:101CD0002046696C653A20004372656174696F6ED5
:101CE000206661696C6564004469726563746F7233
:101CF00079206372656174656400657874727564D7
:101D0000657220636F6F6C65722073706565642007
:101D10005B302D3235355D0064697374616E6365C7
:101D200020746F2072657472616374207768656EC9
:101D30002068656174696E67205B6D6D5D00746518
:101D40006D702E20666F72207265747261637469A3
:101D50006F6E207768656E2068656174696E6720B4
:101D60005B435D0074656D702E2073746162696CF5
:101D7000697A652074696D65205B735D005A2D6F0B
:101D80006666736574205B73746570735D00592DAE
:101D90006F6666736574205B73746570735D00585D
:101DA0002D6F6666736574205B73746570735D0078
:101DB000504944206D61782076616C7565205B30F8
:101DC0002D3235355D0050494420442D6761696EE0
:101DD0000050494420492D6761696E0050494420F4
:101DE000502D6761696E2F646561642D74696D653E
:101DF00000504944206472697665206D696E005018
:101E00004944206472697665206D61780068656177
:101E100074206D616E61676572205B302D335D00EB
:101E2000507265686561742074656D702E205BB0BA
:101E3000435D00616363656C65726174696F6E20F8
:101E40005B6D6D2F735E325D00737461727420661A
:101E500065656472617465205B6D6D2F735D006DE7
:101E600061782E206665656472617465205B6D6DB6
:101E70002F735D00737465707320706572206D6DD3
:101E80000052657472616374696F6E20756E646F61
:101E9000207370656564004578747261206578749C
:101EA000727573696F6E206F6E20756E646F20722D
:101EB000657472616374205B6D6D5D005265747250
:101EC000616374696F6E207A2D6C696674205B6D36
:101ED0006D5D0052657472616374696F6E2073701A
:101EE000656564205B6D6D2F735D00526574726172
:101EF0006374696F6E206C656E677468205B6D6DCE
:101F00005D00456E61626C65207265747261637418
:101F1000696F6E20636F6E76657273696F6E205B9A
:101F2000302F315D0042656420504944206D617856
:101F30002076616C7565205B302D3235355D004251
:101F400065642050494420442D6761696E004265F4
:101F5000642050494420492D6761696E00426564E0
:101F60002050494420502D6761696E00426564200D
:101F7000504944206472697665206D696E0042653F
:101F80006420504944206472697665206D61780050
:101F90004265642048656174204D616E61676572B9
:101FA000205B302D335D00426564205072656865AA
:101FB00061742074656D702E205BB0435D00436FCB
:101FC0006174696E6720746869636B6E65737320F2
:101FD0005B6D6D5D005A2D61786973207472617656
:101FE000656C20616363656C65726174696F6E20F6
:101FF0005B6D6D2F735E325D00592D6178697320C2
:1020000074726176656C20616363656C657261747E
:10201000696F6E205B6D6D2F735E325D00582D61B0
:102020007869732074726176656C20616363656C96
:1020300065726174696F6E205B6D6D2F735E325DCA
:10204000005A2D6178697320616363656C65726104
:1020500074696F6E205B6D6D2F735E325D00592D5C
:102060006178697320616363656C65726174696F1F
:102070006E205B6D6D2F735E325D00582D61786947
:102080007320616363656C65726174696F6E205B58
:102090006D6D2F735E325D005061726B20706F73D7
:1020A0006974696F6E205A207261697365205B6D77
:1020B0006D5D005061726B20706F736974696F6E33
:1020C0002059205B6D6D5D005061726B20706F73E5
:1020D0006974696F6E2058205B6D6D5D005A206DCC
:1020E0006178206C656E677468205B6D6D5D00596A
:1020F000206D6178206C656E677468205B6D6D5D26
:102100000058206D6178206C656E677468205B6D87
:102110006D5D005A206D696E20706F73205B6D6D70
:102120005D0059206D696E20706F73205B6D6D5D71
:102130000058206D696E20706F73205B6D6D5D00BF
:102140004D61782E205A2D6A65726B205B6D6D2F64
:10215000735D004D61782E206A65726B205B6D6D3A
:102160002F735D005A2D6178697320686F6D696EF9
:1021700067206665656472617465205B6D6D2F73A1
:102180005D00592D6178697320686F6D696E6720F5
:102190006665656472617465205B6D6D2F735D00AB
:1021A000582D6178697320686F6D696E6720666568
:1021B000656472617465205B6D6D2F735D005A2DCF
:1021C00061786973206D61782E206665656472613F
:1021D0007465205B6D6D2F735D00592D6178697397
:1021E000206D61782E206665656472617465205B80
:1021F0006D6D2F735D00582D61786973206D617866
:102200002E206665656472617465205B6D6D2F7349
:102210005D005A2D61786973207374657073207046
:102220006572206D6D00592D617869732073746536
:10223000707320706572206D6D00582D6178697320
:1022400020737465707320706572206D6D00537417
:102250006F7020737465707065722061667465724A
:1022600020696E6163746976697479205B6D732C83
:10227000303D6F66665D004D61782E20696E61634A
:10228000746976652074696D65205B6D732C303DD3
:102290006F66665D005072696E746572206163746A
:1022A000697665205B735D0046696C616D656E746F
:1022B000207072696E746564205B6D5D00426175AB
:1022C0006472617465004C616E677561676500508A
:1022D0004944204175746F74756E65206661696C40
:1022E0006564212074696D656F75740050494420E0
:1022F0004175746F74756E65206661696C656421E3
:102300002054656D706572617475726520746F6FAD
:10231000206869676800204B643A2000204B693AC6
:102320002000204B703A2000205479726575732D7F
:102330004C7962656E205049440020506573736586
:102340006E20496E74656772616C2052756C6520F1
:1023500050494400204E6F204F76657273686F6F4E
:1023600074205049440020536F6D65204F7665728C
:1023700073686F6F74205049440020436C6173731D
:10238000696320504944002054753A2000204B7561
:102390003A2000206D61783A2000206D696E3A2065
:1023A0000020643A200020626961733A200050499D
:1023B00044204175746F74756E6520737461727416
:1023C000004E6F2063617365206C696768747300E9
:1023D0004D617854656D703A004469616D6574654E
:1023E000723A00416363656C65726174696F6E3A3D
:1023F000004D617853706565643A004A65726B3AC6
:10240000004D617842656454656D703A00507269A0
:102410006E746572547970653A436172746573695C
:10242000616E005A54726176656C416363656C3A03
:10243000005954726176656C416363656C3A00586B
:1024400054726176656C416363656C3A005A5072F0
:10245000696E74416363656C3A00595072696E74B9
:10246000416363656C3A00585072696E74416363EE
:10247000656C3A005A53697A653A005953697A652E
:102480003A005853697A653A005A4D61783A0059D2
:102490004D61783A00584D61783A005A4D696E3A6C
:1024A00000594D696E3A00584D696E3A0052657494
:1024B00072616374696F6E556E646F5370656564A5
:1024C0003A0052657472616374696F6E556E646F21
:1024D00045787472614C6F6E674C656E6774683ACC
:1024E0000052657472616374696F6E556E646F45F6
:1024F000787472614C656E6774683A0052657472E4
:10250000616374696F6E5A4C6966743A00526574FF
:1025100072616374696F6E53706565643A005265E9
:102520007472616374696F6E4C6F6E674C656E6731
:1025300074683A0052657472616374696F6E4C65B9
:102540006E6774683A004A65726B5A3A004B65656B
:1025500070416C697665496E74657276616C3A009B
:102560004A65726B58593A005072696E746C696EA4
:102570006543616368653A00454550524F4D3A00E6
:102580004175746F6C6576656C3A005A50726F6273
:10259000653A00436173654C69676874733A005328
:1025A0007570706F72744C6F63616C46696C616DAD
:1025B000656E746368616E67653A00537570706F1D
:1025C00072744731304731313A005A486F6D655067
:1025D0006F733A0059486F6D65506F733A005848F1
:1025E0006F6D65506F733A005A486F6D654469723C
:1025F0003A0059486F6D654469723A0058486F6DEA
:10260000654469723A00536F667477617265506F02
:102610007765725377697463683A004C43443A00B3
:1026200046616E323A300046616E3A00534443616F
:1026300072643A004865617465644265643A004DAD
:102640006978696E6745787472756465723A004E90
:10265000756D45787472756465723A00496E70756F
:10266000744275666665723A00426175647261749F
:10267000653A00696E666F3A436F6E74696E756590
:102680002066726F6D20666174616C207374617472
:1026900065000054657374696E6720666174616CCF
:1026A000206572726F7200436F6E66696775726142
:1026B00074696F6E206C6F616465642066726F6D03
:1026C00020454550524F4D2E00436F6E6669677529
:1026D000726174696F6E2073746F72656420746FB9
:1026E00020454550524F4D2E00436F6C6420657855
:1026F00074727573696F6E20646973616C6C6F7747
:10270000656400436F6C6420657874727573696FDB
:102710006E20616C6C6F77656400547269676765E1
:1027200072696E67207761746368646F672E2049F1
:1027300066206163746976617465642C20746865D1
:10274000207072696E7465722077696C6C20726596
:102750007365742E005761746368646F67206469E1
:102760007361626C6564004175746F726574726147
:1027700063743A00205A4A65726B3A004A65726B7C
:102780003A0020746F200053657420766F6C756D6D
:10279000657472696320657874727573696F6E20F1
:1027A000666F722065787472756465722000446982
:1027B0007361626C656420766F6C756D65747269A7
:1027C0006320657874727573696F6E20666F72200E
:1027D00065787472756465722000205052454845D2
:1027E000415400505245484541545F4245443A00E7
:1027F000205A533A002059533A0058533A00505245
:1028000045484541543A3100504155534553544F82
:10281000503A3100544F47474C455F4C4947485464
:10282000533A3000534F4654574152455F504F572B
:1028300045523A31005A5F50524F42453A300041BA
:1028400055544F4C4556454C3A3000454550524F33
:102850004D3A31004155544F5245504F52545F54F8
:10286000454D503A310050524F47524553533A313B
:10287000004649524D574152455F4E414D453A52EF
:10288000657065746965725F312E302E3320434F59
:102890004D50494C45443A53657020313720323011
:1028A0003139204649524D574152455F55524C3AB5
:1028B00068747470733A2F2F6769746875622E6339
:1028C0006F6D2F72657065746965722F52657065E2
:1028D000746965722D4669726D776172652F20503B
:1028E000524F544F434F4C5F56455253494F4E3A07
:1028F000312E30204D414348494E455F5459504593
:102900003A4D656E64656C204558545255444552A5
:102910005F434F554E543A31205245504554494536
:10292000525F50524F544F434F4C3A330050696EF0
:102930002063616E206E6F74206265207365742061
:102940006279204D34322C20697320696E207365C2
:102950006E7369746976652070696E73212000203A
:1029600069732000496C6C6567616C205320766147
:102970006C756520666F72204D34320020746F20B4
:1029800000536574206F75747075743A20000001EF
:1029900036372603023C3D380E0F2E303E12130D03
:1029A0000C0A081A1C180D0E35496E76616C6964A4
:1029B0002061726300205A5F4F46465345543A00E7
:1029C00020595F4F46465345543A00585F4F46469C
:1029D0005345543A0052656C617469766520706F96
:1029E000736974696F6E696E67004162736F6C75AD
:1029F000746520706F736974696F6E696E670055D6
:102A00006E6B6E6F776E20636F6D6D616E643A00F2
:102A10004361703A00436F6E6669673A00496E66BB
:102A20006F3A004572726F723A00494E46004E414D
:102A30004E00436F6E66696775726174696F6E20D0
:102A4000726573657420746F2064656661756C745B
:102A5000732E0050726F746F636F6C2076657273A3
:102A6000696F6E206368616E6765642C207570679E
:102A7000726164696E67004465746563746564209F
:102A8000454550524F4D2076657273696F6E3A001E
:102A9000457874722E004550523A3320004550520A
:102AA0003A3220004550523A3120004550523A30D7
:102AB00020007A5F6D696E3A004C20004820007952
:102AC0005F6D696E3A00785F6D696E3A00656E649D
:102AD00073746F7073206869743A200053656C6575
:102AE000637445787472756465723A003A00546193
:102AF00072676574457874720054617267657442D8
:102B000065643A008F073B07CB067B060000000098
:102B10000000F305E70497041B049F0353039B0283
:102B20002F026B011C151C140000002243141F1FF0
:102B3000132E1B315072696E746572207365742098
:102B4000696E746F206472792072756E206D6F6487
:102B50006520756E74696C2072657374617274217E
:102B600000206D61726B6564206465636F75706CC5
:102B7000656400206D61726B6564206465666563E1
:102B800074003A20776F726B696E67003A20746543
:102B90006D702073656E736F722064656665637413
:102BA000006578747275646572200068656174658B
:102BB0006420626564000000420FA1071605D0037F
:102BC0000D038B022E02E801B2018601630145016B
:102BD0002C0117010401F4000000000000000000B7
:102BE000000000000000000024F403D950C38EB19F
:102BF000C2A23D96828B3582127AE372816CCB66DB
:102C0000A861015DC758EB546151204E1E4B5648D8
:102C1000C14559431A41013F093D2F3B7139CD3719
:102C20004036C93465331432D430A32F802E6B2D37
:102C3000632C672B752A8E29B028DC2710274B269A
:102C40008F25D9242B248223E0224322AC211A2170
:102C50008D200420801F001F841E0C1E971D261D22
:102C6000B81C4E1CE61B821B201BC11A641A0A1AD0
:102C7000B2195D190A19B9186A181C18D1178817E2
:102C80004017FA16B51673163116F115B3157615E9
:102C90003A150015C7148F1458142214EE13BA13E2
:102CA000881356132513F612C71299126C1240128C
:102CB0001512EB11C1119811701148112111FB105F
:102CC000D610B1108D106910461024100210E10FBB
:102CD000C00FA00F800F610F420F230F060FE80EE9
:102CE000CB0EAF0E930E770E5C0E410E270E0D0E1F
:102CF000F30DDA0DC10DA80D900D780D600D490D85
:102D0000320D1B0D050DEF0CD90CC30CAE0C990C3C
:102D1000850C700C5C0C480C350C210C0E0CFB0B5C
:102D2000E80BD60BC40BB20BA00B8E0B7D0B6B0B01
:102D30005A0B4A0B390B290B180B080BF80AE90A36
:102D4000D90ACA0ABB0AAC0A9D0A8E0A800A710A0D
:102D5000630A550A470A390A2C0A1E0A110A040A8C
:102D6000F709EA09DD09D009C409B709AB099F09C8
:102D7000920987097B096F09630958094C094109C0
:102D800036092B09200915090A090009F508EB087D
:102D9000E008D608CC08C208B808AE08A4089A080B
:102DA000900887087D0874086B08610858084F0868
:102DB00046083D0834082C0823081A081208090898
:102DC0000108F807F007E807E007D807D007C807A9
:102DD000C007B807B007A807A1070000010000005E
:102DE00000FFFF0000000001000044656275674CB1
:102DF0006576656C3A005072696E7465724D6F64E9
:102E0000653A434E43005072696E7465724D6F644B
:102E1000653A4C61736572005072696E7465724DEB
:102E20006F64653A464646005A206A65726B2077A1
:102E3000617320746F6F206C6F772C2073657474CE
:102E4000696E6720746F20005859206A65726B2084
:102E500077617320746F6F206C6F772C20736574AB
:102E600074696E6720746F2000534420636172643C
:102E700020696E73657274656400534420636172E7
:102E8000642072656D6F7665640052657175657357
:102E90007453746F703A00627573793A70726F632D
:102EA000657373696E6700627573793A68656174FA
:102EB000696E6700627573793A7061757365642035
:102EC000666F72207573657220696E7465726163D6
:102ED00074696F6E00526573656E643A006F6B20A3
:102EE0000020676F7420004572726F723A657870C7
:102EF0006563746564206C696E652000736B69702E
:102F000020006F6B004563686F3A00466F726D6119
:102F100074206572726F7200436865636B73756DC0
:102F2000207265717569726564207768656E2073BB
:102F30007769746368696E67206261636B20746F80
:102F40002041534349492070726F746F636F6C2E38
:102F500000204F00204C00204B0020420020410068
:102F6000204800204300204400205200204A002036
:102F70004900205000205300204600204500205AE0
:102F800000205900205800202D205072696E746571
:102F9000722073746F7070656420616E6420686560
:102FA00061746572732064697361626C6564206426
:102FB000756520746F2074686973206572726F7212
:102FC0002E20466978206572726F7220616E6420CF
:102FD000726573746172742077697468204D393931
:102FE000392E00666174616C3A0053442065727238
:102FF0006F7220646964206E6F74207265636F76EF
:10300000657221005344206572726F722066697880
:1030100065640053442052656164204572726F728A
:103020000053442072656164206572726F720044BF
:103030006F6E65207072696E74696E672066696C68
:10304000650001FF00004D180000000000000000B6
:103050000000000000000000000000008431446512
:103060007574736368000000042604400000009635
:10307000000000044C0400000000BB000000044DF0
:103080000400000000BC000000042E04000000004A
:1030900090000000042A04000000008F00000004DB
:1030A0002B04000000008E000000042C040000002F
:1030B000008D000000042904000000008C000000C6
:1030C0000413040000000055000000041204000076
:1030D0000000540000000411040000000053000030
:1030E0000004160400000000510000000415040054
:1030F00000000050000000041404000000004F0015
:103100000000040F040000000038000000040E045A
:103110000000000037000000040D0400000000352E
:10312000000000040C040000000034000000040B48
:10313000040000000033000000040A040000000046
:103140003100000004090400000000300000000409
:103150000804000000002F00000000000000000034
:10316000008900000000000000000000880000004E
:1031700000000000000000860000000000000000C9
:10318000000085005E3003A526000000000000005E
:103190000004D004000000002201000004CF04005D
:1031A00000000028010000010000000000002101D3
:1031B0000000038204000000000A010000038104F3
:1031C000000000003F000000038004000000003EFB
:1031D000000000037F04000000003D000000037EAB
:1031E00004000000003C008E38B330A8309D3092BF
:1031F0003087307C3071305E34533448343D343263
:103200003427341C34663011348E38F530EA30DF20
:1032100030D430C930BE308E384D31423137312C48
:1032200031213116310B3100316331583179316E32
:10323000318E388431A5318E389A318F318E38DC19
:1032400031D131C631BB31B0310200001100E7315C
:10325000020000070009320200000900173203587B
:10326000040200293203200402002D320200000271
:103270000031320200000400353202000006003D39
:1032800032000003DB0400000000370100000307E8
:1032900004000000003B00000003060400000000E2
:1032A0003A000000024932000000000F0000000256
:1032B0005032000000004E000000025732000000B3
:1032C0000039000000025E320000000087000000AC
:1032D00002653200000000840000000410040000B9
:1032E00000008B000000026C3200000000E40000CF
:1032F000000273320000000021010000027A320057
:103300000000001100000004BD0400001000E300F4
:10331000000003B90400001000E100000003B8043D
:1033200000001000E000000003B60400001000DF01
:1033300000000003B50400001000DE00000003BE22
:103340000400001000DD00000003B70400001000BE
:10335000DC00000004B60F000000000901000004BA
:10336000B50F000000000801000004B40F000000C9
:10337000000701000000000000000000F200000053
:1033800000000000000000AB000000000000000092
:10339000000070000000000000000000006F00004E
:1033A0000003E803000000002D0100000388130063
:1033B0000000002C01000004F203000000002A01BC
:1033C000000001000000000000CB008E38E432D97C
:1033D00032CE32C332B832AD32A2326C3D97328C2B
:1033E0003281328E38FA32EF328E3847333C333105
:1033F0003326331B33103305338E3868335D335235
:1034000033943389337E337333C033B533AA339F58
:10341000330000042F04000000009B000000042281
:103420000440000000950000000426042000000075
:103430009A00000004250420000000990000000408
:103440002404200000009800000004230420000051
:1034500000970000000422042000000094000000F7
:10346000042D040000000093000200000C00CB3388
:103470000200000300E3330200000800E933020009
:10348000000400F93303F003040001348200000457
:103490000009348E385E34533448343D3432342796
:1034A000341C3411340000026934000010000D0097
:1034B0000000027034000010000E01000002583EAF
:1034C000000000001000000002773400001000D956
:1034D00000000002193E000010000F000000021260
:1034E0003E000010000E0000000457041000000011
:1034F000CA00000004480410000000B100000002EF
:103500008C3410000000CB000000041F04100000E9
:1035100000B000000004610410000000240000005E
:10352000046204100000002500000003C40404002D
:1035300000004A000000034B041000040049000092
:103540000003C50410000400C900000002203E0072
:103550000010000B00000000000000000000E00070
:10356000000000000000000000DA00000000000081
:1035700000000000DF00000000000000000000DA92
:1035800000000000000000000000E100000000005A
:103590000000000000DA0000000000000000000051
:1035A000DE00000000000000000000DA0000000063
:1035B000000000000000DD0000000000000000002E
:1035C00000DA00000000000000000000DC00000045
:1035D00000000000000000DA000000000000000011
:1035E0000000CF00000000000000000000CE00003E
:1035F0000000000000000000CD00000000000000FE
:10360000000000CC000000027E3400000000060133
:103610000000023C3E000000002100000002273EA6
:10362000000000002200000002433E000000001FD6
:10363000000000022E3E0000000020000000024AB0
:103640003E000000001D00000002353E00000000AA
:103650001E0000000300040000100016000000031C
:10366000FF03000010001500000003FE030000101F
:103670000014000000034404000000002E000000BD
:103680000285340000000023000000033A0400001B
:103690000000280000000462040000000025000073
:1036A0000004610400000000240000000336040050
:1036B000000000C6000000034304000010001C00CE
:1036C0000000033104000010001B00000003380458
:1036D000000000001A00000003470400000000186A
:1036E0000000000337040000000017000000028CF7
:1036F0003400000000CB000000044804000000007B
:10370000B1000000041F0400000000B0000000042D
:10371000570400000000CA00000003FD0300001071
:103720000013000000000000000000006E00000018
:10373000000000000000006D00000000000000001C
:1037400000006C000000000000000000006B0000A2
:1037500000000000000000006A00000000000000FF
:103760000000006900000000000000000000680088
:1037700000000000000000000067000000000000E2
:10378000000000006600000000000000000000656E
:1037900000000000000000000000640000000000C5
:1037A00000000000006300000000000000000000B6
:1037B0006200000000000000000000610000000046
:1037C0000000000000006000000000000000000099
:1037D000005F000000000000000000005E0000002C
:1037E000000000000000005D00000000000000007C
:1037F00000005C000000000000000000005B000012
:1038000000000000000000005A000000000000005E
:1038100000000059000000000000000000005800F7
:103820000000000000000000005700000003C62454
:10383000100000000300000003E803000000000483
:1038400000000001000000000000F4000000010082
:103850000000000000C900000003F40301000200A2
:103860004D00000002513E02000000C900000003AC
:10387000F703060000004A00000003F603020004FC
:10388000004900000003F5030100020048000000A9
:1038900003E803000000000A000000000000000030
:1038A00000003901000000000000000000380100A5
:1038B0000000000000000000A80000000000000060
:1038C000000000A700000000000000000000A600AB
:1038D000000000000000000000A500000000000043
:1038E000000000001301000000000000000000F4D0
:1038F00000000000000000000000200100000000A7
:103900000000000000F400020000090093348E382B
:103910004A353F35343529351E3513350835FD34E4
:10392000F234E7348338DC34D134C634BB34B034B9
:10393000A5346035553576356B358C358135A235F6
:103940009735B835AD35CE35C335FA35EF35E43575
:10395000D9358E38183768365D36523647363C369C
:10396000313626361B3610367E3605368E389F3673
:10397000943689367E3673368E3818370D370237CF
:10398000F736EC36E136D636CB36C036B536AA3603
:10399000443739372E372337703765375A374F3723
:1039A0009C37913786377B37C837BD37B237A73753
:1039B000F437E937DE37D337203815380A38FF3780
:1039C0004C38413836382B388E38833878386D3853
:1039D000623857388E38A4389938BA38AF38D0386A
:1039E000C538FC38F138E638DB380000000000004C
:1039F000000000F700000000000000000000DA00F6
:103A0000F539EA390000000000000000001C010048
:103A10000000000000000000F400000000000000B2
:103A20000000001B01000000000000000000170162
:103A30000000000000000000001C01000000000069
:103A400000000000F4000000000000000000001A68
:103A5000010000000000000000001701000000004D
:103A600000000000001C0100000000000000000039
:103A7000F400000000000000000000190100000038
:103A8000000000000000170100000000000000001E
:103A9000001C01000000000000000000F400000015
:103AA00000000000000000180100000000000000FD
:103AB00000001701253A1A3A0F3A043A513A463AA9
:103AC0003B3A303A7D3A723A673A5C3AA93A9E3AC2
:103AD000933A883A000000000000000000F1000066
:103AE0000000000000000000C40000000000000012
:103AF000000000F000000000000000000000C30013
:103B0000000000000000000000F3000000000000C2
:103B100000000000F400000000000000000000AF02
:103B200000000000000000000000AB0000000000EA
:103B30000000000000F30000000000000000000092
:103B40005F000000000000000000005B00000000BB
:103B5000000000000000570000000000000000000E
:103B600000F300000000000000000000EE00000074
:103B700000000000000000ED000000000000000058
:103B80000000EB00F53AEA3ADF3AD43A213B163B23
:103B90000B3B003B4D3B423B373B2C3B793B6E3B69
:103BA000633B583B0000000400843B00000004001D
:103BB0008C3B0000000400943B00000004009C3B90
:103BC000000000002200250028002B002E003100FC
:103BD000340002010000050108010B010000200073
:103BE0002300260029002C002F00320000010000D5
:103BF00003010601090100000A0B02090C0D0E0861
:103C000007030401000000000000000000000000A5
:103C100000000000000000000000000000000000A4
:103C20000000121110000000000000000000000061
:103C300000000000000000000000000002536F665A
:103C4000747761726520526573657400576174639F
:103C500068646F672052657365740042726F776E97
:103C6000206F7574205265736574004578746572B1
:103C70006E616C20526573657400506F7765725584
:103C800070000D0E110A0411040A1111001C1F11FD
:103C9000111F0000040A0A0A0E1F1F0E001F111137
:103CA000111F0000001F1F1F1F1F0000040A040037
:103CB00000000000040E150404041C005374616429
:103CC0007466616272696B616E74656E20652E56F2
:103CD0002E004D697374657220477265656E0052DF
:103CE0006570657469657220312E302E330046721E
:103CF00065652052414D3A0082000001005C304E63
:103D000065656473206C616E6775616765207365B6
:103D10006C656374696F6E007374617274005772BE
:103D20006F6E6720636865636B73756D007761699B
:103D30007400005344207072696E742073746F7045
:103D400070656420627920757365722E005265710A
:103D50007565737450617573653A00526571756568
:103D60007374436F6E74696E75653A0000000207E4
:103D70003900000000A2002F2F20616374696F6E6C
:103D80003A726573756D650044656C6574696F6E34
:103D9000206661696C65640046696C652064656CC9
:103DA000657465640002000012000E3903102702DA
:103DB0000032390310270200363903102702003A77
:103DC0003903102702003E3903102702004239034D
:103DD00010270200463905881304004A392F2F2086
:103DE000616374696F6E3A706175736500696D70B7
:103DF0006F7274616E743A2046696C616D656E74A1
:103E0000206368616E6765207265717569726564AB
:103E100021000200000D00523902000006006C393A
:103E20000200000C00783903FC030400903903FB06
:103E3000030400983903FA030400A03903EF0304D4
:103E400000A83903EE030400B03903ED030400B801
:103E5000390200000400C0390200000600C8390120
:103E600000000100D4390310270200D639031027BF
:103E70000200DA390310270200DE394A616D20633F
:103E80006F6E74726F6C2064697361626C65643A02
:103E90000005CC040400E239008025000040380011
:103EA00000004B00008070000000960000C0DA00A7
:103EB0000000E10000002C010008B2010000C20176
:103EC0000000F401000084030090D0030000E80328
:103ED000000008070020A1070000100E0040420F5C
:103EE0000060E3160000000000000310270200003D
:103EF0003A446F6E6520736176696E672066696CFF
:103F0000652E006572726F722077726974696E67D0
:103F100020746F2066696C650050494420417574B7
:103F20006F74756E652066696E69736865642021BB
:103F300020506C61636520746865204B702C204BA9
:103F40006920616E64204B6420636F6E7374616ED0
:103F5000747320696E2074686520436F6E666967AC
:103F600075726174696F6E2E68206F7220454550BE
:103F7000524F4D002F005344204361726420756EF0
:103F80006D6F756E7465640005CB040400B43A056A
:103F9000CB040400BC3A05CB040400C43A05CB04AE
:103FA0000400CC3A43617264207375636365737374
:103FB00066756C6C7920696E697469616C697A6583
:103FC000642E0043616E2774206F70656E20726FDF
:103FD0006F74206469726563746F72792E0A00438E
:103FE000616E27742066696E6420612076616C6959
:103FF000642046415431362F46415433322070619B
:1040000072746974696F6E2E0A006572726F724302
:104010006F64653A20000A534420696E69746961CF
:104020006C697A6174696F6E206661696C65642E73
:104030000A446F206E6F74207265666F726D6174D2
:10404000207468652063617264210A497320746872
:1040500065206361726420636F72726563746C794A
:1040600020696E7365727465643F0A4973206368E2
:10407000697053656C6563742073657420746F2078
:1040800074686520636F72726563742076616C7505
:10409000653F0A446F657320616E6F7468657220B6
:1040A00053504920646576696365206E65656420B8
:1040B000746F2062652064697361626C65643F0A95
:1040C0004973207468657265206120776972696E32
:1040D000672F736F6C646572696E672070726F62B0
:1040E0006C656D3F00534420696E69742066616998
:1040F0006C000046696C652073656C65637465646B
:10410000002053697A653A0046696C65206F7065D6
:104110006E65643A0066696C652E6F70656E206628
:1041200061696C65640000002100240027002A00FA
:104130002D003000330001010000040107010A01D5
:1041400001021020200808102040102040800201A9
:10415000020108040201010204081020408080408E
:10416000201008040201800402018040201008048D
:10417000020108040201010204081020408001022B
:1041800004081020408005050505070508080808F3
:10419000020202020A0A08080404040401010101DF
:1041A00001010101030303030303030304070707DA
:1041B0000C0C0C0C0C0C0C0C02020202060606067F
:1041C000060606060B0B0B0B0B0B0B0BB93BB23B9E
:1041D000AB3BA43B2020203F2E3F3F0020486F6D8B
:1041E000696E6700206465632000206465662000B6
:1041F0002000040003000000003FCDCC4C3D0AD756
:10420000A33B6F12033A17B75138ACC5A73600402D
:104210001454F8E011241FBECFEFD1E2DEBFCDBFB2
:1042200000E00CBF22E1AAECB3E001C01D92A43D66
:10423000B207E1F713E0A0E0B2E0E8E9F8EE01E050
:104240000BBF02C007900D92AA3CB107D9F711E24B
:10425000CAE0D1E200E006C021970109802FFE01EB
:104260000E94C2F2C930D10780E00807A9F70E9476
:10427000A8E10C944AF40C940000BF92CF92DF9214
:10428000EF92FF920F931F93CF93DF93DB01FC011B
:104290009F012F5F3F4F8081803209F49EC01496AA
:1042A000FC93EE9313979F0189010E1B1F0B722F36
:1042B000632FE90189919E01882379F08F3209F0FB
:1042C0008EC0CF01800F911F782F692FEC012991AB
:1042D000CE012032C9F32F32B9F3EA017883698322
:1042E000E801CE0FDF1F8E010E1B1F0BCE17DF075D
:1042F00009F495C08A918E32B1F38032A1F30F3F59
:10430000110511F00CF06DC012961C930E931197CD
:10431000ED012696CD01419620E229938C179D0749
:10432000E1F7EF019E012E1B3F0B89918E32D1F3F5
:104330008032C1F381E02115310509F080E0A80148
:1043400041505109EF01C00FD11F4F3F540709F0F1
:1043500069C0F12C67E0B12C70E0D8E0ED2E201799
:1043600031070CF0ACC06F01C20ED31EE60198817C
:10437000903209F483C09E3221F42417350709F0E6
:104380007DC0D92F9232E1F09C37D1F0C6EDDC2E02
:10439000D90EC5E0CD1510F09D3291F4C6ECDC2E9F
:1043A000D90EC5E0CD1560F4C5EADC2ED90EC2E009
:1043B000CD1530F4CFEDDC2ED90ECDE5CD15C8F5F9
:1043C0002417350709F076C06A3009F477C06AE02F
:1043D00098E0B92EC0E1EC2E52C0F90159CF8C35CE
:1043E00059F480E0DF91CF911F910F91FF90EF90F2
:1043F000DF90CF90BF900895982F977F923289F3E6
:104400008A3379F3982F9F7B9C3359F392EC980F62
:10441000923038F380528F3508F446CFE2CF10E067
:1044200000E072CF9A919E3209F493CF4150510926
:104430008CCF2417350741F26B15F0F1CFE9DC2E54
:10444000D90EC9E1CD1508F19052FE28DD24D39490
:10445000DB0CED01CB0DD11D9E83D6E0DD1518F0F0
:104460001596DC921597BD2C0AC04217530734F1FC
:104470009A016AE0D8E0BD2E80E1E82E80E02F5F4F
:104480003F4F6DCF80E09FE5DFE5D154DA31F0F6A4
:104490007E29DCCF81E08C9315966C911597A60F41
:1044A000B11D8EE716968C93169781E317968C9321
:1044B00081E098CF6B1530F76A30B9F680E0169638
:1044C0009C911697903209F48CCF882319F37F21A1
:1044D00011F0D2E0FD2EFC9285CF0895DC01CB01D6
:1044E000BA01A901949FE12D969FF02D812D959FF2
:1044F000E00DF11D871FA49FE00DF11D871FA59FF3
:10450000F00D811DB49FF00D811DA69F800DB59FFC
:10451000800D8695F795E7958695F795E795112493
:10452000CF0108959C01229FB001339FC001239FBA
:104530002227700D811D921F700D811D921F112465
:1045400008952F923F924F925F926F927F928F9237
:104550009F92AF92BF92CF92DF92EF92FF920F9312
:104560001F93CF93DF93EC01888180FDE4C08981A4
:1045700080FDE1C0FE01FD9680809180A280B38025
:1045800070962081318142815381C501B4010E941E
:1045900020EE2B013C01FE01E359FF4F0081118108
:1045A000B80190E080E00E94BFED6B017C011E012C
:1045B0002FE6220E311CFE01E75BFF4F2081318187
:1045C00042815381C501B4010E9420EEA7019601EA
:1045D0000E9420EE0E9499F0D1016D937C935E01C0
:1045E000B1E7AB0EB11CA7019601C301B2010E9455
:1045F00020EE0E9499F0F50171836083C80192DF7B
:104600002B013C01D1018D919C918CDF8E01035ACD
:104610001F4FA3019201261B370B480B590BCA01F0
:10462000B9017E0135E6E30EF11CD7012D913D91D4
:104630004D915C91220F331F441F551F0E9427EF9D
:104640002F5F3F4F4F4F5F4FF801208331834283ED
:104650005383D5018D919C9165DFA3019201261BA7
:10466000370B480B590BCA01B901D7012D913D9168
:104670004D915C91220F331F441F551F0E9427EF5D
:1046800029013A01BFEF4B1A5B0A6B0A7B0A1E0134
:10469000E1E62E0E311CD1014D925D926D927C921D
:1046A0001397F801C080D180E280F380D301C2016A
:1046B0008C0D9D1DAE1DBF1DBE016D587F4FFB01B2
:1046C00080809180A280B38088159905AA05BB05DA
:1046D0007CF188199909AA09BB09B695A795979500
:1046E0008795460157018C159D05AE05BF0514F44D
:1046F0004C015D01C818D908EA08FB08F801C0821E
:10470000D182E282F3827301620184159505A605C8
:10471000B70514F46C017D01A30192012C193D0928
:104720004E095F09D1012D933D934D935C931397EF
:10473000888181608883DF91CF911F910F91FF90D5
:10474000EF90DF90CF90BF90AF909F908F907F9031
:104750006F905F904F903F902F9008950895CF9362
:10476000DC011E968C911E97811118C01C96ED914C
:10477000FC911D97CF0101961D969C938E931C97DB
:10478000C491C11107C0CD01ED91FC910684F7855C
:10479000E02D19958C2F90E0CF91089590E080E066
:1047A000FBCFFC01968581E08927089581E008957B
:1047B00080E008950F931F9320919C102130E1F425
:1047C00000919410109195102091961030919710AF
:1047D00040919010509191106091921070919310AF
:1047E000041715072607370759F4DC01ED91FC91F2
:1047F0000684F785E02D199580E01F910F910895AB
:1048000081E0FBCF90919C10915081E0933608F0AD
:1048100080E00895DC011C968D919C91DC01ED9166
:10482000FC910190F081E02D1994DC011C968D9192
:104830009C91DC01ED91FC910284F385E02D1994AB
:10484000DC011C968D919C91DC01ED91FC91008422
:10485000F185E02D199521E0892B09F420E0822FC4
:104860000895CF93DF93682F809122028823B9F0B7
:10487000C62FD0E080912F02D817F4F4ED2FEE0F61
:10488000FF0BE95DFD4F80819181DC01ED91FC9191
:104890000088F189E02D6C2F1995DF5FEBCF8091B7
:1048A0001C0290911D02DC01ED91FC910088F189C0
:1048B000E02DDF91CF911994DF91CF9108958091F0
:1048C0004D0C90914E0C9C01181619060CF03FC02F
:1048D0002150310930934E0C20934D0C209108014A
:1048E0002E7F20930801479820911D0D2E7F209345
:1048F0001D0D209109012270181619065CF5809192
:104900000B01826080930B01439A83E290E0FC01EB
:104910003197F1F730910B01386030930B01419AD8
:10492000E3E0F0E03197F1F788988E9830910B0131
:10493000377F30930B0141980197F1F780910B017C
:10494000222379F0826080930B01439A08952F5FB0
:104950003F4FC0CF80910B018D7F80930B01439817
:10496000D4CF8D7F80930B01439808954F925F922F
:104970006F927F928F929F92AF92BF92CF92DF926F
:10498000EF92FF92CF93C82F6091B40C7091B50C49
:104990008091B60C9091B70C0E94C1ED2091EB0C68
:1049A0003091EC0C4091ED0C5091EE0C0E9420EEF9
:1049B0006B017C016091B80C7091B90C8091BA0CBC
:1049C0009091BB0C8090810490908204A09083040D
:1049D000B0908404681979098A099B090E94C1ED85
:1049E0002091EF0C3091F00C4091F10C5091F20CB1
:1049F0000E9420EE20912404309125044091260449
:104A0000509127040E9462EF2B013C016091B00C91
:104A10007091B10C8091B20C9091B30C0E94C1EDD9
:104A20002091E70C3091E80C4091E90C5091EA0C90
:104A30000E9420EE20912A0C30912B0C40912C0CDE
:104A400050912D0C0E9462EF4B015C018092C00CD2
:104A50009092C10CA092C20CB092C30C20912E0C6B
:104A600030912F0C4091300C5091310CC701B601A0
:104A70000E9462EF6B017C01C092C40CD092C50C05
:104A8000E092C60CF092C70C2091320C3091330C9E
:104A90004091340C5091350CC301B2010E9462EF79
:104AA0006093C80C7093C90C8093CA0C9093CB0C84
:104AB000CC23C1F08092410C9092420CA092430C06
:104AC000B092440CC092450CD092460CE092470C38
:104AD000F092480C6093490C70934A0C80934B0CF5
:104AE00090934C0CCF91FF90EF90DF90CF90BF90C0
:104AF000AF909F908F907F906F905F904F900895B0
:104B0000CF93DF93FC0126853785D901A05CBF4F89
:104B10009C919F5F9F73E901CF5BDF4F888189176D
:104B2000E9F3AC91A20FB32FB11D6C93A685B785A5
:104B3000A05CBF4F9C93A689B7898C91958D21E08D
:104B400030E001C0220F9A95EAF7822B8C9381E026
:104B500090E0DF91CF910895DC011E968D919C919C
:104B6000FC01E05CFF4F8F5B9F4F3081DC012C919B
:104B70003213FBCF0895FC0184859585FC01E05834
:104B8000FF4F308131962081321759F0A081A80F54
:104B9000B92FB11D8C9190819F5F9F77908390E09A
:104BA00008958FEF9FEF0895FC0184859585FC01A2
:104BB000E058FF4F308131962081321739F0E08183
:104BC000E80FF92FF11D808190E008958FEF9FEF9E
:104BD0000895FC0124853585F901E058FF4F808157
:104BE0002F573F4FF901208190E080589F4F821B43
:104BF00091098F7799270895DC01CB01F894AA23B6
:104C0000E1F49F3FD1F01092CA031092CB031092AF
:104C1000CC03A0918400B091850024E6A20FB11DC1
:104C20008A179B0728F4B0938900A093880012C0CC
:104C300090938900809388000DC09058A040809385
:104C4000CA039093CB03A093CC03B0E8B093890040
:104C50001092880008954F925F92EF92FF920F9307
:104C6000811520E2920708F07FC0811522E09207AB
:104C700008F050C08A30910510F48AE090E040E0DE
:104C800054E264EF70E0EE24FF187723A1F466236A
:104C900009F012C001E1441F551F0A9509F431C003
:104CA000EE1CFF1CE81AF90A20F4E80EF91E88949D
:104CB000F2CF0894F0CF12C009E1441F551F661FC0
:104CC0000A9509F41EC0EE1CFF1CE81AF90A20F42C
:104CD000E80EF91E8894F1CF0894EFCF01E2441F4B
:104CE000551F661F771F0A9509F40BC0EE1CFF1CA9
:104CF000E81AF90A20F4E80EF91E8894F0CF089417
:104D0000EECFCB01642F752F0F91FF90EF905F9046
:104D10004F900895E8EDFBE2282F2F719695879527
:104D20009695879596958795969587958E7FE80FAA
:104D3000F91F459155912A0105904018059050089A
:104D4000249DC001259D900DE12D880F991FEE1F18
:104D5000880F991FEE1F880F991FEE1F491B5E0BCE
:104D6000662777271124CDCFE6EBFBE29C013F704D
:104D70009695969596959E7FE90FF11D45915591D3
:104D80002A010590401805905008249DC001359DCA
:104D9000E02D259D900DE11D349D900DE11D907F2E
:104DA0009295E2958E2F807F982BEF70491B5E0BBA
:104DB000662777271124A5CF90E080E008954F92D1
:104DC0005F926F927F928F929F92AF92BF92CF929B
:104DD000DF92EF92FF920F931F93CF93DF93EC013B
:104DE0008981853308F0A4C0823308F0AAC08D30D1
:104DF00008F096C029E130E0813060F0EA81F0E00F
:104E0000EE0FFF1FE85FF34F408151812CEF3FE031
:104E1000241B350B3D832C836C817D81813108F00F
:104E20009CC08E3030F48D3008F0CEC0813008F454
:104E3000BFC08150282F30E0F901EC5DF44D949112
:104E4000990FF901EE0FFF1FEC5FF44D259134919E
:104E5000F901E590F490F9013296059114914CEF27
:104E60005FE0FA01E61BF70BBF01B12CA12C82E039
:104E7000891708F000C1E82FF0E0EE0FFF1FE20FE6
:104E8000F31FC590D490E1E0E80FF0E08E5FEE0FE5
:104E9000FF1FE20FF31FA590B4906C157D050CF079
:104EA00090C06E197F09072E000C880B990B0E9489
:104EB000C1ED2B013C01B501601B710B072E000CED
:104EC000880B990B0E94C1ED9B01AC01C301B2019B
:104ED0000E9420EE4B015C01B6016E197F09072E7E
:104EE000000C880B990B0E94C1ED9B01AC01C50120
:104EF000B4010E942CF06B017C01B801110F880BEA
:104F0000990B0E94C1ED9B01AC01C701B6010E9443
:104F100063EF20E030E040E05EE30E9420EEDBC083
:104F20008D3079F0813108F469CF2FEF3FE072CFF7
:104F3000843680F4813608F061CF94EC980F92307B
:104F4000A0F7EA81F0E0EE0FFF1FE85FF34F20814A
:104F5000318160CF8436A9F3E8CF8C3309F492C055
:104F6000A8F49EEC980F933078F1DF91CF911F91C8
:104F70000F91FF90EF90DF90CF90BF90AF909F90F8
:104F80008F907F906F905F904F9008958E3309F4CB
:104F9000A7C008F488C0843641F7072E000C880BA0
:104FA000990B0E94C1ED20E030E04AEF53E474C059
:104FB00080E090E0A8ECB1E48E839F83A887B98756
:104FC000D4CF8501760154CF823308F44FC08E527E
:104FD00090E0FC01EC5DF44D2491220FFC01EE0FFA
:104FE000FF1FEC5FF44D85919491FC01C590D49026
:104FF000FC01329605911491B12CA12C32E03217AC
:1050000008F039C0E32FF0E0EE0FFF1FE80FF91FA3
:10501000E590F490E1E0E30FF0E03E5FEE0FFF1F5C
:10502000E80FF91FA590B4906E157F050CF56C196B
:105030007D09072E000C880B990B0E94C1ED2B01F6
:105040003C01B501601B710B072E000C880B990BFE
:105050000E94C1ED9B01AC01C301B2010E9420EE90
:105060004B015C01B7016C197D0939CF8150B0CF7C
:1050700085016701C4CFB501BB0C880B990B0E9459
:10508000C1ED47CF072E000C880B990B0E94C1ED94
:1050900020E030E04AE754E40E9420EE20E030E0D7
:1050A00040E859E33ACF072E000C880B990B0E9479
:1050B000C1ED20E030E04AE754E40E9420EE20E019
:1050C00030E040E859E30E9420EE20E030E04AE77B
:1050D00053E40E9462EF6E837F838887998745CF70
:1050E000072E000C880B990B0E94C1ED20E030E0E8
:1050F0004AEF53E40E9420EE20E030E040E859E31C
:105100000E9420EE20E030E048E452E4E2CF8F92AB
:105110009F92AF92BF92EF92FF921F93CF93DF9334
:10512000FC0115A912FD2DC07B01EC018284938442
:10513000A484B584A50194016681778180859185D9
:105140000E9462EF9F7720E030E040E85FE30E943A
:1051500063EF20E030E040EA51E40E9476F1181657
:1051600084F0F70180819181A281B3818EAB9FABE6
:10517000A8AFB9AF8AAE9BAEACAEBDAE197F14601E
:105180001DABDF91CF911F91FF90EF90BF90AF903B
:105190009F908F900895FC0195A991FD14C0DB01AB
:1051A0004D915D916D917C9146AB57AB60AF71AF06
:1051B000468157816085718542AF53AF64AF75AF4B
:1051C000997F926095AB08958091C80287FD07C0D2
:1051D00061E09091C902911160E00C942ED2089583
:1051E0000F931F93CF93DF931F921F92CDB7DEB71C
:1051F0008C010196F80120812032D1F34AE050E081
:10520000BE016F5F7F4FC8010E9470EC29813A8117
:105210000217130719F460E070E0CB010F900F90B4
:10522000DF91CF911F910F9108950F931F93CF930B
:10523000DF931F921F92CDB7DEB78C010196F80164
:1052400020812032D1F3BE016F5F7F4FC8010E94E1
:105250001BEB29813A810217130719F460E070E013
:10526000CB010F900F90DF91CF911F910F91089577
:105270000C9472F30C9472F30C9472F32FB7F894AD
:105280006091F80B7091F90B8091FA0B9091FB0BE8
:105290002FBF08951F920F920FB60F9211242F93D4
:1052A0003F938F939F93AF93BF938091F80B90910F
:1052B000F90BA091FA0BB091FB0B3091F70B23E0A7
:1052C000230F2D3758F50196A11DB11D2093F70B23
:1052D0008093F80B9093F90BA093FA0BB093FB0B10
:1052E0008091FC0B9091FD0BA091FE0BB091FF0BF8
:1052F0000196A11DB11D8093FC0B9093FD0BA09313
:10530000FE0BB093FF0BBF91AF919F918F913F9197
:105310002F910F900FBE0F901F90189526E8230F26
:105320000296A11DB11DD2CFCF93DF93EC01E9818D
:10533000FA81908181819CBD8DBDE981FA8160E017
:1053400082810E942ED281E08B83DF91CF910895DC
:105350008EBD0DB407FEFDCF08958FEF8EBD0DB449
:1053600007FEFDCF8EB50895CF93DF93FC01238117
:10537000222359F0EC010180F281E02D61E082816D
:105380000E942ED28FEFE4DF1B82DF91CF91089530
:105390000F931F93CF93DF938C01862FEA01D8DF01
:1053A00088818EBD8981FE013296DE5F0DB407FED5
:1053B000FDCF8EBDEC17FD0711F08191F7CF0DB435
:1053C00007FEFDCF8FEFC4DF8FEFC2DFC6DFF8012E
:1053D00084838F71853051F087E58083C801C4DFF5
:1053E00080E0DF91CF911F910F91089581E0F9CF77
:1053F000DF92EF92FF920F931F93CF93DF938C0175
:10540000C62FD22FF32EE42ED52EFC0183818111DD
:1054100002C0C80189DF0E9409C98C2F806498DF0F
:105420008D2D96DF8E2D94DF8F2D92DF8D2F90DFC7
:1054300087E8C11101C085E98BDFCC3009F48DDF2D
:10544000C0E08BDFF801848387FF04C0CF3F11F0F9
:10545000CF5FF7CFDF91CF911F910F91FF90EF902A
:10546000DF9008950F931F93CF93DF93EC01890191
:105470008D81833039F089E0440F551F661F771FF7
:105480008A95D1F79A01AB0168E1CE01B1DF88239B
:1054900031F082E38883CE0167DF10E01BC0A801F2
:1054A0006EEFCE0175DF8823B1F30E9409C9182F72
:1054B0008AE5112379F320E030E0A9016DE0CE0107
:1054C00097DF882311F089E2E5CF47DF8111FBCF19
:1054D000CE014ADF812FDF91CF911F910F91089567
:1054E0000F931F93CF93DF93EC0189018D8183305C
:1054F00039F089E0440F551F661F771F8A95D1F751
:105500009A01AB0161E1CE0173DF882331F080E3C2
:105510008883CE0129DF10E009C0B801CE010E94C6
:10552000C5C8182F8823A9F3CE011EDF812FDF9174
:10553000CF911F910F910895A1DECB010895EF92B5
:10554000FF921F93CF93DF93FC01208111E020FF96
:1055500013C0EC017C01F7E0EF0EF11C4B815C8184
:105560006D817E81E981FA819701808191817ADF65
:10557000182F811108C010E0812FDF91CF911F916A
:10558000FF90EF900895888181FD04C088818E7F0F
:105590008883F2CFE981FA814B815C816D817E81C4
:1055A00084859585A685B785480F591F6A1F7B1F7F
:1055B00097018081918156DF8111E8CFDCCFCF92B6
:1055C000DF92EF92FF921F93CF93DF93EC016A017A
:1055D0007B01122F8B819C81AD81BE818C159D0535
:1055E000AE05BF05A9F0CE01AADF81110AC090E087
:1055F00080E0DF91CF911F91FF90EF90DF90CF90EF
:10560000089512FF0CC01882CB82DC82ED82FE82EC
:1056100013708881182B1883CE010796EACFE98191
:10562000FA819E01295F3F4FB701A60180819181D8
:1056300057DF8111E8CFDBCF8F929F92AF92BF925D
:10564000CF92DF92EF92FF920F931F93423051055A
:105650006105710560F480E01F910F91FF90EF905C
:10566000DF90CF90BF90AF909F908F900895FC01F6
:10567000C08CD18CE28CF38CC416D506E606F706F6
:1056800050F3480159016A017B018581803239F567
:1056900084899589A689B78917E076956795579586
:1056A00047951A95D1F7480F591F6A1F7B1F23E0B2
:1056B000CF01809684DF009771F2E894C7F8DD246B
:1056C000EE24FF24CC0CDD1CCC0CDD1C8C0D9D1DB0
:1056D000FC0180829182A282B38281E0BDCF8031C1
:1056E00009F0B9CF44895589668977894D0D511DD7
:1056F000611D711D23E0CF01809661DF009709F4E1
:10570000AACFDD24EE24FF24CC0CDD1CC80ED91E4C
:10571000F60111830083E1CFCF92DF92EF92FF92E7
:105720000F931F93CF93DF934230510561057105AD
:1057300050F48FEFDF91CF911F910F91FF90EF9079
:10574000DF90CF900895FC01C08CD18CE28CF38C5B
:10575000C416D506E606F70660F389016A017B01E7
:10576000EC0185818032B1F584899589A689B78954
:10577000E7E07695679557954795EA95D1F7480FF5
:10578000591F6A1F7B1F22E0CE01809618DF009709
:1057900081F2E894C7F8DD24EE24FF24CC0CDD1C54
:1057A000CC0CDD1C8C0D9D1DFC0180819181A281A2
:1057B000B381BF70488D598D6A8D7B8D481759070D
:1057C0006A077B0730F1F80180839183A283B3835A
:1057D00081E0B0CF803109F0ACCF4489558966892A
:1057E00077894D0D511D611D711D22E0CF018096FD
:1057F000E6DE009709F49DCFDD24EE24FF24CC0CD7
:10580000DD1CC80ED91EF60180819181B0E0A0E0B8
:10581000D1CF80E08FCF9F92AF92BF92CF92DF9295
:10582000EF92FF920F931F93CF93DF9300D01F92BD
:10583000CDB7DEB75C016A017B019E012F5F3F4F50
:10584000B701A601C50168DF982E87FD2DC000E0D5
:1058500010E09801B701A601C501EEDE882321F111
:10586000F5014085518562857385C416D506E60627
:10587000F70620F4C086D186E286F386C980DA80F6
:10588000EB80FC809110D9CF0F900F900F900F906C
:10589000DF91CF911F910F91FF90EF90DF90CF900C
:1058A000BF90AF909F90089580E0EECF3F924F92CF
:1058B0005F926F927F928F929F92AF92BF92CF92A0
:1058C000DF92EF92FF920F931F93CF93DF9300D05D
:1058D00000D01F921F92CDB7DEB74C01DC011296AB
:1058E0008C911297806812968C9312971696AD90B1
:1058F000BC9017971C964D905D906D907C901F9773
:10590000411451046104710409F059C0D50118967D
:105910008D919D910D90BC91A02D8D839E83AF8321
:10592000B887CD80DE80EF80F884BFEFCB1ADB0A2A
:10593000EB0AFB0AF501808D918DA28DB38D8C153C
:105940009D05AE05BF0528F482E0C82ED12CE12CC0
:10595000F12C9E012F5F3F4FB701A601C501DCDE90
:1059600087FD13C0882341F089819A81AB81BC8176
:10597000892B8A2B8B2B41F18D819E81AF81B8853C
:10598000C816D906EA06FB0681F6312C832D289627
:105990000FB6F894DEBF0FBECDBFDF91CF911F9140
:1059A0000F91FF90EF90DF90CF90BF90AF909F90BE
:1059B0008F907F906F905F904F903F9008954D82B1
:1059C0005E826F827886ADCF0FEF1FEF2FEF3FE043
:1059D000B701A601C50130DE382E8823B1F241148B
:1059E00051046104710471F097018601B301A201B1
:1059F000C50122DE882349F2F401C486D586E686F5
:105A0000F786C4CFD5011896CD92DD92ED92FC9227
:105A10001B97F2CFAF92BF92CF92DF92EF92FF929D
:105A20000F931F93CF93DF93EC01888185FF0DC007
:105A300010E0812FDF91CF911F910F91FF90EF9098
:105A4000DF90CF90BF90AF90089588899989AA89F7
:105A5000BB8981159E4FAF41B10550F7CE0126DFBE
:105A6000182F882329F3EE81FF81CC84DD84EE8416
:105A7000FF8432E0C31AD108E108F108848104C030
:105A8000CC0CDD1CEE1CFF1C8A95D2F78089918915
:105A9000A289B389C80ED91EEA1EFB1E25E0B701F4
:105AA000A601CF0180968BDD5C01892B09F4C0CF64
:105AB00080E092E0F5019C01119221503040E1F725
:105AC00001E0EE81FF818281081778F49501B7012A
:105AD000A601400F511D611D711D80819181C2DCA5
:105AE000882309F4A5CF0F5FECCF90E0B0E0A0E0F1
:105AF00029E0880F991FAA1FBB1F2A95D1F7488953
:105B000059896A897B89840F951FA61FB71F888BC7
:105B1000998BAA8BBB8B8DCFFC019C01255F3F4FDE
:105B200080E080FB879587F99191890F2E173F07B9
:105B3000C1F708954F925F926F927F928F929F92DA
:105B4000AF92BF92CF92DF92EF92FF920F931F938B
:105B5000CF93DF93EC014A015B014C845D846E843A
:105B60007F84A881AA2309F485C0488959896A8954
:105B70007B89481559056A057B0569F081149104F4
:105B8000A104B10451F41C861D861E861F86888AD6
:105B9000998AAA8ABB8A81E072C0A3FF58C0088D87
:105BA000198D2A8D3B8D081519052A053B0508F42A
:105BB00061C0EE81FF81848190E009968A019B019A
:105BC0000150110921093109082E04C03695279585
:105BD000179507950A94D2F775016401B1E0CB1AC5
:105BE000D108E108F10804C0F694E794D794C7946B
:105BF0008A95D2F7C016D106E206F30628F0452BA7
:105C0000462B472B09F051C0A6FF4AC0848D958DC5
:105C1000A68DB78D8C879D87AE87BF878E01045F69
:105C20001F4FC114D104E104F10409F4B0CF4C8535
:105C30005D856E857F8598018E819F816DDD91E008
:105C4000C91AD108E108F10818165CF313C0A5FFC2
:105C5000B0CFEE81FF818681978125E0880F991F63
:105C60002A95E1F7B0E0A0E088159905AA05BB05E3
:105C700008F08DCF4C865D866E867F8680E0DF9152
:105C8000CF911F910F91FF90EF90DF90CF90BF9039
:105C9000AF909F908F907F906F905F904F900895FE
:105CA0008C8D9D8DAE8DBF8DB5CFC01AD10AE20A05
:105CB000F30AB4CFEF92FF920F931F93CF93DF932A
:105CC0001F92CDB7DEB77C01962FF701408951892D
:105CD000628973898A019B0185E03695279517951E
:105CE00007958A95D1F70F7011F0911129C0BE0167
:105CF0006F5F7F4FC7010E941FC9813051F090E054
:105D000080E00F90DF91CF911F910F91FF90EF9066
:105D10000895F70180899189A289B3894F96A11DC1
:105D2000B11D808B918BA28BB38BF70186819781FC
:105D30008796F0E20F9F90011124820F931FE1CF0D
:105D4000405E5F4F6F4F7F4F408B518B628B738BE9
:105D5000ECCFFC01808181110FC080E2DF01982F20
:105D60001D929A95E9F777836683DB0115969C91DE
:105D7000903129F0903211F080E0089580E4808322
:105D800081E082830895CF92DF92EF92FF920F938A
:105D9000CF93DF93EC0180E2DE011D928A95E9F753
:105DA000FB01868197819F838E835D834C83C48CA6
:105DB000D58CE68CF78CC886D986EA86FB86FA01F4
:105DC000EF70FF27DC01979645E0EE0FFF1F4A9525
:105DD000E1F7BD016E0F7F1FDB011B963C9133FD88
:105DE0004EC0AC014E0F5F1FDA01D2963C91377165
:105DF0003883DB011B964C91487111F4386038836D
:105E00000B83322F327319F038813171C1F5322F83
:105E10003F703A83DC0193964D915D916D917C9139
:105E200096974C8B5D8B6E8B7F8BE80FF91F43AD84
:105E300054AD70E060E0BA0155274427DF01AF5B45
:105E4000BF4FCD90DC90F12CE12C4C295D296E29BF
:105E50007F2924FF17C0411551056105710561F4C3
:105E60008A8180688A8381E0DF91CF910F91FF90D2
:105E7000EF90DF90CF900895CEDC8111F1CF1882A2
:105E800080E0F2CF4C8F5D8F6E8F7F8FED5BFF4F89
:105E900080819181A281B381888F998FAA8FBB8FD6
:105EA000E2CFCF93DF93EC01262F4C895D896E8979
:105EB0007F898E819F81809682DB009771F02C8193
:105EC0003D812F70332745E0220F331F4A95E1F7BC
:105ED000820F931FDF91CF91089590E080E0FACF79
:105EE0009F92AF92BF92CF92DF92EF92FF920F9369
:105EF0001F93CF93DF93CDB7DEB7A0970FB6F8947B
:105F0000DEBF0FBECDBF19821A82DC012C9123FFA8
:105F100015C012962C9121FF11C08C01FC01448DFB
:105F2000558D668D778D411551056105710541F4DB
:105F300061E0C801B6DF7C01009741F480E06FC0EA
:105F40008681978168DC8111F3CFF8CFE5DD982E4B
:105F500085EEF7018083D8011C9216968D919C9155
:105F60008096EDDA882351F3F8019381992309F49F
:105F700056C080859185A285B385668177819E0113
:105F80002F5F3F4F69010097A105B10509F059C086
:105F9000C901DFDE882391F2EE24E394F12C25EE93
:105FA000A22ED80113968C9113978E1538F2149661
:105FB0004D915C914E195F0970E060E085E0440FFF
:105FC000551F661F771F8A95D1F7C601B3DD882359
:105FD00009F4B4CF60E0C6016DDEFC01892B09F441
:105FE000ADCF83858F3009F0A9CF9081892F8F7134
:105FF000E812A4CF85858911A1CFA082D801169679
:10600000ED91FC9180A1816080A3BFEFEB1AFB0AA8
:1060100096FFC7CFF80186819781809690DAA09687
:106020000FB6F894DEBF0FBECDBFDF91CF911F91A9
:106030000F91FF90EF90DF90CF90BF90AF909F9027
:1060400008952CE1F60111922A95E9F720E12983C0
:1060500021E02B8378876F838D8F9E8FAF8FB8A3BE
:106060009BCFCF93DF93FC012081211104C081E0FD
:10607000DF91CF910895EC01828187FF26C061E016
:10608000CF010FDFFC01892B29F48981816089838D
:1060900080E0EECF8081853EC1F3888183FF08C018
:1060A000888D998DAA8DBB8D848F958FA68FB78F84
:1060B0008C8D9D8D938F828F8C8D9D8DAE8DBF8DA0
:1060C000B58BA48B8A818F778A838E819F818096FE
:1060D00036DA8823D1F2CBCF2F923F924F925F9244
:1060E0006F927F928F929F92AF92BF92CF92DF92E8
:1060F000EF92FF920F931F93CF93DF9300D000D0C6
:1061000000D01F92CDB7DEB79E838D833B015A83AB
:106110004983DC018C9183FFE6C012968C9181FF4C
:10612000E2C082FDD4C0E981FA81AF0170E060E095
:10613000ED81FE8180899189A289B38980959095AE
:10614000A095B09584179507A607B70708F4CBC0AC
:10615000C980DA8022242A94322C21013C96FC83C7
:10616000EB83ED81FE814089518962897389C11475
:10617000D10409F472C1868197818A019B0169E08B
:1061800036952795179507956A95D1F7DC011396F3
:10619000EC910E237A01B1E0FB2201111DC0ED81CB
:1061A000FE814485558566857785E114F10409F003
:1061B0008CC1411551056105710509F49FC02B8102
:1061C0003C81AADA87FD8FC0811106C08D819E8136
:1061D0006DDB882309F487C0AD81BE811696ED91F1
:1061E000FC9117971C964D915D916D917C911F9735
:1061F0004250510961097109848104C0440F551F3F
:10620000661F771F8A95D2F780899189A289B38901
:10621000840F951FA61FB71FAC01BD01400F511D74
:10622000611D711DE114F10429F4C114B2E0DB0613
:1062300008F084C080E092E08E199F0986018C15D9
:106240009D0508F48C01E114F104A1F4AD81BE8137
:1062500050968D909D90AD90BC90539758968D918F
:106260009D910D90BC91A02D25E088169906AA0657
:10627000BB0608F421E0CF018096A1D9009799F1DF
:10628000A801B3018E0D9F1D0E940CF4E00EF11EBB
:10629000E114B2E0FB0641F4ED81FE818681978135
:1062A00080964DD98823F9F0ED81FE81808991890E
:1062B000A289B389800F911FA11DB11D808B918B85
:1062C000A28BB38B600E711EC01AD10A4ACFAD816A
:1062D000BE8158964D915D916D917C915B97CD01FA
:1062E00029DC811120CFAD81BE8111968C9111974F
:1062F000816011968C938FEF9FEFC8C0ED81FE8176
:10630000848D958DA68DB78D0097A105B10579F483
:10631000CF01CCDA882339F3ED81FE818485958520
:10632000A685B785848F958FA68FB78F55CFED81C2
:10633000FE8184879587A687B7874ECF83A194A1D6
:10634000A5A1B6A1C11424E0D20608F46DC096013F
:10635000232F332726958280801A912C2815390502
:1063600008F44901481759076A077B0770F0880D40
:10637000991DA11DB11D481759076A077B0728F40D
:1063800010A223A234A245A256A2AD81BE811696C8
:10639000ED91FC91E080F180F7018581833039F047
:1063A00099E0440F551F661F771F9A95D1F79A0100
:1063B000AB0169E1C7011CD8882351F083E3D70101
:1063C0008C93C7010E94B429C7010E94B4298BCFC6
:1063D000530110E000E008151905A1F00E9409C959
:1063E000811104C08AE5F7018083EBCFA5016CEF32
:1063F000C7010E94C829882321F30F5F1F4FFEEFBA
:10640000BF1AE9CF0E9409C9882351F0102F002735
:10641000110F8DEF0E94A829C7010E94B42944CF13
:1064200086E5D7018C93D0CF481759076A077B07B9
:1064300029F410A223A234A245A256A2AD81BE81A6
:106440001696ED91FC919301808191810BD8882360
:1064500009F449CF00E012E027CFED81FE81808D65
:10646000918DA28DB38D84179507A607B70738F4D1
:106470008281408F518F628F738F80688283ED811C
:10648000FE81828183FD1BC089819A812A960FB685
:10649000F894DEBF0FBECDBFDF91CF911F910F915A
:1064A000FF90EF90DF90CF90BF90AF909F908F9034
:1064B0007F906F905F904F903F902F9008958D81C7
:1064C0009E81CFDD8111E0CF0ECFFC0142505109FA
:1064D00061097109848104C0440F551F661F771F2D
:1064E0008A95D2F780899189A289B389480F591F6B
:1064F0006A1F7B1F9FCE0496EFCDCF93DF931F9231
:10650000CDB7DEB7698341E050E0BE016F5F7F4FDA
:106510000496E2DD0F90DF91CF910895CF93DF9342
:10652000EC019FDD1882DF91CF910895049699CDFB
:10653000E091F60BF0E0EE0FFF1FEC5BFF4C2591B6
:106540003491FC01EE0FFF1FE20FF31F8591949130
:106550000895E2E4F0E39FEF482F880F550B249154
:106560002F3F49F09F3F21F02417150609F0292FEE
:106570003196922FF4CF9093F60B089590910201EB
:10658000662309F442C092609093020184FF3FC0E9
:10659000119A85FF3EC0139A86FF3DC0159A87FF6A
:1065A0003CC0179AE3E0F0E0DF011197F1F790911A
:1065B00002019160909302013197F1F790910201ED
:1065C0009E7F9093020180FF2AC0119A81FF29C00B
:1065D000139A82FF28C0159A83FF27C0179A83E079
:1065E00090E0FC013197F1F72091020121602093A6
:1065F00002010197F1F7809102018E7F80930201E1
:106600008BE891E00197F1F708959D7FBDCF119838
:10661000C0CF1398C1CF1598C2CF1798C3CF119888
:10662000D5CF1398D6CF1598D7CF1798D8CF82301B
:10663000E9F0119A139A15981798000000000000CD
:10664000000000000000809102018160809302013F
:1066500083E090E00197F1F7809102018E7F8093B3
:10666000020183EC90E00197F1F708951198E2CFD1
:10667000FC013596E4910E2E000CFF0B309749F08B
:106680002091AA0C3091AB0C2E233F232E173F07ED
:1066900079F4FC01379685919491009759F02091F7
:1066A000AA0C3091AB0C2823392381E0232B19F05D
:1066B00080E0089581E0089540E050E0BA013ACAD0
:1066C0002F923F924F925F926F927F928F929F9202
:1066D000AF92BF92CF92DF92EF92FF920F931F93F0
:1066E000CF93DF9300D000D000D0CDB7DEB74C0100
:1066F0007F836E83FA01DB018C918077D1F480E097
:1067000029960FB6F894DEBF0FBECDBFDF91CF91B3
:106710001F910F91FF90EF90DF90CF90BF90AF90BF
:106720009F908F907F906F905F904F903F902F90B1
:106730000895D4018C918111E2CFA180B280808133
:10674000837033243394882349F0C5010C966DE09F
:1067500070E00E947FF233243394360E2A837F0147
:10676000EE81FF81F987E887CF01A6DF1C821D82B9
:106770001982212C10E000E01B8297012A5F3F4F15
:106780003F832E83A885B98550964D905D906D907E
:106790007C90539795E076946794579447949A9594
:1067A000D1F7620161E0CD0185DA009709F05BC0A5
:1067B000E885F98581818111A2CF8A818274823432
:1067C00009F09DCF112311F0CC80DD801315E8F482
:1067D00060E0888599856EDA892B09F0E0C0E8854C
:1067E000F985818181118BCF8885998513D988237B
:1067F00009F485CFA885B9851696ED91FC91828123
:10680000823018F4105F131578F3BB81BB2309F4B1
:10681000F4C0F701558002E010E08EE7482E370102
:10682000F6E06F0E711CD70111962D913C911297D5
:10683000C801820F931F1396ED91FC912E0F3F1FFD
:106840002E173F0709F4ADC0AC01B5E0440F551F4A
:10685000BA95E1F7840F951F4191042E000C550B5A
:1068600084279527EDCFDC012C91253E11F02111D5
:106870000EC0111102C04C825D82131508F41F5F17
:10688000222309F49ACF253E21F400E07BCF131593
:1068900050F12E32D1F3FC0133853F3009F05AC05C
:1068A000011123C026FF6ECF022F0F71F585F983EA
:1068B000202EE22DE150FF0BAF01FDE0F49F90018F
:1068C000F59F300D11242A153B05F8F6FC01D12C5B
:1068D00064E06D1590F081819281A216B306B1F447
:1068E000892B99F64FCF10E0D4CF2A942211CDCF27
:1068F0002585B9812B17E9F2C8CF8AE08D1518F0EC
:1069000084819581EACF86819781E7CF8F3F91057A
:1069100011F008F0BACF4FEB480F4A3108F4805E0F
:10692000B9016F5F7F4FD70113964D915C91240F92
:10693000351FD9019C912FEB290F2A3108F4905E65
:106940009813A3CFD3943296BDE0DB1609F41ACF87
:106950009B01BECF33FD99CF002389F0E1E02E12D9
:10696000CECEDAD8F9818F13CACEBA81B7FDC7CEA1
:106970002A81A60168857985C40105DAC1CE4BE07C
:1069800050E06E817F810E94FFF3892B09F0FACEDF
:10699000D7018C9180FFE9CF31E03B83F3CE1F5FBD
:1069A00015CFB3E0B51510F4A3E05A2E34E0350D41
:1069B000282F2F702A3008F085C0205DF701E30FE3
:1069C000F11D2683F4E096958795FA95E1F731500D
:1069D000531670F3F701E50DF11D46828885998500
:1069E0006BDE61E08885998565D9009709F06CC0F8
:1069F000E885F9858181811182CEA60170E060E091
:106A0000E5E0440F551F661F771FEA95D1F788858B
:106A1000998590D8882309F472CE0FEF030D102FBB
:106A20003FE0532E3701B6E06B0E711C4DE0442E53
:106A3000112309F475C060E0888599853BD96C0104
:106A4000892B09F45CCEA885B9851696ED91FC9149
:106A500080A1816080A3312E101302C0689436F8A3
:106A6000F601308253861486C30156D8D6011D968E
:106A70008C931D975B961C921E925A97F701238167
:106A80003481832D8F718150990B489EA001499EBE
:106A9000500D1124F60160E04A155B0570F5D9012F
:106AA000A40FB51F8C91082E000C990B653080F552
:106AB000928381836F5F4F5F5F4F32966D3061F7D6
:106AC0001150B6CF295C7ACFDC012C91222309F436
:106AD00094CF1B962C9123FD84CF4BE050E0BC015A
:106AE000C3010E94FFF3892B09F07BCF0F5F1F4F7B
:106AF0000436110509F097CE02CE81E090E0A4168D
:106B0000B50611F490E080E0919581959109CECF82
:106B10006B3018F495838483CDCF97838683CACF57
:106B2000A885B98550964D905D906D907C90539757
:106B300060E0CD01BFD8009709F4E1CD25E076945F
:106B40006794579447942A95D1F7620120E2FC019B
:106B500011922A95E9F7F70136962BE0DC010190B6
:106B60000D922A95E1F7D7012C912871FC01248719
:106B700021E238E2318B208B40E058E0578746878E
:106B8000338B228B318F208F578B468BA885B9850D
:106B90001696ED91FC9180A1816080A3E9CEDF92F1
:106BA000EF92FF920F931F93CF93DF93CDB7DEB792
:106BB000E3970FB6F894DEBF0FBECDBF7C018B010B
:106BC0005BAB4AABD22E19821A82FC0180818823EA
:106BD00079F080E0E3960FB6F894DEBF0FBECDBF2C
:106BE000DF91CF911F910F91FF90EF90DF9008956B
:106BF000FB018081807769F3EAA9FBA980818F324C
:106C0000C9F4EAA9FBA980818F3221F43196FBAB4C
:106C1000EAABF7CFF80166817781811103C0C70124
:106C200098D8D8CFCE01019694D8882391F28E01BE
:106C30000F5F1F4FAE014E5C5F4FBE016F5D7F4F18
:106C40008AA99BA90E943D21882309F4C2CFEAA901
:106C5000FBA980818823A9F021E0AE014F5D5F4F41
:106C6000B801C7012DDD882309F4B3CF80E2F70115
:106C7000DE01119601900D928A95E1F7C7014EDC75
:106C8000D6CF2D2DAE014F5D5F4FB801C70118DD86
:106C9000A1CF08950895CF93DF938091380220917A
:106CA0001C0230911D02E0E3F2E0C0E0C817E4F0FE
:106CB000C0E0D0E080913802D817ECF4CF5FC8175D
:106CC0000CF0C0E0EC2FEE0FFF0BE05DFD4F80817C
:106CD0009181DC01ED91FC910284F385E02D199501
:106CE000811109C0DF5FE6CF4191519142175307EF
:106CF00001F3CF5FDBCFEC2FEE0FFF0BE05DFD4F1D
:106D00008081918190931D0280931C0210923D0C12
:106D1000DF91CF910895E0913802A0E3B2E050E016
:106D200040E04E17CCF49A016D917D914F5F5F4F1B
:106D300068177907B1F7E150E0933802F0E0EE0F01
:106D4000FF1FE05DFD4F40815181F901EE0FFF1FF4
:106D5000E05DFD4F51834083E0912F02A7E2B2E056
:106D600050E040E04E17CCF49A016D917D914F5F59
:106D70005F4F68177907B1F7E150E0932F02F0E019
:106D8000EE0FFF1FE95DFD4F40815181F901EE0FCC
:106D9000FF1FE95DFD4F5183408320911C0230911C
:106DA0001D022817390709F476CF0895CF93DF9392
:106DB000FC01268521110CC0EC0181E08687CF0102
:106DC000AADF61E08F859889DF91CF910C94D8D4A8
:106DD000DF91CF91089508951F920F920FB60F92F1
:106DE00011240BB60F928F939F93EF93FF93909183
:106DF000031180910411981310C08091C1008F7D00
:106E00008093C100FF91EF919F918F910F900BBEE6
:106E10000F900FBE0F901F901895E0910411F0E0B5
:106E2000ED53FF4E80818093C600809104118F5FE7
:106E30008F7380930411E6CF1F920F920FB60F92BB
:106E400011240BB60F922F938F939F93EF93FF9381
:106E50009091C600809185118F5F8F772091861168
:106E6000821741F0E0918511F0E0EB5FFE4E9083D8
:106E700080938511FF91EF919F918F912F910F90AA
:106E80000BBE0F900FBE0F901F9018951F920F9280
:106E90000FB60F9211240BB60F921F932F933F93AF
:106EA0004F935F936F937F938F939F93AF93BF9312
:106EB000CF93DF93EF93FF9388B5805C88BD80917B
:106EC0000D04811111C08091E10C809307048111A0
:106ED0002C9A8091E20C80930804882329F08091F9
:106EE00002018062809302018091060481110BC02F
:106EF00080912D0380930504882329F0809102015D
:106F00008064809302018091070490910D0489139D
:106F100003C08F3F09F02C988091050490910604DE
:106F2000891307C08F3F29F0809102018F7B8093E6
:106F300002018091080490910D04891307C08F3FCE
:106F400029F0809102018F7D8093020180910304DA
:106F5000909104040196863821E0920708F0E0C081
:106F6000909304048093030480917A0086FD52C0BC
:106F700020917800309179008091070CE82FF0E0A3
:106F8000AF01440F551FDA01A45FB34F6D917C919F
:106F90001197260F371F2D933C93E05FF34F90819D
:106FA0009F5F9083903288F190910204992311F0B1
:106FB000823058F093E0369527959A95E1F7DA01FB
:106FC000A85FB34F11963C932E93445F534FDA0161
:106FD0001D921C9210828F5F823008F0B1C08093A6
:106FE000070CE091070CF0E0EE57F34CE491809130
:106FF0007B00E3FFA8C0886080937B0080917C00C9
:10700000807EE770E82BE0937C0080917A008064BA
:1070100080937A00809103049091040483709927EF
:10702000039709F056C01FB7F89480912B0D8A7012
:1070300009F04EC080912B0D886080932B0D8091BC
:10704000B60DB4E08B02C00111248F708093B60D91
:10705000349903C082608093B60D369905C0809143
:10706000B60D81608093B60DE091B60D0E2E000C2A
:10707000FF0BE652F24DE4918091B50D8E1B80938B
:10708000B50D329B62C0D0E0C0E0909902C0CAE466
:10709000D4E080916B0D90916C0D8C179D0799F049
:1070A0000E943E2960936D0D70936E0D80936F0D5D
:1070B0009093700DD0936C0DC0936B0D80912B0D40
:1070C000816080932B0D80912B0D877F80932B0DFA
:1070D0001FBF809106048F5F8093060480910D048A
:1070E0008F5F80930D048091AE0C882319F0A895D2
:1070F0001092AE0CFF91EF91DF91CF91BF91AF91C4
:107100009F918F917F916F915F914F913F912F91BF
:107110001F910F900BBE0F900FBE0F901F901895F0
:10712000109204041092030481E080930204809181
:107130000104882309F418CF81508093010414CFEF
:107140001092070C4ECF877F57CFC9EED3E09DCF6B
:10715000F0E0E0E01994E0911E0DF0911F0D81899F
:1071600087FD06C061E09289911160E00C942ED2F7
:107170000895CF92DF92EF92FF92CF93DF93FC01BD
:1071800023812130B1F5EC01C4A0D5A0E6A0F7A081
:1071900020E030E0A901C701B6010E94BBED8823C1
:1071A00041F16E8D70E090E080E00E94BFED20E044
:1071B00030E040E251E40E9420EEA70196010E94D7
:1071C0002CF06DA77EA78FA798AB6F8D70E090E035
:1071D00080E00E94BFED20E030E040E251E40E94F8
:1071E00020EEA70196010E942CF069AB7AAB8BAB25
:1071F0009CABDF91CF91FF90EF90DF90CF900895FF
:107200001F93CF93DF9310E0D0E0C0E0C836D105E4
:1072100021F0CE010E94E7EE180F2196C11588E0FB
:10722000D807A1F7812FDF91CF911F910895CF93B8
:10723000E7DFC82F88E690E00E94E7EE8C1731F078
:107240006C2F88E690E0CF910C9402EFCF910895D7
:10725000CF93DF93EC018991882319F00E943124A8
:10726000FACFDF91CF9108954F925F926F927F9204
:10727000BF92CF92DF92EF92FF920F931F93CF9323
:10728000DF9300D000D000D01F921F92CDB7DEB7A1
:107290006B017C011B868E01055F1F4F8AE0482E23
:1072A000512C612C712C9AE0B92EC701B601A301B3
:1072B00092010E9427EF80E3C80EB29EC0181124ED
:1072C000F801C2928F0169017A01C114D104E1046D
:1072D000F10459F7CF01BCDF2B960FB6F894DEBF4F
:1072E0000FBECDBFDF91CF911F910F91FF90EF9017
:1072F000DF90CF90BF907F906F905F904F900895F8
:10730000CF92DF92EF92FF926B017C01F7FE0BC0F0
:107310008DE20E943124F094E094D094C094C11C7A
:10732000D11CE11CF11CC701B601FF90EF90DF906A
:10733000CF909ACFBC01990F880B990BE1CFCF93D7
:10734000DF93EC01FE0184912196882319F00E94BD
:107350003124F8CFDF91CF9108958F929F92AF9211
:10736000BF92CF92DF92EF92FF92CF93DF936B01A8
:107370007C01D42FAC019B010E9463F2882369F049
:107380008EE29AE2DF91CF91FF90EF90DF90CF9065
:10739000BF90AF909F908F90D2CF46015701E89455
:1073A000B7F82FEF3FEF4FE75FE7C501B4010E9449
:1073B00063F281110DC02FEF3FEF4FE75FE7C5018B
:1073C000B4010E94BBED18161CF48AE29AE2DACFEF
:1073D00020E030E0A901C701B6010E94BBED87FFA4
:1073E00007C08DE20E943124F7FAF094F7F8F09488
:1073F000C0E060E070E080E09FE3DC1741F020E057
:1074000030E040E251E40E942CF0CF5FF6CFA701BC
:1074100096010E9463EF6B017C010E9499F04B0181
:107420005C0122DFCC2379F1C501B4010E94BFEDDC
:107430009B01AC01C701B6010E9462EF6B017C01A8
:107440008EE20E943124C150F0F020E030E040E2B2
:1074500051E4C701B6010E9420EE4B015C010E947D
:1074600094F06B01CB0166DFB601DD0C880B990B44
:107470000E94C1ED9B01AC01C501B4010E9462EF05
:107480006B017C01E0CFDF91CF91FF90EF90DF9017
:10749000CF90BF90AF909F908F900895CF92DF9242
:1074A000EF92FF92CF936A017B01C22F48DF4C2FEE
:1074B000C701B601CF91FF90EF90DF90CF904DCFF5
:1074C000CF92DF92EF92FF926A017B0138DFC70112
:1074D000B601FF90EF90DF90CF9012CFCF93DF9364
:1074E000EB012DDFCE01DF91CF9124CF885C910994
:1074F000883522E0920760F464E670E00E947FF233
:107500006F5F7F4F80E99AE2E9DF80E20C943124DB
:1075100008958DE00E9431248AE00C943124CF93A9
:10752000DF93EC01888180FF0BC08EE40E94312440
:107530006C817D8190E080E0E3DE80E20E94312476
:10754000888181FF09C08DE40E9431248E819F8152
:10755000F1DE80E20E943124888182FF09C087E445
:107560000E94312488859985E5DE80E20E943124DD
:107570008881998191FF0CC084E50E943124FE012D
:10758000EC5AFF4F808190E0D5DE80E20E943124EA
:10759000888183FF08C04A855B856C857D8522E0F4
:1075A00084E89FE27BDF888184FF08C04E855F8589
:1075B0006889798922E081E89FE270DF888185FF10
:1075C00008C04A895B896C897D8922E08EE79FE249
:1075D00065DF888186FF08C04E895F89688D798D57
:1075E00024E08BE79FE25ADF8881998190FF08C0F1
:1075F0004A8D5B8D6C8D7D8D22E088E79FE24EDFAA
:107600008881998192FF07C04E8D5F8D68A179A115
:1076100085E79FE255DF8881998193FF07C04AA1E2
:107620005BA16CA17DA182E79FE24ADF8A8180FF96
:1076300008C04EA15FA168A579A522E08FE69FE270
:107640002DDF8A8181FF08C04AA55BA56CA57DA5B9
:1076500022E08CE69FE222DF8A8182FF08C04EA5ED
:107660005FA568A979A922E089E69FE217DF8A81F0
:1076700083FF08C04AA95BA96CA97DA922E086E620
:107680009FE20CDF8A8184FF08C04EA95FA968AD24
:1076900079AD22E083E69FE201DF8A8185FF08C0A1
:1076A0004AAD5BAD6CAD7DAD22E080E69FE2F6DEDB
:1076B0008A8186FF0AC0FE01FE9640815181628167
:1076C000738122E08DE59FE2E9DE8A8187FF0BC0AE
:1076D000FE01EE5BFF4F408151816281738122E0A8
:1076E0008AE59FE2DBDE8A819B8190FF0BC0FE0171
:1076F000EA5BFF4F408151816281738122E087E51F
:107700009FE2CCDE8A819B8191FF0BC0FE01E65B8C
:10771000FF4F408151816281738122E084E59FE2C5
:10772000BDDE8A819B8192FF0BC0FE01E25BFF4FB1
:10773000408151816281738122E081E59FE2AEDE6A
:107740008881998197FF05C0CE5ADF4F8881998142
:107750007FDDDF91CF91DDCECF93DF932091330397
:1077600020FF08C0EC0185E09FE2E9DDCE01DF915A
:10777000CF91D5CEDF91CF910895EEDF80913F0C70
:107780008F5F813041F080933F0C8091400C81509D
:107790008093400C089510923F0CF7CF8DEC9AE245
:1077A000CEDD86EC9AE2CBDD8091220D80FD18C003
:1077B00089EB9AE2C4DD8FEB9AE2C1DD8091220D64
:1077C00082FD11C089EB9AE2BADD82EB9AE2B7DD65
:1077D0008091220D84FD0AC089EB9AE2B0DD99CE3A
:1077E0008CEB9AE2E7CF8CEB9AE2EECF8CEB9AE24D
:1077F000F5CFCF93DF9380910301C4E081FDC0E01A
:10780000659BC1604B9BC061DFB7F8948091F0032A
:107810008C238093F0039091220D891759F0809367
:10782000220D9091EF03892B8093EF038091330316
:1078300086FDB4DFC093F003DFBFDF91CF910895E1
:107840001F920F920FB60F9211240BB60F924F9208
:107850005F926F927F928F929F92AF92BF92CF92E0
:10786000DF92EF92FF920F931F932F933F934F93CB
:107870005F936F937F938F939F93AF93BF93CF93B8
:10788000DF93EF93FF9380E07091CC03772381F433
:107890007091CB03772319F46091CA0391F0709330
:1078A0008900609388001092CA031092CB0308C02D
:1078B0006091CB03605870406093CB037093CC030E
:1078C00081E0811139C080916F008D7F80936F00BE
:1078D00088E49EEE90938900809388008091FD0C4F
:1078E000882309F40CC4C091FF03D09100042097B1
:1078F00009F04AC1E0914A0427E7E29FF001112410
:10790000EB57FB4FF0930004E093FF03818187FF67
:1079100036C0109200041092FF03E0EDCE2EE7E097
:10792000DE2EE12CF12CC701B6010E94FC258091CE
:107930006F00826080936F00FF91EF91DF91CF9194
:10794000BF91AF919F918F917F916F915F914F9177
:107950003F912F911F910F91FF90EF90DF90CF906B
:10796000BF90AF909F908F907F906F905F904F905F
:107970000F900BBE0F900FBE0F901F90189578942C
:107980008091330385FF2DC080914A048F3028F504
:107990008F5F80934A04109200041092FF03F894C2
:1079A0008091FD0C81508093FD0C8091FD0C811124
:1079B0000DC08091AA0C9091AB0C2091CC0C23FFB0
:1079C0000EC080619093AB0C8093AA0C88EEC82EF9
:1079D00083E0D82EE12CF12CA6CF80E0DACF8F7E89
:1079E000F1CFE091FF03F0910004818180FF31C06D
:1079F0008091FD0C9381981708F08BCFC580D680BD
:107A0000E780F08480914A048F30F8F48F5F809390
:107A10004A04109200041092FF03F8948091FD0C28
:107A200081508093FD0C8091FD0C81117CCF809161
:107A3000AA0C9091AB0C2091CC0C23FF08C0806164
:107A40009093AB0C8093AA0C6ECF80E0E0CF8F7E3A
:107A5000F7CF848184FD5F98E091FF03F0910004EB
:107A6000848185FD8A98E091FF03F0910004848170
:107A700086FF06C0809108018E7F80930801479899
:107A8000E091FF03F0910004848187FD1298E0915A
:107A9000FF03F09100048081866080837894C09118
:107AA000FF03D0910004EB8144E0E402F0011124D3
:107AB000EC0FFD1F81859285A385B4858093FB0320
:107AC0009093FC03A093FD03B093FE03888180FD97
:107AD00003C0CE010E94A122C159DF4F8881998144
:107AE0009093FA038093F9031092F5031092F60332
:107AF0001092F7031092F8031092F1031092F20320
:107B00001092F3031092F403F894E091FF03F091C4
:107B1000000484818171813151F5899AE091FF03DC
:107B2000F091000484818272823219F58F9AE0917B
:107B3000FF03F0910004848184748434E1F4809123
:107B40000B01826080930B01439AE091FF03F09157
:107B50000004848188788838A9F4169AC0901802A5
:107B6000D0901902E0901A02F0901B02DCCE8998A6
:107B7000D5CF8F98DCCF80910B018D7F80930B0147
:107B80004398E3CF1698EACF898184FF20C031DE85
:107B90009091220D9923D9F08C81282F21712031C9
:107BA00021F490FF02C08F7E8C838C81282F22725B
:107BB000203221F492FF02C08F7D8C838C81282F8C
:107BC0002474203421F494FF02C08F7B8C83F090C6
:107BD0001702E091FF03F0910004ED58FF4F808100
:107BE0009181A281B3814F2D0F2C000C550B660B98
:107BF000770B84179507A607B7070CF4F82E20E03B
:107C00002F150CF0E6C0E091FF03F091000485A170
:107C100096A1A7A1B0A5458956896789708D841B57
:107C2000950BA60BB70B85A396A3A7A3B0A7B7FF89
:107C300019C0149AE091FF03F091000485A196A168
:107C4000A7A1B0A54091FB035091FC036091FD03F7
:107C50007091FE03840F951FA61FB71F85A396A3DF
:107C6000A7A3B0A7E091FF03F0910004848184FFF3
:107C70002BC0818D928DA38DB48D418552856385F6
:107C80007485841B950BA60BB70B818F928FA38FE6
:107C9000B48FB7FF19C0889AE091FF03F0910004F8
:107CA000818D928DA38DB48D4091FB035091FC0387
:107CB0006091FD037091FE03840F951FA61FB71FEF
:107CC000818F928FA38FB48FE091FF03F091000416
:107CD000848185FF2BC0858D968DA78DB0A14585AC
:107CE000568567857089841B950BA60BB70B858F0E
:107CF000968FA78FB0A3B7FF19C08E9AE091FF03AC
:107D0000F0910004858D968DA78DB0A14091FB0365
:107D10005091FC036091FD037091FE03840F951F49
:107D2000A61FB71F858F968FA78FB0A3E091FF0383
:107D3000F0910004848186FF30C081A192A1A3A1AB
:107D4000B4A14189528963897489841B950BA60B60
:107D5000B70B81A392A3A3A3B4A3B7FF1EC08091C6
:107D60000B01886080930B01419AE091FF03F09131
:107D7000000481A192A1A3A1B4A14091FB03509161
:107D8000FC036091FD037091FE03840F951FA61FF5
:107D9000B71F81A392A3A3A3B4A31498E091FF03F8
:107DA000F0910004ED58FF4F80819181A281B38151
:107DB0000197A109B10980839183A283B383889835
:107DC0008E9880910B01877F80930B0141982F5FE4
:107DD00017CF7894C091FF03D09100048090F503F1
:107DE0009090F603A090F703B090F803FE01E35AD9
:107DF000FF4F80819181A281B3818E010D581F4F69
:107E000088159905AA05BB0508F4CBC04090F1037D
:107E10005090F2036090F3037090F4033C9620813D
:107E2000318142815381C301B2010E946E22FE0161
:107E3000E159FF4F20813181820F931F9093FA0304
:107E40008093F9033297208131812817390720F474
:107E50003093FA032093F9038091F9039091FA0388
:107E6000813E6EE2960708F498C0813C7DE5970755
:107E700008F48DC024E02093170296958795969577
:107E800087950E942B2660931802709319028093A5
:107E90001A0290931B02460E571E681E791E4092CE
:107EA000F1035092F2036092F3037092F4038F2D6A
:107EB000FF0C990BAA0BBB0B880D991DAA1DBB1DAE
:107EC0008093F5039093F603A093F703B093F80320
:107ED000C0901802D0901902E0901A02F0901B0294
:107EE000F80180819181A281B381181619061A06C2
:107EF0001B0624F48C81807F09F03EC080914A04E7
:107F00008F3008F0F8C08F5F80934A04109200040D
:107F10001092FF03F8948091FD0C81508093FD0C2A
:107F20008091FD0C81110DC08091AA0C9091AB0C39
:107F30002091CC0C23FFE1C080619093AB0C809327
:107F4000AA0C8091FD0C81110BC08091CC0C83FD9B
:107F500007C087E090E00E94983260E00E94A6C8C7
:107F6000F594E794D794C794C0921802D09219025E
:107F7000E0921A02F0921B0280914D0C90914E0CEF
:107F8000892B09F4D0CCF8940E945F24CCCC22E059
:107F9000209317029695879574CF21E020931702BE
:107FA00070CFF8014081518162817381FE01EF59E8
:107FB000FF4F80819181A281B38184179507A60725
:107FC000B7070CF468C0898182FD0BC01092F103E1
:107FD0001092F2031092F3031092F40389818460EB
:107FE0008983C090F103D090F203E090F303F09006
:107FF000F403FE01E759FF4F208131814281538113
:10800000C701B6010E946E222091F9033091FA0354
:10801000FE01EF58FF4F2817390740F58081918105
:10802000813E7EE2970798F1813CEDE59E0748F19D
:1080300024E02093170296958795969587950E9440
:108040002B26609318027093190280931A02909362
:108050001B02C60ED71EE81EF91EC092F103D09275
:10806000F203E092F303F092F40332CF40815181A6
:10807000B901681B790BCB016417750788F6CA0133
:10808000CFCF22E02093170296958795D8CF21E095
:1080900020931702D4CFFE01E359FF4F2081318195
:1080A000749780819181A281B381213EFEE23F07D6
:1080B000F0F0213C3D4598F024E02093170232E097
:1080C000880F991FAA1FBB1F3A95D1F780931802FA
:1080D00090931902A0931A02B0931B02F9CE22E0EA
:1080E00020931702880F991FAA1FBB1FEFCF21E013
:1080F00020931702EBCF80E007CF8F7E1ECF8091B9
:108100004D0C90914E0C892B59F00E945F24609188
:1081100018027091190280911A0290911B0205CCED
:1081200080914B0490914C04892B49F080914B0431
:1081300090914C04019790934C0480934B041092BF
:10814000CA031092CB031092CC031092CD038CED96
:108150009FEF9093890080938800E9CBCF92DF92C4
:10816000EF92FF92CF936A017B01C22FE8D84C2F88
:10817000C701B601F2D8CF91FF90EF90DF90CF907A
:10818000C8C92F923F924F925F926F927F928F92C7
:108190009F92AF92BF92CF92DF92EF92FF920F9396
:1081A0001F93CF93DF93CDB7DEB768970FB6F894E0
:1081B000DEBF0FBECDBF4090390250903A026090B2
:1081C0003B0270903C024D865E866F86788A809076
:1081D0001A0C90901B0CA0901C0CB0901D0C2091C0
:1081E000260C3091270C4091280C5091290CC50188
:1081F000B4010E9463EFA30192010E9420EE0E944D
:1082000094F069837A838B839C83609328047093B2
:10821000290480932A0490932B0440903D025090AF
:108220003E0260903F0270904002498A5A8A6B8AEF
:108230007C8AC090160CD090170CE090180CF0902F
:10824000190C2091220C3091230C4091240C509158
:10825000250CC701B6010E9463EFA30192010E94A1
:1082600020EE0E9494F06D837E838F8398876093C5
:10827000300470933104809332049093330440901F
:1082800041025090420260904302709044024D8A35
:108290005E8A6F8A788E4090120C5090130C60901A
:1082A000140C7090150C20911E0C30911F0C4091F5
:1082B000200C5091210CC301B2010E9463EF2D8963
:1082C0003E894F89588D0E9420EE0E9494F0698764
:1082D0007A878B879C8760931C0470931D0480931E
:1082E0001E0490931F04A50194016D857E858F85E2
:1082F00098890E9420EE0E9494F04B015C018092CC
:108300002C0490922D04A0922E04B0922F04A70169
:10831000960169897A898B899C890E9420EE0E9446
:1083200094F06B017C01C0923404D0923504E09249
:108330003604F0923704A30192016D897E898F89FA
:10834000988D0E9420EE0E9494F060932004709318
:10835000210480932204909323042091B802309149
:10836000B9024091BA025091BB022D8B3E8B4F8BCC
:10837000588F09811A812B813C814D885E886F88D6
:10838000788C041915092609370949805A806B80B1
:108390007C80041515052605370514F49301820128
:1083A00000934604109347042093480430934904F3
:1083B000950184014D885E886F88788C04191509B1
:1083C0002609370980169106A206B30614F4950112
:1083D000840100931604109317042093180430931B
:1083E00019048090BC029090BD02A090BE02B09093
:1083F000BF020D811E812F813885081919092A09AC
:108400003B094D805E806F80788404151505260534
:10841000370514F49301820100934204109343043E
:1084200020934404309345049701860108191909E3
:108430002A093B09C016D106E206F30614F4970197
:1084400086010093120410931304209314043093B4
:108450001504C090C002D090C102E090C202F0901A
:10846000C30209851A852B853C850C191D092E0927
:108470003F0969847A848B849C8406151705280536
:10848000390514F49401830100933E0410933F04D2
:1084900020934004309341048B019C010C191D0969
:1084A0002E093F09601771078207930714F48B01A7
:1084B0009C0100930E0410930F042093100430933A
:1084C000110429E332E03A83298387EEA82E8CE059
:1084D000B82E94E4C92E93E0D92E2DE5E22E24E0A7
:1084E000F22E04E313E03DE4832E34E0932E49E4BE
:1084F000242E42E0342EA981BA814D905D906D907A
:108500007D90BA83A983A301920160E070E080E8C6
:108510009FE30E942CF0F5016193719381939193F5
:108520005F01D6012D913D914D915D916D01C3018A
:10853000B2010E9420EE0E9499F0F70161937193BD
:10854000819391937F01D8012D913D914D915D9142
:108550008D01C301B2010E9420EE0E9499F0F40146
:1085600061937193819391934F0149805A802414B0
:10857000350409F600913403109135035090360309
:108580005D82609037036982C0904403D0904503B8
:10859000E0904603F09047039601A701B801852DAE
:1085A000962D0E9476F118161CF08601ED82F98254
:1085B00098014D8159816D857E858F8598890E94AE
:1085C00020EE9B01AC0160E070E080E090E40E944E
:1085D0002CF00E9422F26B017C0121EE3AE744EB81
:1085E0005FE3B8018D8199810E9420EEA701960179
:1085F0000E9420EE8B018D839983C0903803D09028
:108600003903E0903A03F0903B0380904803909048
:108610004903A0904A03B0904B039401A501B60111
:10862000C7010E9476F1181614F0640175019601D5
:10863000A70169897A898B899C890E9420EE9B0118
:10864000AC0160E070E080E090E40E942CF00E94B9
:1086500022F24B015C0121EE3AE744EB5FE3B60105
:10866000C7010E9420EEA50194010E9420EE6B013B
:108670007C019B01AC01B8018D8199810E94BBED09
:1086800087FF03C08601ED82F98298014D815981EF
:10869000B8018D8199810E9463EF6B017C0120916B
:1086A000270D3091280D4091290D50912A0D0E94DF
:1086B00076F1181674F4C092270DD092280DE0922E
:1086C000290DF0922A0D22E0B701A60188E49EE26E
:1086D00045DD00913C0310913D0370903E037D8287
:1086E00080903F038982C0904C03D0904D03E0906E
:1086F0004E03F0904F039601A701B801872D982DE6
:108700000E9476F118161CF08601ED82F982209104
:108710004102309142024091430250914402B8011B
:108720008D8199810E9420EE9B01AC0160E070E098
:1087300080E090E40E942CF00E9422F26B017C0108
:1087400020E030E040E05FE3B8018D8199810E9434
:1087500020EEA70196010E9420EE9B01AC010E9431
:1087600063EF6B017C012091230D3091240D40912A
:10877000250D5091260D0E9476F1181674F4C092C2
:10878000230DD092240DE092250DF092260D22E0CB
:10879000B701A60188E29EE2E1DC80911D0D8D7F8C
:1087A00080931D0D68960FB6F894DEBF0FBECDBF47
:1087B000DF91CF911F910F91FF90EF90DF90CF90BD
:1087C000BF90AF909F908F907F906F905F904F90F1
:1087D0003F902F900895CF92DF92EF92FF92CF9328
:1087E000DF936B017C01D42F20E030E040EF52E4B6
:1087F0000E9476F118160CF443C020E030E0A90185
:10880000C701B6010E94BBED87FF03C0C12CD12C6C
:108810007601A70196016091790270917A028091A8
:108820007B0290917C020E94BBED882311F1C092E3
:108830007902D0927A02E0927B02F0927C02C0919F
:10884000A402C97FD11123C0C093A40220E0B701C4
:10885000A60189EF9AE282DC20E030E040E751E4B3
:10886000C701B6010E9476F11816ECF48FEF8093E1
:10887000E30CDF91CF91FF90EF90DF90CF900895C0
:10888000C12CD12C80EFE82E82E4F82EC2CF20E05C
:1088900030E040EF51E4C701B6010E9476F11816AE
:1088A0009CF6C160D1CF80911D0D80FFE2CF109268
:1088B000E30CDFCFCF92DF92EF92FF921F93CF9323
:1088C000DF93EC016A017B01122F85E19AE20E949D
:1088D0009F39212FB701A601CE01DF91CF911F91C2
:1088E000FF90EF90DF90CF9039CC4F925F926F92D4
:1088F0007F928F929F92AF92BF92CF92DF92EF9230
:10890000FF922091C00C3091C10C4091C20C50914B
:10891000C30C6091D50C7091D60C8091D70C9091BE
:10892000D80C0E9463EF2B013C012091C40C3091C4
:10893000C50C4091C60C5091C70C6091D90C709138
:10894000DA0C8091DB0C9091DC0C0E9463EF4B0100
:108950005C012091C80C3091C90C4091CA0C509117
:10896000CB0C6091DD0C7091DE0C8091DF0C90914E
:10897000E00C0E9463EF6B017C0180911A0420E0FF
:1089800030E040E85FE3882321F020E732E441E271
:108990005DE3C301B2010E9420EEAB01BC0122E005
:1089A00088EF9BE10E944E3A80911A0420E030E06B
:1089B00040E85FE3882321F020E732E441E25DE311
:1089C000C501B4010E9420EEAB01BC0122E084EF9E
:1089D0009BE10E944E3A80911A0420E030E040E88A
:1089E0005FE3882321F020E732E441E25DE3C70141
:1089F000B6010E9420EEAB01BC0123E080EF9BE1B9
:108A00000E944E3A6091BC0C7091BD0C8091BE0CDE
:108A10009091BF0C0E94C1ED2091F30C3091F40CA9
:108A20004091F50C5091F60C0E9420EE20911A0412
:108A3000211118C020E030E040E85FE30E9420EE02
:108A4000AB01BC0124E08CEE9BE1FF90EF90DF9046
:108A5000CF90BF90AF909F908F907F906F905F90DE
:108A60004F907CCB20E732E441E25DE3E7CF4F92C9
:108A70005F926F927F928F929F92AF92BF92CF92AE
:108A8000DF92EF92FF920F931F93CF93DF9300D06B
:108A90001F92CDB7DEB72B013C0149015A01E98293
:108AA000FA820B831C83C0901A0CD0901B0CE090B0
:108AB0001C0CF0901D0C2AE037ED43E25CE3C7018B
:108AC000B6010E9462EFA30192010E94BBED18164D
:108AD0000CF485C02091260C3091270C4091280C75
:108AE0005091290CC701B6010E9463EF2AE037EDCF
:108AF00043E25CE30E9463EF9B01AC01C301B2015E
:108B00000E94BBED18160CF46AC0C090160CD090F1
:108B1000170CE090180CF090190C2AE037ED43E2A6
:108B20005CE3C701B6010E9462EFA50194010E94B7
:108B3000BBED18160CF453C02091220C3091230C7D
:108B40004091240C5091250CC701B6010E9463EF9F
:108B50002AE037ED43E25CE30E9463EF9B01AC0146
:108B6000C501B4010E94BBED1816CCF1C090120CE7
:108B7000D090130CE090140CF090150C2AE037ED17
:108B800043E25CE3C701B6010E9462EF29813A81AA
:108B90004B815C810E94BBED18160CF120911E0CDC
:108BA00030911F0C4091200C5091210CC701B6014F
:108BB0000E9463EF20E030E0A9010E9463EF2AE009
:108BC00037ED43E25CE30E9463EF9B01AC016981F6
:108BD0007A818B819C810E94BBED1816D4F481E0D0
:108BE0000E94B62482DE80E00F900F900F900F90CD
:108BF000DF91CF911F910F91FF90EF90DF90CF9079
:108C0000BF90AF909F908F907F906F905F904F90AC
:108C1000089581E0E9CF3F924F925F926F927F92E9
:108C20008F929F92AF92BF92CF92DF92EF92FF927C
:108C30000F931F93CF93DF9300D000D000D01F92EB
:108C4000CDB7DEB79A878987FC01808191819C012D
:108C500028733327232B21F586FF22C02091200D76
:108C600021FF1EC066897789808D918D20911B041C
:108C700040911E0D50911F0D5A834983222309F400
:108C800088C020E030E0A9010E94BBED682F661F7C
:108C90006627661F89819A810E94E2CF312CA7C086
:108CA00020911B0E25FFBCC0E985FA85008111814A
:108CB000980128733327232B09F0CEC03324339433
:108CC000E985FA85008111819801207433273E835C
:108CD0002D8306FF04C08091330383FF8FC28091F0
:108CE000BC0C9091BD0CA091BE0CB091BF0C8093B8
:108CF0007D0490937E04A0937F04B093800410FFC2
:108D000035C0E985FA85C28CD38CE48CF58C2DECCA
:108D10003CEC4CEC5DE3C701B6010E9476F11816FD
:108D20002CF56091F90C7091FA0C072E000C880B51
:108D3000990B0E94C1ED4B015C0180911A048823BC
:108D400009F418C32FE737EB4AE85BE3C701B60124
:108D50000E9420EEA50194010E9420EE6093530C26
:108D60007093540C8093550C9093560C31100DC396
:108D700080917D0490917E04A0917F04B091800445
:108D80008093BC0C9093BD0CA093BE0CB093BF0C11
:108D90002EC03090210D311074CF209145023091BA
:108DA000460240914702509148020E9420EE2091D5
:108DB0001A04222331F023E333E34BEC51E40E9405
:108DC00020EE0E9494F041E00091BC0C1091BD0C8B
:108DD0002091BE0C3091BF0C60177107820793077A
:108DE0000CF040E0642F89819A810E94E2CF832DAC
:108DF0002A960FB6F894DEBF0FBECDBFDF91CF919C
:108E00001F910F91FF90EF90DF90CF90BF90AF90A8
:108E10009F908F907F906F905F904F903F900895BC
:108E20002091CC0C20FD05C0877FE985FA859183D0
:108E3000808321FD07C0E985FA85808191818F7E3D
:108E40009183808322FD30CFE985FA8580819181ED
:108E50008F7D9183808328CF98012870332740919C
:108E60001B047801F0E1EF22FF2400721127411169
:108E70003FC1232B51F1E985FA856285738584858D
:108E8000958520911A04222331F023E333E34BEC40
:108E900051E40E9420EE2091D50C3091D60C4091E7
:108EA000D70C5091D80C0E9462EF6093C00C709365
:108EB000C10C8093C20C9093C30C6093410C7093CF
:108EC000420C8093430C9093440CEF2851F1E985B8
:108ED000FA85668577858089918920911A042223F5
:108EE00031F023E333E34BEC51E40E9420EE209178
:108EF000D90C3091DA0C4091DB0C5091DC0C0E94C3
:108F000062EF6093C40C7093C50C8093C60C909371
:108F1000C70C6093450C7093460C8093470C90935C
:108F2000480C012B51F1E985FA856289738984899E
:108F3000958920911A04222331F023E333E34BEC8B
:108F400051E40E9420EE2091DD0C3091DE0C409126
:108F5000DF0C5091E00C0E9462EF6093C80C70939C
:108F6000C90C8093CA0C9093CB0C6093490C7093FE
:108F70004A0C80934B0C90934C0CC090490CD090B1
:108F80004A0CE0904B0CF0904C0C4090450C5090EB
:108F9000460C6090470C7090480C20912E0C30913C
:108FA0002F0C4091300C5091310CC301B2010E9442
:108FB00063EF69837A838B839C838090410C9090CC
:108FC000420CA090430CB090440C2091320C309194
:108FD000330C4091340C5091350CC701B6010E94FE
:108FE00063EF209124043091250440912604509190
:108FF00027040E9463EF6D837E838F83988720917F
:109000002A0C30912B0C40912C0C50912D0CC50149
:10901000B4010E9463EF2091390230913A024091ED
:109020003B0250913C020E9420EE20E030E040E004
:109030005FE30E9463EF0E94C5F00E9494F060938A
:10904000710470937204809373049093740420915C
:109050003D0230913E0240913F02509140026981B1
:109060007A818B819C810E9420EE20E030E040E0FC
:109070005FE30E9463EF0E94C5F00E9494F060934A
:10908000750470937604809377049093780420910C
:1090900041023091420240914302509144026D815D
:1090A0007E818F8198850E9420EE20E030E040E0B4
:1090B0005FE30E9463EF0E94C5F00E9494F060930A
:1090C000790470937A0480937B0490937C0480915C
:1090D0001B0E85FDF3CD8091200D86FDEFCD870120
:1090E0007601A3019201C501B401C1DC382EE8CD9F
:1090F000232B51F1E985FA856285738584859585F1
:1091000020911A04222331F023E333E34BEC51E4A2
:109110000E9420EE2091410C3091420C4091430C72
:109120005091440C0E9463EF6093410C7093420C89
:109130008093430C9093440C6093C00C7093C10CCB
:109140008093C20C9093C30CEF2851F1E985FA8506
:10915000668577858089918920911A04222331F0D0
:1091600023E333E34BEC51E40E9420EE2091450CC5
:109170003091460C4091470C5091480C0E9463EF8F
:109180006093450C7093460C8093470C9093480C69
:109190006093C40C7093C50C8093C60C9093C70C5D
:1091A000012B09F4EACEE985FA85628973898489FD
:1091B000958920911A04222331F023E333E34BEC09
:1091C00051E40E9420EE2091490C30914A0C4091CC
:1091D0004B0C50914C0C0E9463EF6093490C7093C0
:1091E0004A0C80934B0C90934C0C6093C80C70937A
:1091F000C90C8093CA0C9093CB0CBFCEE985FA853D
:1092000086889788A08CB18C409045025090460289
:109210006090470270904802A3019201C501B40119
:109220000E9420EE20911A04222331F023E333E33D
:109230004BEC51E40E9420EE0E9494F06B017C0103
:1092400020911E0D30911F0D3A832983F90167A5E6
:1092500070A981A992A920911B04211104C0209119
:10926000210D2223B1F120E030E046E153E40E94D9
:10927000BBED87FF09C080911B0E87FD05C0E9810A
:10928000FA8182A5811115C0C501B4019F77209193
:1092900023023091240240912502509126020E941F
:1092A00020EE20E030E040E253E40E9476F1181610
:1092B0001CF4C12CD12C76018091BC0C9091BD0C7A
:1092C000A091BE0CB091BF0C8C0D9D1DAE1DBF1D9D
:1092D0000ECD20E030E046E153E40E94BBED87FF75
:1092E00009C080911B0E87FD05C0E981FA8182A526
:1092F00081112FC08091BC0C9091BD0CA091BE0C2F
:10930000B091BF0CA7019601281B390B4A0B5B0BD0
:10931000CA01B9010E94C1ED9F77209123023091CB
:10932000240240912502509126020E9420EE4B011A
:109330005C0120E030E040E253E4C301B2010E944E
:1093400020EE9B01AC01C501B4010E9476F1181614
:1093500044F4C092BC0CD092BD0CE092BE0CF092D2
:10936000BF0CC0927D04D0927E04E0927F04F09204
:109370008004C5CCA5019401C701B6010E9420EE6E
:109380002EE333EC4EE259E3E7CC08731127012BAF
:1093900009F02DCD2D813E81232B09F47FCC332480
:1093A000339440917D0450917E0460917F047091CC
:1093B00080048091BC0C9091BD0CA091BE0CB0912A
:1093C000BF0C481759076A077B0709F010CD66CC18
:1093D000CF92DF92EF92FF926A017B010E949F3948
:1093E000C701B6010E943439FF90EF90DF90CF9013
:1093F0000C94893ACF93DF93EB010E949F39CE0101
:109400000E949A39DF91CF910C94893A909133035D
:10941000981719F18093330383FF1FC01092EA025B
:109420001092EB021092EC021092ED02E091E00239
:10943000F0E0EF51F34F10821092790210927A020D
:1094400010927B0210927C02E0916F02F0E0EF51EB
:10945000F34F10829FEF90930102682F70E08AEE25
:109460009DE2C8CF0F931F93CF93DF93EC018B0145
:1094700085E19AE20E949F39B801CE01DF91CF9138
:109480001F910F91B7CF8F929F92AF92BF92CF92C1
:10949000DF92EF92FF92CF93DF93893C910514F016
:1094A00088EC90E0EC01499714F4C9E1D0E0D09346
:1094B000FC0CC093FB0CE0911E0DF0911F0DE958C0
:1094C000FF4FC080D180E280F380BE010D2E000CE2
:1094D000880B990B0E94C1ED2AE037ED43E25CE373
:1094E0000E9420EE4B015C0120E030E0A901C701A1
:1094F000B6010E94BBED1816B4F080922302909240
:109500002402A0922502B0922602BE018CE29CE1C8
:10951000DF91CF91FF90EF90DF90CF90BF90AF9011
:109520009F908F9067CF20E030E040E850E4C50185
:10953000B4010E9420EE4B015C01A7019601C70116
:10954000B6010E9420EE2BED3FE049E450E40E947A
:1095500020EE9B01AC01C501B4010E942CF0609388
:109560002302709324028093250290932602CDCF8C
:10957000CF92DF92EF92FF92CF93DF93853F21E06E
:10958000920714F084EF91E0EC01499714F4C9E1DB
:10959000D0E0BE010D2E000C880B990B0E94C1ED8E
:1095A0006B017C016091F90C7091FA0C072E000C94
:1095B000880B990B0E94C1ED9B01AC01C701B6015C
:1095C0000E942CF09B01AC016091530C7091540CE3
:1095D0008091550C9091560C0E9420EE6093530C94
:1095E0007093540C8093550C9093560CD093FA0CB6
:1095F000C093F90CBE018DE19CE1DF91CF91FF900A
:10960000EF90DF90CF90F6CE0E949F390C94893A6C
:1096100010929C100E948B368091CC0C877F809397
:10962000CC0C8091AA0C9091AB0C897E9093AB0CE2
:109630008093AA0C8FE290E3E7CFCF93C0912202F0
:1096400021E020932202E0DFC0932202CF9108950F
:10965000CF92DF92EF92FF92CF93DF93EC010E94C3
:109660003E296B017C01209709F18091380490918B
:109670003904A0913A04B0913B04A7019601281B3C
:10968000390B4A0B5B0BDA01C901803D9740A105FC
:10969000B105A0F084EB9EE2C230D10531F087EA3B
:1096A0009EE2239711F087E99EE2C7DFC09238045B
:1096B000D0923904E0923A04F0923B04DF91CF91CA
:1096C000FF90EF90DF90CF9008958AE09EE00E9497
:1096D000D6368091AA0C81FF0DC080919D1081111A
:1096E0000E94E0D180911B0E84FD08C010922D0DC8
:1096F0000C9444CA8AE89EE2A0DFF4CF089581E08A
:109700008093220283EE9FE20E949F3980913C0465
:1097100090913D040E949F3987E89FE275DF61E0E8
:1097200080913C0490913D040C94A6C887E891E197
:109730000E94AC2510923D0C80913C0CE0911C02E3
:10974000F0911D028823B1F08EE183870E94893A4F
:10975000E0911C02F0911D02428153816481758168
:109760004F5F5F4F6F4F7F4F85ED9EE231DE82E0AE
:109770009FE24ACF8EE0E9CFBF92CF92DF92EF9285
:10978000FF920F931F93CF93DF93EC01888181FFAA
:109790002DC08E819F818E36910519F5E0911C02B6
:1097A000F0911D028091370C9091380CA091390CEA
:1097B000B0913A0C82839383A483B58382E09FE2C5
:1097C00023DFE0911C02F0911D028FEF8387DF9170
:1097D000CF911F910F91FF90EF90DF90CF90BF90AE
:1097E00008958037910511F40E94A838B880B0FE22
:1097F00064C0E0911C02F0911D0282819381A481DA
:10980000B5816C017D012FEFC21AD20AE20AF20A79
:109810004091370C5091380C6091390C70913A0C92
:109820009701860104271527262737272227332764
:10983000012B022B032B09F43CC0841B950B88974A
:1098400088F410923D0C8CEF9EE2C2DD82E09FE234
:10985000DF91CF911F910F91FF90EF90DF90CF900C
:10986000BF90D2CE838587FF21C08091330382FFD2
:1098700013C087EE9EE20E949F39C701B6010E9485
:1098800034394091370C5091380C6091390C7091FB
:109890003A0C81EE9EE29CDDDF91CF911F910F91FA
:1098A000FF90EF90DF90CF90BF9040CF81508387A3
:1098B000C8CF428353836483758380913C04909125
:1098C0003D04892B39F0B1FE22C08E819F81873EF5
:1098D0009340E9F410923B0C8091400C8F5F809391
:1098E000400C4091370C5091380C6091390C7091BC
:1098F0003A0C8DED9EE26CDDE0911C02F0911D02B0
:1099000080913C0C868390E080E0A2DE5ACFF7DEA7
:10991000E8CF8091AA0C9091AB0C8F779C7F9093AD
:10992000AB0C8093AA0C2091AF0C213061F018F0A1
:10993000223089F0089580689093AB0C8093AA0C34
:1099400088E19EE261CE91609093AB0C8093AA0C6B
:1099500086E09EE2F7CF92609093AB0C8093AA0CC6
:1099600086EF9DE2EFCFCF93DF93EC0183E29AE2A3
:109970000E949F39CE01DF91CF9146CE0F931F9366
:10998000CF93DF931F92CDB7DEB78C01BE016F5F1F
:109990007F4F80E790E10E941FC9019789F181E222
:1099A00090E332DE61E083E190E30E94A6C840913B
:1099B000941050919510609196107091971080E7D7
:1099C00090E10E949A2DBE016F5F7F4F80E790E18A
:1099D0000E941FC9019751F18AEE9FE2C4DFD801AE
:1099E000ED91FC910684F785E02DC801199510E0F2
:1099F00000E0C8010F90DF91CF911F910F91089562
:109A0000098110E08091941090919510A09196108A
:109A1000B09197100196A11DB11D80939410909361
:109A20009510A0939610B0939710E3CF098110E0A2
:109A300061E084E090E30E94A6C8E4CF2F923F92B9
:109A40005F926F927F928F929F92AF92BF92CF92CE
:109A5000DF92EF92FF920F931F93CF93DF93CDB7D7
:109A6000DEB72C970FB6F894DEBF0FBECDBF9C8734
:109A70008B877B01B42EDC0111961C921E921396EB
:109A80001C921E921297FC01EB5AFF4F81E0842733
:109A900080834B01A12C552453943D01BEE46B0EF1
:109AA000711CEB85FC85E65BFF4FFA83E9838B85B0
:109AB0009C858A5B9F4F9C838B83AB85BC85AE5B0B
:109AC000BF4FBE83AD83EB85FC85FE96F887EF83A1
:109AD0008B859C858C5A9F4F9A878987CB84DC84A1
:109AE00092E5C90ED11C87010F5F1F4FD701EC9182
:109AF000EE2309F444C2E83209F441C2E53209F424
:109B00003EC2EA52E13508F05DC00E2E000CFF0B9C
:109B10008827E257F24B8F4F0C94C2F2A84FE24DC8
:109B2000E24DE24DE24DE24DE24DE24DE24DE24DBD
:109B3000E24DE24DE24DE24DE24DE24DE24DE24DAD
:109B4000E24DE24DE24DE24DE24D544F654F364F4E
:109B5000254FA64EB34EF94D434FED4EFF4E764F77
:109B6000874F154EE44D984FDD4EE24D184FD04EC5
:109B7000C34EE24DE24DE24D794E894E964EE24D96
:109B8000E24DE24DE24DE24DE24D544F654F364F0E
:109B9000254FA64EB34EF94D434FED4EFF4E764F37
:109BA000874F154EE44D984FDD4EE24D184FD04E85
:109BB000C34EE24DE24DE24D794E894E964E47013D
:109BC000AA24A39478018FCFC8010E94F028609343
:109BD000370C7093380C8093390C90933A0CEB85CA
:109BE000FC852081318121603183208375836483EA
:109BF000E9CFC8010E94F028AB85BC8519967C93FB
:109C00006E9318972D913C911197C9016F3F710583
:109C100009F020F484608D939C93D4CF846090618C
:109C2000EB85FC8591838083CDCFC8010E94F0280D
:109C3000DB01EB85FC857783668320813181A90177
:109C40004260518340836F3F7105D9F0D0F02260AC
:109C50003061318320839B012C5131092330310540
:109C6000B0F01B01E89422F8F0E22F16310479F0ED
:109C7000A537B10561F0A33182E0B80709F0A2CFA2
:109C800006C06431710519F06731710521F7F801DB
:109C90002191222351F020532A3038F198012F5F6F
:109CA0003F4FF8014081403211F1F60111830083EA
:109CB000F8018F012191222371F0A537B10549F0F8
:109CC000A431B10531F0A33182E0B80711F02032A0
:109CD00011F02A3271F7D8011C9250923E0CEB859C
:109CE000FC858081918190689DCF8F01D0CF8901C3
:109CF000D5CFC8010E941529AB85BC851A966D93F6
:109D00007D938D939C931D978D919C911197886065
:109D100082CFC8010E941529EB85FC85668777876D
:109D2000808B918B8081918180617CCFC8010E9462
:109D30001529AB85BC8552966D937D938D939C932D
:109D400055978D919C911197806265CFC8010E94B3
:109D50001529EB85FC85668B778B808F918F8081B1
:109D6000918180645FCFC8010E941529AB85BC85B5
:109D70005A966D937D938D939C935D978D919C9155
:109D80001197916048CFC8010E94F028E985FA85B3
:109D90006083AB85BC858D919C91119792603BCF80
:109DA000C8010E94F028EB85FC85668F778F80A321
:109DB00091A380819181946035CFC8010E94F028E1
:109DC000AB85BC8592966D937D938D939C9395976F
:109DD0008D919C91119798601ECFC8010E94152902
:109DE000EB85FC8566A377A380A791A782819381E9
:109DF00081609383828380819181906113CFC801B8
:109E00000E941529AB85BC859A966D937D938D93A1
:109E10009C939D9712968D919C91139782601396B7
:109E20009C938E9312978D919C9111979061F3CE94
:109E3000C8010E941529EB85FC8566A777A780AB32
:109E400091AB828193818460D4CFC8010E9415298F
:109E5000AB85BC85D2966D937D938D939C93D5975E
:109E600012968D919C9113978860D9CFC8010E945A
:109E70001529EB85FC8566AB77AB80AF91AF82810E
:109E800093818061B6CFC8010E941529AB85BC853E
:109E9000DA966D937D938D939C93DD9712968D91B9
:109EA0009C9113978062BBCFC8010E941529EF8156
:109EB000F8856083718382839383AB85BC8512961A
:109EC0008D919C9113978064AACFC8010E94152997
:109ED000ED81FE816083718382839383AB85BC8532
:109EE00012968D919C911397806899CFC8010E941A
:109EF0001529EB81FC816083718382839383AB8519
:109F0000BC8512968D919C911397916088CFC80162
:109F10000E941529E981FA8160837183828393838A
:109F2000AB85BC8512968D919C911397926077CFEB
:109F3000C8010E941529F301608371838283938392
:109F4000AB85BC8512968D919C911397946067CFD9
:109F5000C8010E94F028F40180E0EE16FF0619F017
:109F600091918927FACF861709F429CE809133037E
:109F700082FF03C08EE19DE3F6DC10E012C0E091A9
:109F80001C02F0911D028681882321F1A11022C0BC
:109F9000BB2001F110913E0C11111CC088E19FE221
:109FA000E2DC812F2C960FB6F894DEBF0FBECDBF3A
:109FB000DF91CF911F910F91FF90EF90DF90CF90A5
:109FC000BF90AF909F908F907F906F905F903F90E9
:109FD0002F900895EB85FC858281938197FF12C0B5
:109FE0008091360C8F5F8093360C8091330382FF13
:109FF00003C08BE09FE2B7DC11E08091360C833028
:10A0000080F6BBCF1092360C11E0CBCFFF920F93AE
:10A010001F93CF93DF9380911D0D82FF42C00AE50D
:10A0200013E0F12C70E060E081EA9BE20E946E3A5E
:10A03000F801C191D1918F016E817F8188859985C9
:10A040000E9494F0665F7F4F8CE89BE26D32714016
:10A0500010F482E89BE20E949F398DA983FF04C01F
:10A0600083E79BE20E949F398DA984FF04C081E6AB
:10A070009BE20E949F390E94893A81E0F8120AC04F
:10A0800084E39BE270DC81E0DF91CF911F910F911F
:10A09000FF900895FF24F3948BEA9BE20E949F397E
:10A0A000C7CF80E0F1CFCF93DF93EC018DE19AE24F
:10A0B0000E949F39CE01DF91CF91A6CACF93DF9343
:10A0C000EC0180E19AE20E949F39CE01DF91CF91AD
:10A0D0009BCACF93C82FE0911E0DF0911F0D47A58D
:10A0E00050A961A972A922E08AE19CE10E944E3A3E
:10A0F000E0911E0DF0911F0D43A954A965A976A901
:10A1000020E087E19CE10E944E3A40917502509117
:10A110007602609177027091780222E083E19CE1FF
:10A120000E944E3A4091790250917A0260917B02EE
:10A1300070917C0220E087E19CE10E944E3A809180
:10A14000A40283FD66C084FD66C080E0682F082EEF
:10A15000000C770B882321F08EE09CE10E946E3A80
:10A16000CC2391F061E070E089E09CE10E946E3ABE
:10A1700080917302909174026CEF7FE0681B790B01
:10A180008CEE9AE20E946E3AE0916F02F0E0EF519D
:10A19000F34F608170E084E09CE10E946E3AE091B0
:10A1A0000102EF3F29F4E0911E0DF0911F0DE081B7
:10A1B000F0E0EF51F34F608170E080E09CE10E949D
:10A1C0006E3A8091150383FD28C084FD28C080E08D
:10A1D000682F082E000C770B882321F08BEF9BE172
:10A1E0000E946E3ACC2391F070E060E089E09CE13F
:10A1F0000E946E3A8091E4029091E5026CEF7FE05C
:10A20000681B790B8CEE9AE20E946E3ACF910C9407
:10A21000893A81E09BCF82E099CF81E0D9CF82E07B
:10A22000D7CF0FB6F894A89580916000886180938D
:10A230006000109260000FBE0895CF93DF9300D0AE
:10A240001F92CDB7DEB744E050E0BC01CE010196CD
:10A250000E94D7EE69817A818B819C810F900F904B
:10A260000F900F90DF91CF9108954F925F926F9270
:10A270007F928F929F92AF92BF92CF92DF92EF9296
:10A28000FF92CF93DF93CDB7DEB7C458D1090FB695
:10A29000F894DEBF0FBECDBF412C512C80E2682E5A
:10A2A00082E4782E49825A826B827C8244E050E0BC
:10A2B00068E273E0CE0101960E94F9EE80E090E042
:10A2C000A0E0B0E48D839E83AF83B88744E050E084
:10A2D0006CE273E0CE0105960E94F9EE80E090E01A
:10A2E000A6E1B3E489879A87AB87BC8744E050E056
:10A2F00068E473E0CE0109960E94F9EE1D861E8681
:10A300001F86188A44E050E060E273E0CE010D96AB
:10A310000E94F9EE198A1A8A1B8A1C8A44E050E0CE
:10A3200064E273E0CE0141960E94F9EE1D8A1E8A16
:10A330001F8A188E44E050E060E074E0CE0145963C
:10A340000E94F9EEC12CD12C90EAE92E91E4F92E6D
:10A35000C98EDA8EEB8EFC8E44E050E060E373E051
:10A36000CE0149960E94F9EECD8EDE8EEF8EF8A2D8
:10A3700044E050E064E373E0CE014D960E94F9EEB4
:10A38000812C912C20E2A22E23E4B22E89A29AA243
:10A39000ABA2BCA244E050E068E373E0CE0181963A
:10A3A0000E94F9EECDA2DEA2EFA2F8A644E050E0B2
:10A3B0006CE373E0CE0185960E94F9EEC9A6DAA699
:10A3C000EBA6FCA644E050E060E473E0CE01899681
:10A3D0000E94F9EE8DA69EA6AFA6B8AA44E050E072
:10A3E00064E473E0CE018D960E94F9EE19AA1AAAD0
:10A3F0001BAA1CAA44E050E060ED73E0CE01C196B8
:10A400000E94F9EE1DAA1EAA1FAA18AE44E050E051
:10A4100064ED73E0CE01C5960E94F9EE19AE1AAE56
:10A420001BAE1CAE44E050E068ED73E0CE01C9966F
:10A430000E94F9EE812C912C30E2A32E31E4B32E50
:10A4400021968CAE9DAEAEAEBFAE219744E050E0FB
:10A4500061EA73E0CE01CD960E94F9EE80E094E0CF
:10A46000ECDE6093BF107093C0108093C110909386
:10A47000C21025961CAE1DAE1EAE1FAE259744E041
:10A4800050E060ED73E0CE018F5B9F4F0E94F9EECC
:10A4900029961CAE1DAE1EAE1FAE299744E050E0BB
:10A4A00064ED73E0CE018B5B9F4F0E94F9EE2D9619
:10A4B0001CAE1DAE1EAE1FAE2D9744E050E068ED01
:10A4C00073E0CE01875B9F4F0E94F9EE60E08CED58
:10A4D00093E00E9402EF80E090E0A0E4B0E4619697
:10A4E0008CAF9DAFAEAFBFAF619744E050E060EE80
:10A4F00073E0CE01835B9F4F0E94F9EE80E090E015
:10A50000A0E5B1E465968CAF9DAFAEAFBFAF6597E8
:10A5100044E050E064EE73E0CE018F5A9F4F0E94FA
:10A52000F9EE69964CAE5DAE6EAE7FAE699744E0D3
:10A5300050E068EE73E0CE018B5A9F4F0E94F9EE17
:10A540006D961CAE1DAE1EAE1FAE6D9744E050E082
:10A550006CEE73E0CE01875A9F4F0E94F9EEA196F0
:10A560001CAE1DAE1EAE1FAEA19744E050E060EFE2
:10A5700073E0CE01835A9F4F0E94F9EEA5961CAE60
:10A580001DAE1EAE1FAEA59744E050E064EF73E031
:10A59000CE018F599F4F0E94F9EEA996CCAEDDAE49
:10A5A000EEAEFFAEA99744E050E068EF73E0CE0155
:10A5B0008B599F4F0E94F9EE60E08CEF93E00E9470
:10A5C00002EFAD961CAE1DAE1EAE1FAEAD9744E0C1
:10A5D00050E06CE074E0CE0187599F4F0E94F9EE85
:10A5E000E1961CAE1DAE1EAE1FAEE19744E050E0FA
:10A5F00060E174E0CE0183599F4F0E94F9EEE59629
:10A600001CAE1DAE1EAE1FAEE59744E050E064E107
:10A6100074E0CE018F589F4F0E94F9EE80E090E0E9
:10A62000A8ECB2E4E9968CAF9DAFAEAFBFAFE997AF
:10A6300044E050E068E074E0CE018B589F4F0E94E8
:10A64000F9EEED961CAE1DAE1EAE1FAEED9744E0CA
:10A6500050E060E274E0CE0187589F4F0E94F9EE0F
:10A66000C358DF4F88829982AA82BB82CD57D040DF
:10A6700044E050E064E274E0CE0183589F4F0E94B2
:10A68000F9EECF57DF4F88829982AA82BB82C158E8
:10A69000D04044E050E068E274E0CE018F579F4F15
:10A6A0000E94F9EECC57DF4F0FB6F894DEBF0FBE15
:10A6B000CDBFDF91CF91FF90EF90DF90CF90BF9013
:10A6C000AF909F908F907F906F905F904F90089584
:10A6D0001F93CF93DF93CDB7DEB7CC59D1090FB617
:10A6E000F894DEBF0FBECDBF182F409149025091A4
:10A6F0004A0260914B0270914C028BE490E00E9400
:10A7000010EF4091190D50911A0D60911B0D709131
:10A710001C0D8FE490E00E9410EF40914F02509189
:10A720005002609151027091520283E590E00E94C4
:10A7300010EF8091390290913A02A0913B02B091C2
:10A740003C0289A79AA7ABA7BCA744E050E063E00E
:10A7500070E0CE0189960E94F9EE80913D029091C1
:10A760003E02A0913F02B09140028DA79EA7AFA7E5
:10A77000B8AB44E050E067E070E0CE018D960E94F7
:10A78000F9EE8091410290914202A0914302B09172
:10A79000440289AB9AABABABBCAB44E050E06BE09E
:10A7A00070E0CE01C1960E94F9EE80915F02909117
:10A7B0006002A0916102B09162028DAB9EABAFAB23
:10A7C000B8AF44E050E06FE070E0CE01C5960E9463
:10A7D000F9EE8091630290916402A0916502B091BC
:10A7E000660289AF9AAFABAFBCAF44E050E063E123
:10A7F00070E0CE01C9960E94F9EE809167029091B7
:10A800006802A0916902B0916A0221968CAF9DAF57
:10A81000AEAFBFAF219744E050E067E170E0CE01FA
:10A82000CD960E94F9EE8091530290915402A0912E
:10A830005502B091560225968CAF9DAFAEAFBFAF1B
:10A84000259744E050E06BE170E0CE018F5B9F4FB5
:10A850000E94F9EE8091570290915802A0915902FE
:10A86000B0915A0229968CAF9DAFAEAFBFAF29977A
:10A8700044E050E06FE170E0CE018B5B9F4F0E949F
:10A88000F9EE80915B0290915C02A0915D02B09123
:10A890005E022D968CAF9DAFAEAFBFAF2D9744E05B
:10A8A00050E063E270E0CE01875B9F4F0E94F9EEBB
:10A8B0008091270D9091280DA091290DB0912A0D1E
:10A8C00061968CAF9DAFAEAFBFAF619744E050E0F3
:10A8D00067E270E0CE01835B9F4F0E94F9EE8091AA
:10A8E000230D9091240DA091250DB091260D659614
:10A8F0008CAF9DAFAEAFBFAF659744E050E06FE265
:10A9000070E0CE018F5A9F4F0E94F9EE8091440370
:10A9100090914503A0914603B091470369968CAF8F
:10A920009DAFAEAFBFAF699744E050E063E370E026
:10A93000CE018B5A9F4F0E94F9EE8091480390916F
:10A940004903A0914A03B0914B036D968CAF9DAF24
:10A95000AEAFBFAF6D9744E050E067E370E0CE016B
:10A96000875A9F4F0E94F9EE80914C0390914D03BE
:10A97000A0914E03B0914F03A1968CAF9DAFAEAFA7
:10A98000BFAFA19744E050E06BE370E0CE01835A83
:10A990009F4F0E94F9EE8091340390913503A0916E
:10A9A0003603B0913703A5968CAF9DAFAEAFBFAF66
:10A9B000A59744E050E06FE370E0CE018F599F4FC0
:10A9C0000E94F9EE8091380390913903A0913A03E7
:10A9D000B0913B03A9968CAF9DAFAEAFBFAFA99727
:10A9E00044E050E063E470E0CE018B599F4F0E9439
:10A9F000F9EE80913C0390913D03A0913E03B0910C
:10AA00003F03AD968CAF9DAFAEAFBFAFAD9744E007
:10AA100050E067E470E0CE0187599F4F0E94F9EE45
:10AA2000609172028AE690E00E9402EF6091B502A6
:10AA30007091B60288E194E00E9415EF60918D025A
:10AA40008BE690E00E9402EF60918E028CE790E02E
:10AA50000E9402EF80918F0290919002A09191024A
:10AA6000B0919202E1968CAF9DAFAEAFBFAFE197D0
:10AA700044E050E06CE670E0CE0183599F4F0E94A5
:10AA8000F9EE8091930290919402A0919502B09179
:10AA90009602E5968CAF9DAFAEAFBFAFE59744E0B1
:10AAA00050E060E770E0CE018F589F4F0E94F9EEB2
:10AAB0008091970290919802A0919902B0919A0288
:10AAC000E9968CAF9DAFAEAFBFAFE99744E050E0E1
:10AAD00064E770E0CE018B589F4F0E94F9EE6091C1
:10AAE0009B0288E790E00E9402EF80911A0C9091FF
:10AAF0001B0CA0911C0CB0911D0CED968CAF9DAF62
:10AB0000AEAFBFAFED9744E050E065E870E0CE0136
:10AB100087589F4F0E94F9EE8091160C9091170C68
:10AB2000A091180CB091190CC358DF4F88839983FA
:10AB3000AA83BB83CD57D04044E050E069E870E081
:10AB4000CE0183589F4F0E94F9EE8091120C909194
:10AB5000130CA091140CB091150CCF57DF4F8883C4
:10AB60009983AA83BB83C158D04044E050E06DE88C
:10AB700070E0CE018F579F4F0E94F9EE8091260C16
:10AB80009091270CA091280CB091290CCB57DF4F46
:10AB900088839983AA83BB83C558D04044E050E0A2
:10ABA00061E970E0CE018B579F4F0E94F9EE8091D2
:10ABB000220C9091230CA091240CB091250CC75726
:10ABC000DF4F88839983AA83BB83C958D04044E070
:10ABD00050E065E970E0CE0187579F4F0E94F9EE83
:10ABE00080911E0C90911F0CA091200CB091210C13
:10ABF000C357DF4F88839983AA83BB83CD58D04046
:10AC000044E050E069E970E0CE0183579F4F0E9415
:10AC1000F9EECF56DF4F188219821A821B82C15972
:10AC2000D04044E050E06DE970E0CE018F569F4F78
:10AC30000E94F9EECB56DF4F188219821A821B82CE
:10AC4000C559D04044E050E061EA70E0CE018B5637
:10AC50009F4F0E94F9EEC756DF4F188219821A8261
:10AC60001B82C959D04044E050E065EA70E0CE0153
:10AC700087569F4F0E94F9EE6091F60B84E094E0B6
:10AC80000E9402EF81E08093AE0C8091C40290910B
:10AC9000C502A091C602B091C7028D839E83AF8387
:10ACA000B88744E050E068EC70E0CE0105960E9461
:10ACB000F9EE8091CA029091CB02A091CC02B091A2
:10ACC000CD0289879A87AB87BC8744E050E06CEC63
:10ACD00070E0CE0109960E94F9EE8091D202909127
:10ACE000D302A091D402B091D5028D879E87AF8701
:10ACF000B88B44E050E060ED70E0CE010D960E940C
:10AD0000F9EE8091CE029091CF02A091D002B09145
:10AD1000D102898B9A8BAB8BBC8B44E050E064ED05
:10AD200070E0CE0141960E94F9EE6091E30288ED59
:10AD300090E00E9402EF609126037091270386E263
:10AD400091E00E9415EF6091FE0289ED90E00E9473
:10AD500002EF6091FF0285EF90E00E9402EF809188
:10AD6000000390910103A0910203B09103038D8B26
:10AD70009E8BAF8BB88F44E050E06AED70E0CE015F
:10AD800045960E94F9EE8091040390910503A091ED
:10AD90000603B0910703898F9A8FAB8FBC8F44E075
:10ADA00050E06EED70E0CE0149960E94F9EE809180
:10ADB000080390910903A0910A03B0910B038D8FB2
:10ADC0009E8FAF8FB8A344E050E062EE70E0CE01FA
:10ADD0004D960E94F9EE60910C0386EE90E00E9481
:10ADE00002EF4091B8025091B9026091BA0270919D
:10ADF000BB0287EE90E00E9410EF4091BC025091A0
:10AE0000BD026091BE027091BF028BEE90E00E9485
:10AE100010EF4091C0025091C1026091C202709146
:10AE2000C30282E291E00E9410EF6091DA02709119
:10AE3000DB028FEE90E00E9415EF6091DC027091D2
:10AE4000DD028AEF90E00E9415EF6091DE027091C2
:10AE5000DF028CEF90E00E9415EF60912C038EEFE3
:10AE600090E00E9402EF19A21AA21BA21CA244E0C9
:10AE700050E061EF70E0CE0181960E94F9EE1DA2D4
:10AE80001EA21FA218A644E050E066EF70E0CE01BB
:10AE900085960E94F9EE1123A1F040E050E0BA013E
:10AEA0008DE790E00E9410EF19821A821B821C82AB
:10AEB00044E050E061E870E0CE0101960E94F9EEB6
:10AEC000D4D963E189E690E00E9402EF0E94003944
:10AED000682F88E690E00E9402EFC456DF4F0FB65D
:10AEE000F894DEBF0FBECDBFDF91CF911F910895C3
:10AEF0008F929F92AF92BF92CF92DF92EF92FF928A
:10AF00001F93CF93DF93CDB7DEB7C857D1090FB6E4
:10AF1000F894DEBF0FBECDBFF82E89E690E00E9408
:10AF2000E7EE182F682F70E087E79AE20E94FA494F
:10AF30008BE490E00E94EFEE6093490270934A0226
:10AF400080934B0290934C028FE490E00E94EFEECE
:10AF50006093190D70931A0D80931B0D90931C0D27
:10AF600083E590E00E94EFEE60934F0270935002F1
:10AF7000809351029093520283E090E05ED96093F7
:10AF8000390270933A0280933B0290933C0287E02F
:10AF900090E053D960933D0270933E0280933F024C
:10AFA000909340028BE090E048D960934102709307
:10AFB000420280934302909344028FE090E03DD997
:10AFC00060935F02709360028093610290936202CB
:10AFD00083E190E032D960936302709364028093BE
:10AFE00065029093660287E190E027D9609367023B
:10AFF000709368028093690290936A028BE190E0FB
:10B000001CD960935302709354028093550290931D
:10B0100056028FE190E011D9609357027093580265
:10B020008093590290935A0283E290E006D960938C
:10B030005B0270935C0280935D0290935E0287E2F4
:10B0400090E0FBD86093270D7093280D8093290D15
:10B0500090932A0D8FE290E0F0D86093230D7093C7
:10B06000240D8093250D9093260D83E390E0E5D881
:10B070006093440370934503809346039093470382
:10B0800087E390E0DAD86093480370934903809394
:10B090004A0390934B038BE390E0CFD860934C032B
:10B0A00070934D0380934E0390934F038FE390E092
:10B0B000C4D8609334037093350380933603909320
:10B0C000370383E490E0B9D8609338037093390371
:10B0D00080933A0390933B0387E490E0AED860936B
:10B0E0003C0370933D0380933E0390933F038AE6B5
:10B0F00090E00E94E7EE8093720288E194E00E9463
:10B10000F4EE9093B6028093B5028BE690E00E9435
:10B11000E7EE80938D028CE790E00E94E7EE80934B
:10B120008E028CE690E089D860938F027093900233
:10B13000809391029093920280E790E07ED8609392
:10B14000930270939402809395029093960284E701
:10B1500090E073D86093970270939802809399025D
:10B1600090939A0288E790E00E94E7EE80939B021A
:10B1700085E890E062D860931A0C70931B0C809362
:10B180001C0C90931D0C89E890E057D86093160C26
:10B190007093170C8093180C9093190C8DE890E025
:10B1A0004CD86093120C7093130C8093140C9093F2
:10B1B000150C81E990E041D86093260C7093270C20
:10B1C0008093280C9093290C85E990E036D8609301
:10B1D000220C7093230C8093240C9093250C89E906
:10B1E00090E02BD860931E0C70931F0C8093200C62
:10B1F0009093210CFF2009F4BFC081E08093AE0C36
:10B2000088EC90E01AD86093C4027093C5028093D2
:10B21000C6029093C7028CEC90E00FD86093CA02EC
:10B220007093CB028093CC029093CD0280ED90E09E
:10B2300004D86093D2027093D3028093D402909387
:10B24000D50284ED90E00E941D516093CE02709370
:10B25000CF028093D0029093D10288ED90E00E94BB
:10B26000E7EE8093E30286E291E00E94F4EE909391
:10B2700027038093260389ED90E00E94E7EE8093F8
:10B28000FE0285EF90E00E94E7EE8093FF028AEDD8
:10B2900090E00E941D51609300037093010380931E
:10B2A0000203909303038EED90E00E941D51609382
:10B2B000040370930503809306039093070382EEC3
:10B2C00090E00E941D5160930803709309038093DE
:10B2D0000A0390930B0386EE90E00E94E7EE8093C2
:10B2E0000C0387EE90E00E94EFEE6093B80270933B
:10B2F000B9028093BA029093BB028BEE90E00E9459
:10B30000EFEE6093BC027093BD028093BE029093F7
:10B31000BF028FEE90E00E94F4EE9093DB028093E8
:10B32000DA028AEF90E00E94F4EE9093DD028093BF
:10B33000DC028CEF90E00E94F4EE9093DF028093A9
:10B34000DE02123008F00BC24091C0025091C102DF
:10B350006091C2027091C30282E291E00E9410EFFC
:10B3600082E291E00E94EFEE6093C0027093C1020E
:10B370008093C2029093C302133109F418C283E58B
:10B380009AE20E945350133008F0F3C180E090E03D
:10B39000A0E2B2E461968CAF9DAFAEAFBFAF619754
:10B3A00044E050E068E273E0CE01835B9F4F0E946F
:10B3B000F9EE80E090E0A0E0B0E465968CAF9DAF40
:10B3C000AEAFBFAF659744E050E06CE273E0CE01F2
:10B3D0008F5A9F4F0E94F9EE80E090E0A6E1B3E41F
:10B3E00069968CAF9DAFAEAFBFAF699744E050E0B8
:10B3F00068E473E0CE018B5A9F4F0E94F9EE6D9680
:10B400001CAE1DAE1EAE1FAE6D9744E050E060E274
:10B4100073E0CE01875A9F4F0E94F9EEA1961CAEB1
:10B420001DAE1EAE1FAEA19744E050E064E273E093
:10B43000CE01835A9F4F0E94F9EEC12CD12C90EA85
:10B44000E92E91E4F92EA596CCAEDDAEEEAEFFAEC0
:10B45000A59744E050E060E373E0CE018F599F4F21
:10B460000E94F9EEA996CCAEDDAEEEAEFFAEA99786
:10B4700044E050E064E373E0CE018B599F4F0E949B
:10B48000F9EE812C912C20E2A22E23E4B22EAD966F
:10B490008CAE9DAEAEAEBFAEAD9744E050E068E37B
:10B4A00073E0CE0187599F4F0E94F9EEE196CCAE32
:10B4B000DDAEEEAEFFAEE19744E050E06CE373E04A
:10B4C000CE0183599F4F0E94F9EEE596CCAEDDAEDA
:10B4D000EEAEFFAEE59744E050E060E473E0CE01ED
:10B4E0008F589F4F0E94F9EEE9968CAE9DAEAEAE9E
:10B4F000BFAEE99744E050E064E473E0CE018B58BE
:10B500009F4F0E94F9EE80E090E0A0E2B1E42D961A
:10B510008CAF9DAFAEAFBFAF2D9744E050E061EA76
:10B5200073E0CE01875B9F4F0E94F9EE21961CAE1F
:10B530001DAE1EAE1FAE219744E050E060ED73E0FB
:10B54000CE01CD960E94F9EE25961CAE1DAE1EAE24
:10B550001FAE259744E050E064ED73E0CE018F5BB1
:10B560009F4F0E94F9EE29961CAE1DAE1EAE1FAE77
:10B57000299744E050E068ED73E0CE018B5B9F4F6C
:10B580000E94F9EE60E08CED93E00E9402EF80E013
:10B5900090E0A0E4B0E489A39AA3ABA3BCA344E0E9
:10B5A00050E060EE73E0CE0181960E94F9EE80E0FB
:10B5B00090E0A0E5B1E48DA39EA3AFA3B8A744E0BB
:10B5C00050E064EE73E0CE0185960E94F9EE80E0D3
:10B5D00090E0A0E2B2E489A79AA7ABA7BCA744E099
:10B5E00050E068EE73E0CE0189960E94F9EE1DA648
:10B5F0001EA61FA618AA44E050E06CEE73E0CE0130
:10B600008D960E94F9EE19AA1AAA1BAA1CAA44E058
:10B6100050E060EF73E0CE01C1960E94F9EE1DAAE2
:10B620001EAA1FAA18AE44E050E064EF73E0CE01FA
:10B63000C5960E94F9EE80E090E0A0EAB1E489AFFF
:10B640009AAFABAFBCAF44E050E068EF73E0CE011F
:10B65000C9960E94F9EE60E08CEF93E00E9402EF41
:10B660001D8E1E8E1F8E18A244E050E060E074E034
:10B67000CE014D960E94F9EE6EEF84E094E00E94B8
:10B6800002EF8EEF8093F60B1D861E861F86188AAA
:10B6900044E050E06CE074E0CE010D960E94F9EEBB
:10B6A000198A1A8A1B8A1C8A44E050E060E174E01F
:10B6B000CE0141960E94F9EE1D8A1E8A1F8A188EBD
:10B6C00044E050E064E174E0CE0145960E94F9EE5A
:10B6D00080E090E0A8ECB2E4898F9A8FAB8FBC8FAA
:10B6E00044E050E068E074E0CE0149960E94F9EE33
:10B6F00087E390E09093B6028093B50282ED90E0EC
:10B70000909327038093260319821A821B821C823E
:10B7100044E050E060E274E0CE0101960E94F9EE50
:10B72000C12CD12C80E2E82E81E4F82ECD82DE827D
:10B73000EF82F88644E050E064E274E0CE010596C2
:10B740000E94F9EEC986DA86EB86FC8644E050E07A
:10B7500068E274E0CE0109960E94F9EE25C08EEFF2
:10B7600090E00E94E7EE80932C031D3008F0F8CDA6
:10B77000EBCD183008F4C7CE1A3008F4D7CE1A3003
:10B7800009F400CF1B3009F402CF1E3008F468CF53
:10B790001E3009F471CF1F3009F476CF103109F44F
:10B7A000A7CF133108F4B0CF80E00E94685380E047
:10B7B00094E00E941D516093BF107093C01080935D
:10B7C000C1109093C21084E094E00E94E7EE0E94C2
:10B7D000A9320E94C1408FE692E00E94B938C85851
:10B7E000DF4F0FB6F894DEBF0FBECDBFDF91CF9114
:10B7F0001F91FF90EF90DF90CF90BF90AF909F9000
:10B800008F9008958F929F92AF92BF92CF92DF92C6
:10B81000EF92FF922FE632E143E85AE36091CD0CBC
:10B820007091CE0C8091CF0C9091D00C0E9420EEA4
:10B830006B017C0181E890E00E941D519B01AC01ED
:10B84000C701B6010E9463EFAB01BC0122E080E6B4
:10B850009CE10E944E3A8DE59CE10E949F3920E0D8
:10B8600030E040E751E46091EA027091EB02809190
:10B87000EC029091ED020E9476F118160CF455C07E
:10B88000C12CD12C76018DE790E00E94EFEEC60E20
:10B89000D71EE81EF91EC701B60120E831E541E0D8
:10B8A00050E00E94A6F260E87EEA8EEF9FEF0E94D1
:10B8B00018EFC60ED71EE81EF91EBA01A9018EE4C4
:10B8C0009CE10E94603AC701B60120E13EE040E001
:10B8D00050E00E94A6F249015A01BA01A90187E489
:10B8E0009CE10E94603AA0EFB1EFA50194010E9493
:10B8F000D2F26C0D7D1D8E1D9F1D2CE330E040E0CB
:10B9000050E00E94A6F2BA01A9018FE39CE10E94D7
:10B91000603A8AE39CE1FF90EF90DF90CF90BF9078
:10B92000AF909F908F900C94044B0E943E29C09042
:10B93000D10CD090D20CE090D30CF090D40C6C19B8
:10B940007D098E099F0928EE33E040E050E00E9417
:10B9500027EF69017A0197CF2F923F924F925F9222
:10B960006F927F928F929F92AF92BF92CF92DF920F
:10B97000EF92FF920F931F93CF93DF93CDB7DEB774
:10B98000A4970FB6F894DEBF0FBECDBF4B015C018C
:10B99000D42E122F3324339420E030E040E751E4DA
:10B9A0006091EA027091EB028091EC029091ED02BD
:10B9B0000E9476F118160CF0312C81E03826398E71
:10B9C00020E030E849E853E4C501B4010E9476F173
:10B9D00018160CF491C220E030E0A901C501B401B1
:10B9E0000E94BBED87FD90C22D2C312CF101EE0F92
:10B9F000FF1FE65AFC4FE080F180D70111968C9131
:10BA0000882309F485C220E030E040E252E4C50119
:10BA1000B4010E94BBED87FF7FC2F701EE5BFF4FD1
:10BA20001082118212821382D7011A968D929D92F2
:10BA3000AD92BC921D97D5968C91D597897FD5965E
:10BA40008C93C7010E94B938112371F020E030E0D7
:10BA500040E252E4C501B4010E9476F1181624F4C4
:10BA6000F70185A9816085AB20E030E048E452E42D
:10BA7000C501B4010E9476F187FD10C02CE7229D1C
:10BA8000C001239D900D112489549D4FFC01EA585B
:10BA9000FF4F8B589F4FDC018C9180836D2D70E0A0
:10BAA00090E080E00E94BFEDAB01BC0120E08EEE93
:10BAB0009AE20E944E3A20E0B501A4018CEE9AE28F
:10BAC0000E94AE40002309F47AC120E030E040E259
:10BAD00052E4C501B4010E9476F118160CF06FC152
:10BAE000F701228533854485558566817781808578
:10BAF00091850E9462EF4B015C0120E030E0A901DA
:10BB00000E9476F118160CF01DC220E030E040E0F3
:10BB100050E4C501B4010E94BBED182F111F11277D
:10BB2000111F81E0182709F44AC11CE7D19EC0010A
:10BB300011249C0129543D4F3B8F2A8F81EA90E0CC
:10BB40000E94983260E00E94A6C80E9444CA129DDA
:10BB5000F001139DF00D1124E954FD4F83A994A920
:10BB6000A5A9B6A98F87988BA98BBA8B27A530A9D1
:10BB700041A952A92B8B3C8B4D8B5E8B8091CC0CB9
:10BB8000382F30713C8F80618093CC0C1D821E82D7
:10BB90001F82188610E019861A861B861C86AF0144
:10BBA000415D5F4F5E874D87CF01C396988F8F8B26
:10BBB000DF019796BE8FAD8F9F012B5D3F4F38A35E
:10BBC0002F8F4C5151095AA349A340979CA38BA393
:10BBD0000E943E292B013C0140924F0C5092500C88
:10BBE0006092510C7092520C81E0E6D283E090E0BA
:10BBF0000E94284B80911E0D90911F0DAA8DBB8D28
:10BC00008A179B0709F0ACC1ED8DFE8DE080F180B5
:10BC10001E141F040CF0A4C11111A2C12B893C8970
:10BC20004D895E896F85788989899A890E9476F124
:10BC300018160CF095C1AF8DB8A16D917C91072EAF
:10BC4000000C880B990B0E94C1ED9B01AC01ED85A6
:10BC5000FE8560817181828193810E9476F1181640
:10BC6000ECF5662777276E197F09072E000C880BE5
:10BC7000990B0E94C1ED20914502309146024091FE
:10BC80004702509148020E9420EE0E9494F05B010E
:10BC90006C0181E08F931F921F9220E030E040E81A
:10BCA0005EE3A9A1BAA16D917D918D919C910E94B5
:10BCB00020EE9F938F937F936F93E12CF12C87015C
:10BCC00020E030E0A90160E070E0CB010E94677ADB
:10BCD0000FB6F894DEBF0FBECDBF11E02D813E81BF
:10BCE0004F815885232B242B252B09F44FC18D819F
:10BCF0009E81AF81B88584199509A609B709811578
:10BD00009449A543B74708F063C18091CC0C4C8D92
:10BD1000442309F4DBC180618093CC0C112309F426
:10BD20004EC080911E0D90911F0DAA8DBB8D8A175C
:10BD30009B0709F044C08CE7829D8001839D100D14
:10BD4000112409541D4FF80167A170A5072E000C9E
:10BD5000880B990B0E94C1ED20914502309146025B
:10BD600040914702509148020E9420EE0E9494F0B8
:10BD70005B016C0181E08F931F921F9220E030E005
:10BD800040E85EE3D80153966D917D918D919C9131
:10BD900056970E9420EE9F938F937F936F93E12C91
:10BDA000F12C870120E030E0A90160E070E0CB01D8
:10BDB0000E94677A0FB6F894DEBF0FBECDBF109217
:10BDC000A00D20E030E040E751E46091EA0270917C
:10BDD000EB028091EC029091ED020E9476F1181630
:10BDE0000CF476C1498D41116EC020E030E0A9010C
:10BDF0006091CD0C7091CE0C8091CF0C9091D00CB5
:10BE00000E94BBED882309F45EC08091200D82FD65
:10BE10005AC00E943E290091D10C1091D20C209161
:10BE2000D30C3091D40C601B710B820B930B28EE5A
:10BE300033E040E050E00E9427EF69017A018DE78E
:10BE400090E00E94EFEEAB01BC014C0D5D1D6E1D3C
:10BE50007F1D8DE790E00E9410EF81E890E00E9446
:10BE60001D516B017C012FE632E143E85AE36091FA
:10BE7000CD0C7091CE0C8091CF0C9091D00C0E9483
:10BE800020EEA70196010E9463EF69837A838B837A
:10BE90009C8344E050E061E870E0CE0101960E948E
:10BEA000F9EE8091200D84608093200D0E943E2940
:10BEB0006093D10C7093D20C8093D30C9093D40CDC
:10BEC0000E9417399FDCA4960FB6F894DEBF0FBE10
:10BED000CDBFDF91CF911F910F91FF90EF90DF9039
:10BEE000CF90BF90AF909F908F907F906F905F901A
:10BEF0004F903F902F900895812C90E8992E99E8CB
:10BF0000A92E93E4B92E70CD812C912C54016CCDC7
:10BF1000812C912C540181CD20E030E0A901F70162
:10BF200062857385848595850E94BBED81117CCDEA
:10BF30000E943E29F701EE5BFF4F6083718382838D
:10BF4000938372CD11E020E030E040E050ECC50179
:10BF5000B4010E9476F118160CF4E3CD10E0E1CDA7
:10BF60002D813E814F815885232B242B252B09F0D1
:10BF7000BECE2B893C894D895E896F8578898989F8
:10BF80009A890E9476F118160CF07AC020E030E011
:10BF900040EA50E4AF89B88D6D917D918D919C916F
:10BFA0000E9462EF9B01AC01ED85FE85608171818D
:10BFB000828193810E9476F187FD75C0A301920171
:10BFC00020543B424E4F5F4F2D833E834F83588713
:10BFD00089859A85AB85BC85892B8A2B8B2B09F0AB
:10BFE00040C0AD85BE85CD90DD90ED90FC90EF8991
:10BFF000F88D80809180A280B3802B893C894D8907
:10C000005E896F85788989899A890E9476F120E016
:10C0100030E040E85FE318160CF04AC0C501B401F7
:10C020000E9462EF9B01AC01C701B6010E9476F14C
:10C0300087FDCECDEBA1FCA1A081B18128EE33E03C
:10C040000E94CAF29B01AC01240D351D461D571DEF
:10C0500029873A874B875C87232B242B252B09F4D0
:10C06000B7CD89859A85AB85BC8584199509A609C4
:10C07000B70981159449A543B74708F4A9CD45CE22
:10C0800020E030E040EA50E4AF89B88D6D917D91B9
:10C090008D919C910E9463EFED85FE852081318119
:10C0A0004281538187CF1D821E821F82188690CFC6
:10C0B000C501B4010E9463EF9B01AC01C701B60149
:10C0C0000E94BBED18160CF483CDB4CF8F7E24CE26
:10C0D000398D332309F4F7CE0E943E296093D10CA9
:10C0E0007093D20C8093D30C9093D40C1092CD0CFF
:10C0F0001092CE0C1092CF0C1092D00C8091200D8B
:10C100008B7F8093200DDFCE0F93CF9390911D0DE9
:10C1100090FF02C081114DC090911B0E93FD49C04C
:10C12000C82F5F9A8A9A80910801816080930801E4
:10C13000479A0E94E42880911D0D816080931D0D17
:10C1400080911B0E8E7F80931B0E8091CC0C887F7C
:10C150008093CC0CC11123C000E020E040E060E0FF
:10C1600070E0CB01F9DB40E060E070E0CB010E94C1
:10C17000EB4388ED90E00E94983260E00E94A6C8F0
:10C180000E9444CA269A2E9A80911B0E8F7B88604B
:10C1900080931B0E80E0CF910F910C94695084EA3C
:10C1A00090E00E94983260E00E94A6C80E9444CAB3
:10C1B000F1CFCF910F9108952F923F924F925F92BE
:10C1C0006F927F928F929F92AF92BF92CF92DF92A7
:10C1D000EF92FF920F931F93CF93DF93CDB7DEB70C
:10C1E00060970FB6F894DEBF0FBECDBF9091CE031F
:10C1F00091111092CE0390910204992309F449C33E
:10C20000109202049091D0039F5F9A3009F49EC06F
:10C210009093D003888B81E0809322028093AE0CB0
:10C220000E943E2969837A838B839C832AE533E0CD
:10C230003F872E871B861D821C86AE85BF850D918C
:10C240001D91BF87AE87C8010E94DF26CC84C11034
:10C250001EC020E030E048E452E4D80116966D910B
:10C260007D918D919C9119970E94BBED87FF74C0C1
:10C2700020E030E048E452E4F8016285738584856B
:10C2800095850E94BBED87FF67C010922D038091BA
:10C290000102CC848C1509F47CC2D8011696CD908D
:10C2A000DD90ED90FC90199720E030E040E251ECF9
:10C2B000C701B6010E94BBED87FD0BC020E030E056
:10C2C00041E953E4C701B6010E9476F118160CF05B
:10C2D00069C020E030E0A901F8016285738584859A
:10C2E00095850E9476F118160CF05CC07801F2E496
:10C2F000EF0EF11CF70180819181A281B381892B1E
:10C300008A2B8B2B71F58091CF038A3008F468C09B
:10C3100080911D0DD801D5969C91D5979860D596A2
:10C320009C9382FD5AC0846080931D0D80913303DD
:10C3300088600E94064A0E94065082E090E00E94B7
:10C3400004CFB1E0BB87E1E0ED834FC01092D00392
:10C3500061CF31E03C8771CF80912C0380932D0316
:10C3600096CF0E943E29D7018D909D90AD90BC90B4
:10C37000681579058A059B0531F289288A288B285A
:10C3800089F00E943E29F701C080D180E280F380CD
:10C390006C197D098E099F096033754781059105E8
:10C3A00008F0B1CF2C85213001F520E030E04AEFD4
:10C3B00052E46091750270917602809177029091BB
:10C3C00078020E9476F1181684F48091CF038A30A7
:10C3D00008F0C7C08F5F8093CF03F1E0FD8305C0F5
:10C3E0008F5F8093CF0331E03D8330901D0D32FC91
:10C3F000D0C1D80116968D909D90AD90BC901997A4
:10C400001A964D905D906D907C901D97FF24F3944B
:10C41000A3019201C501B4010E9476F187FDF12CC0
:10C42000CC24C394CF24CA86C11009C0D801D596A4
:10C430008C91D59780FF03C08E7FD5968C93CD804D
:10C44000C110BFC0F801FE96C080D180E280F380A9
:10C45000C114D104E104F10409F4B3C029813A8183
:10C460004B815C812E833F8348875987F80186A9D9
:10C4700097A9A0ADB1AD281B390B4A0B5B0BDA01B4
:10C48000C901C816D906EA06FB0608F09AC025A815
:10C49000822D867009F495C080911B0E86FF91C095
:10C4A00021FEA6C022AD33AD44AD55ADC501B401EA
:10C4B0000E9462EF20E030E040E85FE30E94BBEDC5
:10C4C00087FF74C08091CF038F5F8093CF038B3041
:10C4D00008F4EAC0822D8061D801D5968C93832D13
:10C4E000846080931D0D8091330388600E94064A0A
:10C4F00083E090E00E9404CF61E086EB9BE10E9424
:10C50000A6C88FE69BE10E94B34CF80122AD33AD83
:10C5100044AD55AD66817781808591850E9462EF3B
:10C52000AB01BC0122E08BE49BE10E944E3A4981C1
:10C530005A816B817C81F80186A997A9A0ADB1AD24
:10C54000481B590B6A0B7B0B83E49BE10E94603A0A
:10C550008FE39BE10E94044BF1E0FB8721E02D83F8
:10C5600030C0D801D5968C91D5978860D5968C939C
:10C5700087EC9BE10E94B34C80911D0D82FD13C09E
:10C58000846080931D0D8091330388600E94064A69
:10C590000E94065082E090E00E9404CFB1E0BD838B
:10C5A000E1E0EB8722CF21E02D831FCF822D897F11
:10C5B000D801D5968C93BE016F5F7F4FC8010E9452
:10C5C000CB28D8011A96CD90DD90ED90FC901D9768
:10C5D00020E030E040EA51E4C701B6010E94BBED23
:10C5E00087FF65C0F80185A9897F85ABF12C9BC0C9
:10C5F000A3019201C501B4010E9462EF9F7720E080
:10C6000030E040EA51E40E9476F11816DCF58091A2
:10C61000CF038F5F8093CF038B3008F49FCF822DA1
:10C620008061F80185AB832D846080931D0D80911E
:10C63000330388600E94064A83E090E00E9404CFA2
:10C6400061E086EB9BE10E94A6C88FE69BE10E9419
:10C65000B34CD801DA964D915D916D917C91DD9747
:10C6600022E08DE19BE10E944E3AF801468157811C
:10C670006085718522E082E19BE10E944E3A8AE06A
:10C680009BE168CF8E819F81A885B98588519C4F99
:10C69000AF4FBF4F8C199D09AE09BF09F80186AB9A
:10C6A00097ABA0AFB1AF8DCFF1E0FD838ACFD801BA
:10C6B00016962D913D914D915C911997C701B60148
:10C6C0000E9462EF6B017C0120E030E040EA51E41F
:10C6D0000E9476F118160CF0F5C0F801F4A4BE0122
:10C6E0006F5F7F4FC8010E94CB28F80181A992A9F2
:10C6F000A3A9B4A9828F938FA48FB58F8381833030
:10C7000091F4668D70E090E080E00E94BFEDD8016A
:10C710009D966D937D938D939C93D097F80111AA6C
:10C7200012AA13AA14AAF80186809780A084B18463
:10C7300020E030E849E853E4C501B4010E9476F1F5
:10C7400018160CF4F12CD801EC91F0E0EF51F34FF6
:10C75000F0828091D00381110FC01E968D919D9122
:10C760000D90BC91A02DF801828B938BA48BB58B7F
:10C7700086869786A08AB18A80911E0D90911F0DA2
:10C7800089960817190729F4CA84CC2009F47BC2BA
:10C790002F9A2C85213009F0DCCDCD80C11007C047
:10C7A0008091CF03882319F081508093CF03DB84DD
:10C7B000DD20A9F185ED9AE10E94044B1092EA0276
:10C7C0001092EB021092EC021092ED02E091E00266
:10C7D000F0E0EF51F34F10821092790210927A023A
:10C7E00010927B0210927C02E0916F02F0E0EF5118
:10C7F000F34F10828091330383FD08C08091FD0CBC
:10C80000882321F00E94654B80E07EDC8091330319
:10C8100088600E94064A81EC9AE10E946D7B8091BB
:10C82000CC0C84FF22C00E943E290091EB031091A2
:10C83000EC032091ED033091EE036B017C01C01AF3
:10C84000D10AE20AF30A97018601093E1340210545
:10C85000310558F06093EB037093EC038093ED0384
:10C860009093EE0380E00E94695080910002815015
:10C870008093000281110AC08091EA03882319F095
:10C8800080E00E94695085E08093000288890E94C0
:10C8900008DE60960FB6F894DEBF0FBECDBFDF9105
:10C8A000CF911F910F91FF90EF90DF90CF90BF90AD
:10C8B000AF909F908F907F906F905F904F903F9040
:10C8C0002F90089520E030E040EA51ECC701B60116
:10C8D0000E94BBED87FD8ACED80113968C911397E9
:10C8E000813009F083C0BE016F5F7F4FC8010E9495
:10C8F0008728F80120A131A142A153A1C701B601A7
:10C900000E9420EE4B015C01D8015A962D913D9179
:10C910004D915C915D97C701B6010E9463EF2B01B9
:10C920003C01F801C1A8D2A8E3A8F4A89601A70188
:10C930000E94BBED87FD16C0D8019D96CC909D97B7
:10C940009E96DC909E979F96EC909F97D096FC9039
:10C950009601A701B201C3010E9476F1181614F0E6
:10C9600062017301C601D701F801828F938FA48FF2
:10C97000B58F24A135A146A157A1B601C7010E94D8
:10C9800020EE2DEC3CEC4CEC5DE30E9420EEA5018A
:10C9900094010E9463EF6B017C01D8011E962D91DA
:10C9A0003D914D915C91519752966D917D918D91F4
:10C9B0009C9155970E9462EFF80120A531A542A5F0
:10C9C00053A50E9420EEA70196010E9463EF0E94EA
:10C9D00094F077FD0BCED8019C96FC904F2D50E043
:10C9E000641775070CF4AB01F42E9DCE833009F06B
:10C9F00012C1BE016F5F7F4FC8010E948728F801F6
:10CA0000228933894489558966857785808991890A
:10CA10000E9462EF4B015C0120E030E0A9010E941E
:10CA2000BBED87FF8CC020E030E0A901D8015A9609
:10CA30006D917D918D919C915D970E9476F187FD1E
:10CA40007EC0F80161A872A8F3A9FE83D801D4962C
:10CA5000BC91BD87F80125A436A447A450A820E0C6
:10CA600030E040E05FEBC701B6010E94BBED20E083
:10CA700030E040E251E487FF59C0C201B1010E9499
:10CA800062EF6B017C0193014E815D850E94BBEDDD
:10CA900087FD51C0D8015E967C90672D70E090E0D4
:10CAA00080E00E94C1ED9B01AC01B601C7010E946C
:10CAB00076F1181644F4672D70E090E080E00E9453
:10CAC000BFED6B017C01C601D701F80185A796A7D0
:10CAD000A7A7B0ABD80190962D913D914D915C9157
:10CAE0009397C501B4010E9420EEF8012681378199
:10CAF000408551850E9463EFD8011A962D913D9192
:10CB00004D915C911D970E9476F118160CF07BC038
:10CB1000F80161A972A983A994A90E9499F0F62E3F
:10CB2000F801828E938EA48EB58EFDCDC201B10127
:10CB30000E9463EFA6CF6301EE80FD84C4CF20E0A6
:10CB400030E0A901C501B4010E9476F118160CF07D
:10CB5000C1CF20E030E0A901D8015A966D917D91B6
:10CB60008D919C915D970E94BBED18160CF4B2CF8D
:10CB7000F80141A852A863A874A820E030E040E082
:10CB80005FE3C701B6010E9476F120E030E040E2A9
:10CB900051E4181674F5C301B2010E9463EF6B01F2
:10CBA0007C0120E030E0A9010E94BBED87FD26C09A
:10CBB00020E030E040EA51E4D8019D966D917D91EE
:10CBC0008D919C91D0970E9462EF2B013C019B01BB
:10CBD000AC01B601C7010E9476F1181614F4620187
:10CBE0007301C601D701F80181AB92ABA3ABB4AB23
:10CBF00071CFC301B2010E9462EFD1CFC12CD12C01
:10CC0000E12CF12CEECFD8019D966D917D918D9107
:10CC10009C91D09782CF823071F589819A81AB81C6
:10CC2000BC81F80146895789608D718D6C017D0149
:10CC3000C41AD50AE60AF70AB701A60149385341D2
:10CC40006105710508F4A5CDCA84F12CC110F4A4C6
:10CC5000F801868B978BA08FB18FCA84CC2039F0D6
:10CC6000BE016F5F7F4FC8010E94CB285CCD85A9B4
:10CC7000897F85AB58CD8111B9CCCA84CC2029F0ED
:10CC80009C96FC90EDCF2F9884CDD5968C91D5971E
:10CC9000897FD5968C93AACC2F923F924F925F9228
:10CCA0006F927F928F929F92AF92BF92CF92DF92BC
:10CCB000EF92FF920F931F93CF93DF93CDB7DEB721
:10CCC000C755D1090FB6F894DEBF0FBECDBF082FF0
:10CCD00063966FAF639790911B0E80911D0D95FD2C
:10CCE0005FC09091200D96FD5BC04091460450912D
:10CCF00047046091480470914904C0907104D09039
:10CD00007204E0907304F09074044C155D056E0598
:10CD10007F0544F44093710450937204609373044C
:10CD20007093740440914204509143046091440410
:10CD300070914504C0907504D0907604E09077041B
:10CD4000F09078044C155D056E057F0544F4409322
:10CD5000750450937604609377047093780485FD8E
:10CD60001FC040913E0450913F0460914004709177
:10CD70004104C0907904D0907A04E0907B04F09054
:10CD80007C044C155D056E057F0554F486FD08C0D6
:10CD90004093790450937A0460937B0470937C04ED
:10CDA0008E7F80931D0D9FB7F8948091FD0C9FBFDF
:10CDB000803118F080E000DAF6CF8091FD0C81110F
:10CDC00047C080914B0490914C04892B09F040C0DE
:10CDD00063961FAD63971123D9F194E047E751E0C3
:10CDE00067E0E0EACE2EE6E8DE2EEE24E394F12CB6
:10CDF00091508091F50B282F30E09F3F09F4C3C17B
:10CE0000429FF001439FF00D1124EB57FB4F5183DC
:10CE1000608314829383C582D682E782F0868F3046
:10CE2000A8F48F5F8093F50B2091AA0C3091AB0C86
:10CE300020613093AB0C2093AA0C2FB7F89480910B
:10CE4000FD0C8F5F8093FD0C2FBFD2CF80E0EACF27
:10CE500010E02091F50B29A7422F50E058A74FA3CF
:10CE600080E1011101C080E097E7AFA1B8A59A9FCA
:10CE7000F0019B9FF00D1124EB57FB4F81836396CC
:10CE80000FAD6397002309F482C1108287E72FA1B9
:10CE900038A5829FF001839FF00D1124EB57FB4FC3
:10CEA00014821092810410928204109283041092D2
:10CEB00084040091AF0C2E960FAF2E972091230281
:10CEC00030912402409125025091260262962CAFA7
:10CED0003DAF4EAF5FAF629740906D0450906E04CF
:10CEE00060906F0470907004C090CD0CD090CE0C08
:10CEF000E090CF0CF090D00C41E754E021965FAF6A
:10CF00004EAF2197A0EBBCE0B8ABAFA739A5389FD7
:10CF1000900111242D963FAF2EAF2D9722573B4FF6
:10CF20003AA329A347EE5CE058AF4FABCE01419640
:10CF30009CAB8BAB312C212CDF015596BCAFABAF3A
:10CF40009F012C5F3F4F3CA72BA7022D2196EEADF2
:10CF5000FFAD219781919191A191B1912196FFAF60
:10CF6000EEAF21978BA39CA3ADA3BEA3EFA5F8A919
:10CF700081919191A191B191F8ABEFA72BA13CA127
:10CF80004DA15EA1281B390B4A0B5B0BDA01C901CD
:10CF9000E9A1FAA180839183A283B383F3E02F12E6
:10CFA00043C02E962FAD2E9721113EC0ABADBCAD28
:10CFB0006D917D918D919C910E94C1ED62962CADF9
:10CFC0003DAD4EAD5FAD62970E9420EEA301920190
:10CFD0000E9463EF2B013C010E9494F0EBADFCAD8D
:10CFE00060837183828393830E94C1ED4B015C0156
:10CFF000AC019B01C301B2010E9462EF2B013C0115
:10D000002091F30C3091F40C4091F50C5091F60CFA
:10D01000C501B4010E9420EE9B01AC01C701B6011D
:10D020000E9463EF6B017C01E9A1FAA180819181EB
:10D03000A281B381B7FDAEC0ABA5BCA58C9121E0A8
:10D0400030E0002E01C0220F0A94EAF7822B8C9365
:10D05000A9A1BAA18D909D90AD90BD90BAA3A9A3AE
:10D06000AFA9B8AD2D913D914D915D91B8AFAFABEA
:10D0700027962CAF3DAF4EAF5FAF2797C501B401E8
:10D080000E94C1ED27962CAD3DAD4EAD5FAD27970B
:10D090000E9420EEEBA9FCA9619371938193919377
:10D0A000FCABEBAB89288A288B2859F020E130E0D3
:10D0B00001C0220F0A95EAF7ABA5BCA58C91822B83
:10D0C0008C93EFA5F8A934972BA13CA14DA15EA1AB
:10D0D00020833183428353833FEF231A330A44E092
:10D0E0002416310409F031CF40926D0450926E0441
:10D0F00060926F0470927004C092CD0CD092CE0CEE
:10D10000E092CF0CF092D00C87E7AFA1B8A58A9F30
:10D11000F0018B9FF00D1124EB57FB4F128204811D
:10D1200009A3802F807F09F045C0112391F0109250
:10D13000FD0C19A510934A048091AA0C9091AB0C98
:10D140002091CC0C23FF34C080619093AB0C809372
:10D15000AA0CC95ADF4F0FB6F894DEBF0FBECDBF81
:10D16000DF91CF911F910F91FF90EF90DF90CF90C3
:10D17000BF90AF909F908F907F906F905F904F90F7
:10D180003F902F90089563961FAD639762CE82E023
:10D1900080837CCEB095A095909581959F4FAF4FA1
:10D1A000BF4FE9A1FAA180839183A283B38350CFBB
:10D1B0008F7ECBCF25853685478550892BA73CA709
:10D1C0004DA75EA781859285A385B4858FA798AB6F
:10D1D000A9ABBAAB82179307A407B507ACF4818952
:10D1E0009289A389B48982179307A407B50764F4C9
:10D1F00085899689A789B08D82179307A407B507FB
:10D200001CF481E0838327C087E70FA118A5809FC6
:10D21000F001819FF00D1124EB57FB4F818992891A
:10D22000A389B4892FA538A949A95AA982179307B8
:10D23000A407B5070CF04EC4458956896789708DDF
:10D240000FA518A929A93AA9401751076207730722
:10D250000CF040C4138227E70FA118A5209FC0013E
:10D26000219F900D1124DC01AB57BB4F13961C91ED
:10D2700013972F961FAF2F9724E0120280011124DD
:10D2800066961FAF0EAF6697800F911FFC01EB579C
:10D29000FB4F018512852385348527960CAF1DAF82
:10D2A0002EAF3FAF2797FD01ED58FF4F008311834D
:10D2B0002283338319A1107764961FAF64972D8D55
:10D2C0003E8D4F8D58A12BAB3CAB4DAB5EAB690196
:10D2D0007A01E894F7F809A100742E960FAF2E9703
:10D2E000112309F423C469897A898B899C898D88E3
:10D2F0009E88AF88B88C9B01AC010E9420EE2B0168
:10D300003C01A5019401C501B4010E9420EE9B01DE
:10D31000AC01C301B2010E9463EF4B015C01002329
:10D3200009F4EFC3698D7A8D8B8D9C8D9B01AC01C7
:10D330000E9420EEA50194010E9463EF0E9422F258
:10D340005B018C01A70196010E94BBED87FF02C023
:10D350005601870187E72FA138A5829FF001839F9F
:10D36000F00D1124E652FB4FC501D8018083918353
:10D37000A283B38387E70FA118A5809FF001819F47
:10D38000F00D1124E652FB4F2081318142815381FF
:10D390002BAF3CAF4DAF5EAF8091530C9091540CCE
:10D3A000A091550CB091560C23968CAF9DAFAEAFAB
:10D3B000BFAF239720E034E244E75BE46BAD7CAD84
:10D3C0008DAD9EAD0E9420EE23962CAD3DAD4EADB1
:10D3D0005FAD23970E942CF06B017C018091FD0CC6
:10D3E0008A30A0F520E034E244E758E4C701B601F2
:10D3F0000E94BBED87FF2AC01091FD0CA70196018A
:10D4000060E074E284E798E40E9462EF20E030E09C
:10D4100040E450E40E9420EE4B015C01612F70E07B
:10D420006F5F7F4F072E000C880B990B0E94C1ED98
:10D430009B01AC01C501B4010E942CF09B01AC0121
:10D44000C701B6010E9463EF6B017C0187E7AFA1C2
:10D45000B8A58A9F80018B9F100D11240B571B4F7D
:10D46000C701B6010E9494F0F80165837683878333
:10D47000908727966CAD7DAD8EAD9FAD27970E94AE
:10D48000C1ED2B966CAF7DAF8EAF9FAF2B979B01FD
:10D49000AC01C701B6010E942CF00E9494F02B0150
:10D4A0003C012B962CAD3DAD4EAD5FAD2B9760E0B2
:10D4B00074E284E79BE40E942CF06BA37CA38DA311
:10D4C0009EA319A1107109A104FF38C329893A89C3
:10D4D0004B895C890E9420EE20915F0230916002AE
:10D4E00040916102509162020E942CF00E9494F0DF
:10D4F00069837A838B839C835301420146165706C6
:10D500006806790614F44B015C0109A1007229A197
:10D5100025FF1BC32D893E894F89588D6BA17CA1A6
:10D520008DA19EA10E9420EE2091630230916402A1
:10D5300040916502509166020E942CF00E9494F086
:10D540006D837E838F83988786169706A806B90613
:10D5500014F44B015C012E963FAD2E97332309F452
:10D56000F9C2298D3A8D4B8D5C8D6BA17CA18DA16B
:10D570009EA10E9420EE20916702309168024091A6
:10D58000690250916A020E942CF00E9494F069870F
:10D590007A878B879C8786169706A806B90614F4A7
:10D5A0004B015C0149A147FFDAC22BA13CA14DA16F
:10D5B0005EA16BA97CA98DA99EA90E9420EE209155
:10D5C0006B0230916C0240916D0250916E020E948C
:10D5D0002CF00E9494F06D877E878F87988B86163B
:10D5E0009706A806B90614F44B015C018FAA98AE01
:10D5F000A9AEBAAE51E9851651E09506A104B10471
:10D6000044F481E991E0A0E0B0E08FAB98AFA9AF1E
:10D61000BAAF87E7AFA1B8A58A9FF0018B9FF00D45
:10D620001124E252FB4F2FA938AD49AD5AAD2083EA
:10D63000318342835383421653066406750671F0A4
:10D64000CA01B9010E94C1ED2B962CAD3DAD4EAD86
:10D650005FAD2B970E9420EE6B017C01A701960124
:10D6600060E074E284E79BE40E942CF04B015C01D3
:10D67000112309F485C26FA578A989A99AA90E94E6
:10D68000C1ED9B01AC01C701B6010E942CF00E94C4
:10D6900094F069837A838B839C8329893A894B89A7
:10D6A0005C89C501B4010E9420EE29A121712031BD
:10D6B00009F45AC227E74FA158A5249FF001259FDE
:10D6C000F00D1124EB57FB4F61A772A783A794A716
:10D6D000002309F470C26BA57CA58DA59EA50E94B0
:10D6E000C1ED9B01AC01C701B6010E942CF00E9464
:10D6F00094F06D837E838F8398872D893E894F892F
:10D70000588DC501B4010E9420EE29A12272203259
:10D7100009F445C227E70FA118A5209FF001219F1A
:10D72000F00D1124EB57FB4F65A776A787A790ABA9
:10D730002E961FAD2E9787E7112309F454C22FA10F
:10D7400038A5829F8001839F100D11240B571B4F1A
:10D75000D80151966D917D918D919C9154970E9425
:10D76000C1ED9B01AC01C701B6010E942CF00E94E3
:10D7700094F069877A878B879C87298D3A8D4B8DAA
:10D780005C8DC501B4010E9420EE29A124742034CF
:10D7900009F420C2F80161AB72AB83AB94AB19A161
:10D7A00087E717FF37C22FA138A5829F8001839F8B
:10D7B000100D11240B571B4FD80155966D917D917B
:10D7C0008D919C9158970E94C1ED9B01AC01C701BE
:10D7D000B6010E942CF00E9494F06D877E878F879F
:10D7E000988BA50194016BA97CA98DA99EA90E9483
:10D7F00020EE29A12878203809F403C2F80165AB8E
:10D8000076AB87AB90AFA50194016BAD7CAD8DADD0
:10D810009EAD0E9420EE6BA77FA78BA39BAB87E7F3
:10D820000FA118A5809FF001819FF00D1124EB57E7
:10D83000FB4FCB01ABA1BBA981AF92AFA3AFB4AFFC
:10D8400089A18878883809F0F3C18DE594E08E01CC
:10D850000F5F1F4F29961FAF0EAF29971C0110E0D5
:10D8600000E049EAA42E5FE5B52E63E6E62E78E5F2
:10D87000F72E39A1232F30E068963FAF2EAF68977F
:10D8800080E190E0002E02C0880F991F0A94E2F711
:10D8900068964EAD5FAD689784239523892B19F167
:10D8A0002996AEADBFAD29976D917D918D919C91DB
:10D8B0000E94C1ED2B013C01F101608171818281E7
:10D8C00093810E94BFED9B01AC01C301B2010E9494
:10D8D00020EE4B016C019501A7010E9476F118160C
:10D8E00014F0540176010F5F1F4F29962EAD3FAD06
:10D8F00029972C5F3F4F29963FAF2EAF299734E0F1
:10D90000230E311C0430110509F0BACF27968CADD7
:10D910009DADAEADBFAD2797B595A795979587956A
:10D9200027E74FA158A5249F8001259F100D1124A2
:10D930000B571B4FF80185A396A3A7A3B0A781A3FC
:10D9400092A3A3A3B4A3858F968FA78FB0A3818F33
:10D95000928FA38FB48F6801FDE3CF0ED11C2BA54E
:10D960003FA54BA15BA960E070E080E89FE30E94C7
:10D970002CF0D6016D937D938D939C9313976696AF
:10D98000EEADFFAD6697EC0FFD1F61817281838163
:10D9900094810E94C1ED9B01AC01B501C7010E94B9
:10D9A0002CF00E9499F0F801EB59FF4F60837183CE
:10D9B000828393836801B9E6CB0ED11C0E94BFED30
:10D9C00020E030E040E858E40E9420EE20E034E21D
:10D9D00044E75BE40E942CF00E9499F0F60160831A
:10D9E0007183828393832BAD3CAD4DAD5EADCA0197
:10D9F000B9010E9463EF9501A7010E9420EE2BA5BB
:10DA00003FA54BA15BA90E9420EE20E034E244E751
:10DA10005BE40E942CF06BAF7CAF8DAF9EAFF80142
:10DA2000EF5BFF4F608371838283938320E030E05C
:10DA300040E05FE36091270D7091280D8091290DE2
:10DA400090912A0D0E9420EE3B014C012E96FFADD5
:10DA50002E97FF2309F4EFC020E030E040E05FE3C1
:10DA60006091230D7091240D8091250D9091260DCC
:10DA70000E9420EE5B016C0189A1807309F41BC137
:10DA8000D801D1962D903D904D905C90D497E8941C
:10DA900057F8A2019101B501C6010E94BBED87FFB5
:10DAA00016C09501A6016BA57FA58BA19BA90E941D
:10DAB00020EEA20191010E942CF07B018C019B01C0
:10DAC000AC01B301C4010E94BBED87FFBAC0730172
:10DAD0008401B7C027E70FA118A5209FF001219F5F
:10DAE000F00D1124EB57FB4F458956896789708DDE
:10DAF000481759076A077B0714F482E083CB83E059
:10DB000081CB0E9422F25B018C01A70196010E9449
:10DB1000BBED87FF02C05601870187E74FA158A5DB
:10DB2000849FF001859FF00D11241CCCAB5ABF4F90
:10DB3000CD92DD92ED92FC9213971CCC19821A8241
:10DB40001B821C8253014201E0CC1D821E821F8277
:10DB5000188601CD19861A861B861C8623CD1D8644
:10DB60001E861F86188A42CD27E7AFA1B8A52A9F37
:10DB7000F0012B9FF00D1124EB57FB4F9058A4CDD3
:10DB800087E72FA138A5829FF001839FF00D112414
:10DB9000EB57FB4F11A612A613A614A699CD27E7A3
:10DBA0000FA118A5209FF001219FF00D1124EB5724
:10DBB000FB4F9058B9CD87E70FA118A5809FF001C2
:10DBC000819FF00D1124EB57FB4F15A616A617A643
:10DBD00010AAAECD9058D801D1966D937D938D93B8
:10DBE0009C93D497DCCD0FA118A5809FF001819F55
:10DBF000F00D1124EB57FB4F11AA12AA13AA14AA75
:10DC0000CECD9058D801D5966D937D938D939C93EE
:10DC1000D897F9CD0FA118A5809FF001819FF00D35
:10DC20001124EB57FB4F15AA16AA17AA10AEEBCD7D
:10DC30008DE494E00CCE7B018C01A12CB12CC12C85
:10DC4000D12CB9A1B7FF3CC0E0911E0DF0911F0D82
:10DC500020E030E040E05FE3638D748D858D968D2C
:10DC60000E9420EE6496EFAD6497EE2339F19B019C
:10DC7000AC016BA57FA58BA19BA90E9420EE27E795
:10DC80004FA158A5249FF001259FF00D1124EB57BB
:10DC9000FB4F25A936A947A950AD5F770E942CF00C
:10DCA0001B012C019701A8010E9476F1181644F07F
:10DCB0007101820105C075018601C3CF7B018C0112
:10DCC0002F965FAD2F97523008F0E2C09701A80160
:10DCD000B301C4010E94BBED87FD02C07301840142
:10DCE0009701A8016BA57FA58BA19BA90E9476F146
:10DCF000181624F0EBA4FFA40BA11BA987E7AFA182
:10DD0000B8A58A9F60018B9FD00C1124F601EB57B8
:10DD1000FB4F6F014F01F1E58F0E911CC701D80138
:10DD2000F40180839183A283B3835601FDE4AF0E97
:10DD3000B11CF50180839183A283B383F9E4CF0EF4
:10DD4000D11CF60180839183A283B3839701A8013C
:10DD500023966CAD7DAD8EAD9FAD23970E94BBED3C
:10DD600087FF17C023960CAD1DAD2EAD3FAD239799
:10DD7000D4010D931D932D933C931397F5010083CC
:10DD8000118322833383D6010D931D932D933C93EE
:10DD9000139787E7EFA1F8A58E9F80018F9F100D45
:10DDA00011240B571B4FF801E75BFF4F6081718116
:10DDB000828193819B01AC010E9420EE2BAD3CAD92
:10DDC0004DAD5EAD0E9463EF6B017C012BA53FA5BD
:10DDD0004BA15BA96BA57FA58BA19BA90E9420EEFF
:10DDE0009B01AC01C701B6010E9476F187FD07C017
:10DDF000D80111968C911197826011968C9387E7C8
:10DE0000EFA1F8A58E9F80018F9F100D11240E5059
:10DE10001B4F60E074E284EF90E02FA938AD49AD6C
:10DE20005AAD0E9427EFD8012D933C932D960EAD4D
:10DE30001FAD2D970B571B4F2D961FAF0EAF2D9774
:10DE40001FB71FA7F89490914A048091F50B982E64
:10DE50009817B9F199249394990E9F3008F0912C5A
:10DE600040E050E0BA0197E7891559F1999DF0011A
:10DE70001124EB57FB4F0581168127813085400F18
:10DE8000511F621F731F3EE03915A0F0939413C019
:10DE90002F968FAD2F97823009F022CF9501A601E2
:10DEA000B701C8010E9476F118160CF419CF75015C
:10DEB000860116CF912C483C2FEA52076105710567
:10DEC00098F297E709A5901669F0909FF001112448
:10DED000EB57FB4F208121FD83C501112CC01FE0B2
:10DEE00019A7F0CF98122BC087E72FA138A5829FE2
:10DEF0008001839F100D11240B571B4FD8011196E1
:10DF00008C911197806811968C93BFA5BFBFF801C3
:10DF10008081846080832D968EAD9FAD2D970E9469
:10DF2000A122D80111968C9111978F7711968C931D
:10DF30000FA50FBF2CC509A5015009A7C3CF17E72F
:10DF4000919EF0011124EB57FB4F908191FF08C087
:10DF500009A5902E93940F3008F0912C891521F289
:10DF6000092D10E01CA70BA717E7919EF0011124C3
:10DF7000EB57FB4F8181806881830FA50FBF109104
:10DF8000F50B19A3812F8150111101C08FE0C82E0C
:10DF9000D12C87E78C9DF0018D9DF00D1124EB575E
:10DFA000FB4F84800FA118A5809FF001819FF00D89
:10DFB0001124EB57FB4F3480882D807F21E080387F
:10DFC00009F020E091E0832D807F803809F090E017
:10DFD0002917D9F117E71C9DF0011D9DF00D1124A3
:10DFE000EB57FB4F9F012B5B3F4FCF01835B9F4F55
:10DFF000DC014D915D916D917C91D9014D935D93C3
:10E000006D937C9313978081826080832FA138A5C4
:10E01000129FF001139FF00D1124EB57FB4F8081ED
:10E02000846080832D968EAD9FAD2D970E94A12296
:10E030004BA55CA5149FF001159FF00D1124EB5723
:10E04000FB4F81818F77818373CF87E78C9DF001B0
:10E050008D9DF00D1124EB57FB4FB1AC02AD09A71C
:10E0600023ACA4AC0FA118A5809FF001819FF00DF7
:10E070001124EB57FB4FE1ACF2AC03AD14AD9701AB
:10E08000A8016B2D79A5822D9A2D0E9476F1181684
:10E0900024F4BE2CF9A6202EA12E87E72FA138A5A7
:10E0A000829F8001839F100D11240B571B4F8C9D65
:10E0B00090018D9D300D1124A9014B575B4F7A01C2
:10E0C000DA0199962D913D914D915C919C97F801C3
:10E0D00061A572A583A594A50E9462EF2B013C0166
:10E0E000D7019D962D913D914D915C91D097F8016E
:10E0F00065A576A587A590A90E9462EF6BA37CA376
:10E100008DA39EA3A3019201C301B2010E9420EE40
:10E110002B013C012BA13CA14DA15EA1CA01B9017B
:10E120000E9420EE9B01AC01C301B2010E9463EF8B
:10E130000E9422F26BA37CA38DA39EA34090270D87
:10E140005090280D6090290D70902A0DA301920126
:10E150000E9476F118160CF0A1C12BA13CA14DA193
:10E160005EA1C301B2010E942CF07B018C012B2D1A
:10E1700039A5422D5A2D0E9420EE9B01AC010E9430
:10E1800063EF9B01AC01C301B2010E9476F1181646
:10E1900094F42B2D39A5422D5A2D6B2D79A5822D66
:10E1A0009A2D0E9463EF9B01AC01C301B2010E9452
:10E1B0002CF07B018C01832886FE4BC087E72FA1C2
:10E1C00038A5829FF001839FF00D1124EB57FB4F80
:10E1D0008C9DD0018D9DB00D1124AB57BB4FD196B6
:10E1E0002D913D914D915C91D49761A972A983A91C
:10E1F00094A90E9462EF2B013C01E89477F880918A
:10E20000230D9091240DA091250DB091260D8BA387
:10E210009CA3ADA3BEA39C01AD01C301B2010E94AA
:10E2200076F11816B4F4A30192016BA17CA18DA123
:10E230009EA10E942CF0562E672E782E892E9701D3
:10E24000A8010E9476F1181624F0E52CF62C072D73
:10E25000182D87E7AFA1B8A58A9FF0018B9FF00D1D
:10E260001124EB57FB4F8C9DD0018D9DB00D1124D7
:10E27000AB57BB4FD5962D913D914D915C91D89761
:10E2800065A976A987A990AD0E9462EF2B013C0198
:10E29000E89477F8E0911E0DF0911F0D238D348DD9
:10E2A000458D568D2BA33CA34DA35EA3C301B201A4
:10E2B0000E9476F11816B4F4A30192016BA17CA11F
:10E2C0008DA19EA10E942CF0562E672E782E892EAD
:10E2D0009701A8010E9476F1181624F0E52CF62C7F
:10E2E000072D182D97E7892E8C9CC0018D9C900DD1
:10E2F0001124AC0146535B4F3A019701A8016B2DE5
:10E3000079A5822D9A2D0E9420EED3016D937D93E5
:10E310008D939C931397B9A1B89D800111240B573D
:10E320001B4FF801E35BFF4F4080B180C280D38078
:10E3300027E7522EE9A1E91509F41FC1EE2309F4DC
:10E34000B2C0E150E9A329A1222E312C259DC001A4
:10E350001124AC014B575B4F5AA749A7DA0111961C
:10E360008C911197806811968C93F801818181FFBF
:10E370009DC041ACB2ACC3ACD4AC529CC001539C68
:10E38000900D11249C012B573B4F7901F901EB5B58
:10E39000FF4F608071808280A380242D3B2DA601D9
:10E3A000B301882D9A2D0E94BBED18160CF495C070
:10E3B000F701E35BFF4F2081318142815381B3013B
:10E3C000882D9A2D0E94BBED882349F1D7018C91AD
:10E3D0008E7F8C93F701EF5AFF4FB080C180D280BF
:10E3E000F3802B2D3C2D4D2D5F2DB301882D9A2DC3
:10E3F0000E9476F1181624F4B62CC72CD82CFA2CCF
:10E40000529CF001539CF00D1124EE52FB4F8B2DCA
:10E410009C2DAD2DBF2D80839183A283B383780182
:10E42000B9E4EB0EF11CF701208131814281538167
:10E43000B301882D9A2D0E94BBED882309F1F801C4
:10E44000EF5AFF4F4080B180C280D380242D3B2DF6
:10E45000A601B301882D9A2D0E9476F1181624F496
:10E46000462CB72CC82CDA2C842D9B2DD601F70115
:10E4700080839183A283B383D8018C918E7F8C9308
:10E48000529CF001539CF00D1124EE52FB4F408042
:10E49000B180C280D38009A51AA54CCFE12CF12C04
:10E4A00000E81FE388CEFFE0F9A34DCF242D3B2DDC
:10E4B000A601642D7B2DC6010E9420EEF801EF5BC2
:10E4C000FF4F20813181428153810E9463EF0E947E
:10E4D00022F2462EB72E6C0150CFF801EF5AFF4FB3
:10E4E0008080A180E280F380282D3A2DA701642D41
:10E4F0007B2DC6010E9476F118161CF4842CAB2CDF
:10E500007601882D9A2DD701F801E75BFF4F8083B4
:10E510009183A283B383529CF001539CF00D11248C
:10E52000EA52FB4F8080A180E280F380282D3A2DB3
:10E53000A701642D7B2DC6010E94BBED87FF03C0A0
:10E54000482CBA2C6701529CF001539CF00D112409
:10E55000EB57FB4FDF01A35BBF4F442D5B2DB60193
:10E560004D935D936D937C93139780818E7F808311
:10E57000F80180818E7F80838ECF87E7F9A1F89F95
:10E58000800111240B571B4F2BA53CA5829FF00146
:10E59000839FF00D1124E253FB4FC080D180E280B5
:10E5A000F3803091F50B3FAF49A149A7C8018F5ABD
:10E5B0009F4F5C01D801A75BBF4FB8AFAFABBFADFA
:10E5C000E9A5BE1709F489C1EF3008F0D7C0EF5FA5
:10E5D000E9A739A5232F30E03CA32BA349A557E792
:10E5E000459FC0011124DC01AB57BB4FBCAFABAFA3
:10E5F000F801818181FFC4C0F1ADFBA7D801DA9693
:10E600004C90DA97DB965C90DB97DC966C90F5018A
:10E61000708081809280B3809801235B3F4F3CAB38
:10E620002BAB2BA5342D452D562DABA9BCA96D9137
:10E630007D918D919C910E94BBEDF801EB5BFF4FAA
:10E640001F0187FFB3C09601A701672D782D892D83
:10E650009B2D0E9476F1181604F5272D382D492D93
:10E660005B2D672D782D892D9B2D0E9420EEF801C2
:10E67000EF5BFF4F20813181428153810E9463EF24
:10E680000E9422F2ABA9BCA96D937D938D939C93BC
:10E690001397C72CD82CE92CFB2CC601D701EFA966
:10E6A000F8AD80839183A283B38347E72BA13CA17C
:10E6B000429FF001439FF00D1124EA52FB4F8080EE
:10E6C0009180A280B380D101CC901196DC901197FB
:10E6D0001296EC9012971396FC901801BDE42B0E45
:10E6E000311CF10140805180628073809201A3014E
:10E6F000B601C7010E9476F1181614F46201730185
:10E700009601A701B401C5010E9476F1181614F410
:10E710006401750147E72BA13CA1429FC001439FC3
:10E72000900D1124DC01AB57BB4F5D01FD01E75B90
:10E73000FF4FC601D70180839183A283B383F80181
:10E74000EB5BFF4F2081318142815381F101608178
:10E750007181828193810E94BBED811108C0D80133
:10E760008C9182608C93F501808184608083D801D4
:10E770008C918E7F8C930BAD1CAD18CF19A629CF31
:10E780009601A701B601C7010E9420EEF801EF5BD8
:10E79000FF4F20813181428153810E9463EF0E94AB
:10E7A00022F26BA7472E582E692E31CFF8018081B7
:10E7B0008E7F866080839601A701672D782D892D35
:10E7C0009B2D0E9476F11816ECF40F5B1F4F272D3E
:10E7D000382D492D5B2D672D782D892D9B2D0E947D
:10E7E00020EED8012D913D914D915C910E9463EFF7
:10E7F0000E9422F26BA7472E582E692EC72CD82CC8
:10E80000E92CFB2CC601D701EFA9F8AD80839183D9
:10E81000A283B3832BA5342D452D562D672D782D3E
:10E82000892D9B2D0E94BBED87FF03C07BA4420175
:10E83000B62C872D982DA92DBB2DEBA9FCA9808383
:10E840009183A283B38327E70BA11CA1209FF00132
:10E85000219FF00D1124EA52FB4F6080A1800281BC
:10E860001381D101CC901196DC9011971296EC9007
:10E8700012971396FC909601A701672D782D892D8C
:10E880009B2D0E94BBED87FF04C0C72CD82CE92C20
:10E89000FB2C9601A701662D7A2DC8010E9476F106
:10E8A00018161CF4C62CDA2C780127E70BA11CA142
:10E8B000209FF001219FF00D1124EB57FB4FDF014A
:10E8C000A75BBF4FA601B7014D935D936D937C93FA
:10E8D00013978081846080834ECFDC019C901196D9
:10E8E0000C91119712961C9112971396BC90292D9A
:10E8F000302F412F5B2DB601C7010E9476F118160B
:10E9000024F49C2C0D2D1E2DBF2C892D902FA12F72
:10E91000BB2DEFA9F8AD80839183A283B38387E7F2
:10E92000F82EF9A1FF9D800111240B571B4FC80140
:10E930000E94A122D80111968C9111978F77119680
:10E940008C9309A10F3008F047C00F5F09A319A1EC
:10E95000F19EF0011124EB57FB4F81818068818388
:10E960000FAD1013DECF2D968EAD9FAD2D970E946B
:10E97000A1220FA118A5F09EF001F19EF00D112427
:10E98000EB57FB4F81818F7781831FA51FBF639654
:10E990001FAD6397112331F086E490E090934C040F
:10E9A00080934B048091F50B8F30C0F48F5F809380
:10E9B000F50B8091AA0C9091AB0C80619093AB0CFD
:10E9C0008093AA0C9FB7F8948091FD0C8F5F809381
:10E9D000FD0C9FBF0C94A96819A2B9CF80E0E7CFC6
:10E9E00009A58013B5CA80CA4F925F926F927F9239
:10E9F000AF92BF92CF92DF92EF92FF920F931F934D
:10EA0000CF93DF9300D000D01F921F92CDB7DEB717
:10EA10002B013C0129833A834B835C83ED82FE8288
:10EA20000F83188720EF33E244E759E40E94BBEDDF
:10EA3000811140C14090C00C5090C10C6090C20C3C
:10EA40007090C30C20EF33E244E759E469817A8186
:10EA50008B819C810E94BBED811135C18091C40CDA
:10EA60009091C50CA091C60CB091C70C89839A8374
:10EA7000AB83BC8320EF33E244E759E46D817E81B0
:10EA80008F8198850E94BBED81112AC18091C80CAD
:10EA90009091C90CA091CA0CB091CB0C8D839E8330
:10EAA000AF83B88720912E0C30912F0C4091300C01
:10EAB0005091310C69817A818B819C810E9463EF36
:10EAC00069837A838B839C832091320C3091330C41
:10EAD0004091340C5091350C6D817E818F819885E9
:10EAE0000E9463EF20912404309125044091260474
:10EAF000509127040E9463EF6D837E838F839887F4
:10EB000020912A0C30912B0C40912C0C50912D0C03
:10EB1000C301B2010E9463EF2091390230913A02A1
:10EB200040913B0250913C020E9420EE20E030E0F8
:10EB300040E05FE30E9463EF0E94C5F00E9494F002
:10EB400060937104709372048093730490937404BF
:10EB500020913D0230913E0240913F02509140028F
:10EB600069817A818B819C810E9420EE20E030E0D7
:10EB700040E05FE30E9463EF0E94C5F00E9494F0C2
:10EB8000609375047093760480937704909378046F
:10EB9000209141023091420240914302509144023F
:10EBA0006D817E818F8198850E9420EE20E030E08B
:10EBB00040E05FE30E9463EF0E94C5F00E9494F082
:10EBC0006093790470937A0480937B0490937C041F
:10EBD00020EF33E244E759E4C601B5010E94BBEDE2
:10EBE000882309F48AC08091330383FD86C0E090B6
:10EBF0001E0DF0901F0D20E030E046E153E4D701F8
:10EC00009F966D917D918D919C91D2970E9476F106
:10EC1000181644F080911B0E87FD04C0F70182A5F1
:10EC200081116BC02091450230914602409147020C
:10EC300050914802C601B5010E9420EE0E9494F056
:10EC400060937D0470937E0480937F04909380048E
:10EC500020EF33E244E759E46A8D7B8D8C8D9D8DE6
:10EC60000E94BBED882361F08A8D9B8DAC8DBD8D9C
:10EC70008093530C9093540CA093550CB093560C66
:10EC80006E8D81E00E944C6681E028960FB6F89464
:10EC9000DEBF0FBECDBFDF91CF911F910F91FF90CF
:10ECA000EF90DF90CF90BF90AF907F906F905F908C
:10ECB0004F9008954092C00C5092C10C6092C20CCB
:10ECC0007092C30CBFCE89819A81AB81BC81809345
:10ECD000C40C9093C50CA093C60CB093C70CCACEBD
:10ECE0008D819E81AF81B8858093C80C9093C90CAB
:10ECF000A093CA0CB093CB0CD5CE8091BC0C909154
:10ED0000BD0CA091BE0CB091BF0C80937D0490937C
:10ED10007E04A0937F04B09380049ACF4F925F92B9
:10ED20006F927F928F929F92AF92BF92CF92DF921B
:10ED3000EF92FF920F931F93CF93DF93C0915F02E7
:10ED4000D0916002109161020091620284E294E02D
:10ED50000E941D512B013C0180E294E00E941D5154
:10ED600021E02F930F931F93DF93CF9320EFA22ED9
:10ED700023E2B22E24E7C22E29E4D22E86017501A9
:10ED8000A301920131DED0906702C0906802B0907A
:10ED90006902A0906A024090C80C5090C90C609023
:10EDA000CA0C7090CB0C88E294E00E941D519B012C
:10EDB000AC01C301B2010E9463EF7B018C01209181
:10EDC0001E0C30911F0C4091200C5091210C609131
:10EDD000120C7091130C8091140C9091150C0E94E0
:10EDE00063EF4B01D82FC92F0F900F900F900F900A
:10EDF0000F909B01482F592FB701C8010E9476F14F
:10EE000018161CF04701D02FC12F81E08F93AF92CD
:10EE1000BF92CF92DF9280EFA82E83E2B82E84E7D4
:10EE2000C82E89E4D82E74010D2F1C2FA601950140
:10EE3000C601B501D9DD0F900F900F900F900F9084
:10EE4000DF91CF911F910F91FF90EF90DF90CF90C6
:10EE5000BF90AF909F908F907F906F905F904F90FA
:10EE600008954F925F926F927F928F929F92AF928E
:10EE7000BF92CF92DF92EF92FF920F931F93CF93A7
:10EE8000DF93D82F862E742EC22F6E2C5F2C402E2F
:10EE9000912E20E030E0A90160910E0270910F02E6
:10EEA00080911002909111020E94BBED87FDA2C0DB
:10EEB000D1111CC081101AC0711018C0C11121C01D
:10EEC00090EFA92E93E2B92E94E7C92E99E4D92E9A
:10EED000C1E024C010EFE12E13E2F12E04E719E4A3
:10EEE0002FC020EF33E244E759E43FC080EFA82E63
:10EEF00083E2B82E84E7C82E89E4D82ECC2359F0BB
:10EF0000C0E0A0901E02B0901F02C0902002D090DE
:10EF10002102C11103C07720E9F2C0E0E0900A02AB
:10EF2000F0900B0200910C0210910D02E092490C3E
:10EF3000F0924A0C00934B0C10934C0CC11103C07F
:10EF4000882079F2C0E020910602309107024091BA
:10EF50000802509109022093450C3093460C4093CF
:10EF6000470C5093480CC11106C060EF73E284E770
:10EF700099E4DD2381F06091020270910302809197
:10EF80000402909105026093410C7093420C8093AF
:10EF9000430C9093440CE1E0EF939F924F925F9269
:10EFA0006F9222DD80910E0290910F02A0911002CB
:10EFB000B09111028093530C9093540CA093550C74
:10EFC000B093560C0F900F900F900F900F9080E021
:10EFD000DF91CF911F910F91FF90EF90DF90CF9035
:10EFE000BF90AF909F908F907F906F905F904F9069
:10EFF0000C94B624DF91CF911F910F91FF90EF9069
:10F00000DF90CF90BF90AF909F908F907F906F9048
:10F010005F904F900895CF92DF92EF92FF9281E040
:10F020000E94DC600E943E292091FD0C211109C044
:10F030002091AA0C3091AB0C267033272630310575
:10F0400069F560934F0C7093500C8093510C909322
:10F05000520C9091090180919D1090FF60C0811128
:10F0600005C080919C10843609F099C08AE79EE221
:10F070000E94044B61E08BEE93E00E94D8D40E9482
:10F0800028CF8DEB90E00E94983260E00E94A6C8E5
:10F09000FF90EF90DF90CF900C9444CAC0904F0C3B
:10F0A000D090500CE090510CF090520C9B01AC01B0
:10F0B0002C193D094E095F0969017A018091190DEA
:10F0C00090911A0DA0911B0DB0911C0D0097A105F8
:10F0D000B105F9F08C159D05AE05BF05D0F480E0B3
:10F0E0000E94846080914F0290915002A091510241
:10F0F000B09152020097A105B10509F4AACF8C1571
:10F100009D05AE05BF0508F0A4CF81E00E94846094
:10F11000A0CF80911B0E877F80931B0EE3CF8111C0
:10F120003EC080919C108436D1F18EEB90E00E941D
:10F13000983260E00E94A6C80E9444CA10929C10B7
:10F1400010929D108091090180FF0E9473D48091DC
:10F150009C10843621F089E69EE20E94044B809147
:10F160009D108823E1F0E0912D0DF0E0EE0FFF1FE0
:10F17000E55DF24F0188F289E02DE491EF77E5300B
:10F1800071F080911B0E826080931B0E61E085EF11
:10F1900093E2FF90EF90DF90CF900C94D8D4FF9043
:10F1A000EF90DF90CF9008951F93CF93DF93EC0102
:10F1B00020E030E040EF51E46A857B858C859D85B9
:10F1C0000E94BBED87FD2CC08091330383FD28C0D6
:10F1D0008091CC0C182F107180618093CC0C81E051
:10F1E0000E94DC6083E090E00E94284B2E813F81EA
:10F1F000488559856A857B858C859D850E9462EF4F
:10F200009F7720E030E040E85FE30E94BBED1816F6
:10F2100034F38091CC0C112339F080618093CC0CB5
:10F22000DF91CF911F9108958F7EF8CF8091FD0CD3
:10F23000882341F080E00E94DC6081E090E00E9441
:10F24000284BF4CF08952F923F924F925F926F9286
:10F250007F928F929F92AF92BF92CF92DF92EF9266
:10F26000FF920F931F93CF93DF9300D000D01F9294
:10F270001F92CDB7DEB729013A01E982FA820B83EA
:10F280001C832E8C3F8C88A099A02091200D10917A
:10F290001B0E1072022F007426FD18C0111116C02B
:10F2A0002091CC0C20FD03C060E070E0CB0121FD7B
:10F2B00003C0412C512C320122FD08C020911D0DAC
:10F2C00026FD04C019821A821B821C820E94C1ED95
:10F2D0002091E70C3091E80C4091E90C5091EA0C38
:10F2E0000E9420EE2091410C3091420C4091430C41
:10F2F0005091440C0E9463EF6D837E838F839887C7
:10F300006093410C7093420C8093430C9093440C97
:10F31000C301B2010E94C1ED2091EB0C3091EC0CC5
:10F320004091ED0C5091EE0C0E9420EE2091450C86
:10F330003091460C4091470C5091480C0E9463EF6D
:10F340002B013C014092450C5092460C6092470CB8
:10F350007092480C69817A818B819C810E94C1EDF9
:10F360002091EF0C3091F00C4091F10C5091F20C87
:10F370000E9420EE2091490C30914A0C40914B0C98
:10F3800050914C0C0E9463EF6093490C70934A0CAF
:10F3900080934B0C90934C0C112309F471C0809115
:10F3A000330383FD1BC000911E0D10911F0D20E043
:10F3B00030E046E153E4D8019F966D917D918D91A7
:10F3C0009C91D2970E94BBED87FF0BC080911B0ED2
:10F3D00087FD07C0F80182A5882319F0A12CB12C64
:10F3E00065016091BC0C7091BD0C8091BE0C909138
:10F3F000BF0C6A0D7B1D8C1D9D1D0E94C1ED2091CF
:10F40000F30C3091F40C4091F50C5091F60C0E94E5
:10F4100020EE5B016C01E090490CF0904A0C0091E9
:10F420004B0C10914C0C2091450C3091460C4091A6
:10F43000470C5091480C6091410C7091420C8091A6
:10F44000430C9091440CEBA1EF939F928F923F92CB
:10F450002F92CADA80E00E94B6240F900F900F908E
:10F460000F900F908AA18111E1DE0E943E296093E6
:10F470004F0C7093500C8093510C9093520C0EC013
:10F4800001118DCF7B018C01A30192016D817E81E1
:10F490008F8198850E943745811181CF28960FB6BC
:10F4A000F894DEBF0FBECDBFDF91CF911F910F91BA
:10F4B000FF90EF90DF90CF90BF90AF909F908F9094
:10F4C0007F906F905F904F903F902F9008954F9254
:10F4D0005F926F927F92AF92BF92CF92DF92EF9244
:10F4E000FF920F931F93CF93DF93CDB7DEB72C9787
:10F4F0000FB6F894DEBF0FBECDBF69837A838B83CE
:10F500009C8329013A01ED82FE820F831887809146
:10F51000330383FD1BC000911E0D10911F0D20E0D1
:10F5200030E046E153E4D8019F966D917D918D9135
:10F530009C91D2970E94BBED87FF0BC080911B0E60
:10F5400087FD07C0F80182A5882319F0A12CB12CF2
:10F5500065018091200D86FD1BC080911B0E85FDED
:10F5600017C08091CC0C80FD04C019821A821B82C6
:10F570001C8281FD03C0412C512C320182FD08C048
:10F5800080911D0D86FD04C01D821E821F8218867B
:10F590002091530C3091540C4091550C5091560CC5
:10F5A00029873A874B875C878091B00C9091B10C8A
:10F5B000A091B20CB091B30C29813A814B815C814E
:10F5C000820F931FA41FB51F809371049093720440
:10F5D000A0937304B09374048091B40C9091B50C13
:10F5E000A091B60CB091B70C840D951DA61DB71D4A
:10F5F0008093750490937604A0937704B093780475
:10F600008091B80C9091B90CA091BA0CB091BB0C40
:10F610002D813E814F815885820F931FA41FB51FF6
:10F620008093790490937A04A0937B04B0937C0434
:10F630008091BC0C9091BD0CA091BE0CB091BF0C00
:10F640008A0D9B1DAC1DBD1D80937D0490937E048F
:10F65000A0937F04B09380048E8D9F8DA8A1B9A143
:10F660008093530C9093540CA093550CB093560C6C
:10F670006CA18BA10E944C6689859A85AB85BC855F
:10F680008093530C9093540CA093550CB093560C4C
:10F6900080E00E94B6248AA18111C8DD0E943E2923
:10F6A00060934F0C7093500C8093510C9093520CBC
:10F6B0002C960FB6F894DEBF0FBECDBFDF91CF9171
:10F6C0001F910F91FF90EF90DF90CF90BF90AF9080
:10F6D0007F906F905F904F900895AF92BF92CF92BE
:10F6E000DF92EF92FF920F931F9390933D048093CC
:10F6F0003C040E94654B20911E0C30911F0C4091E0
:10F70000200C5091210C6091120C7091130C80917F
:10F71000140C9091150C0E9463EF20E030E040E75C
:10F7200051E40E9462EF9B01AC016091C80C7091A2
:10F73000C90C8091CA0C9091CB0C0E94BBED87FF45
:10F7400034C020E030E040E251E460914102709129
:10F75000420280914302909144020E9420EE0E9456
:10F7600094F07B018C0181E08F938F938F93809134
:10F770005E028F9380915D028F9380915C028F93E4
:10F7800080915B028F93A12CB12C650120E030E0C9
:10F79000A90160E070E0CB019ADE8DB79EB70796B5
:10F7A0000FB6F8949EBF0FBE8DBF40DD80E00E9473
:10F7B00084601F910F91FF90EF90DF90CF90BF90EA
:10F7C000AF900C947F4B2F923F924F925F926F922B
:10F7D0007F928F929F92AF92BF92CF92DF92EF92E1
:10F7E000FF920F931F93CF93DF93CDB7DEB72D9783
:10F7F0000FB6F894DEBF0FBECDBF982E6D87842E56
:10F8000080911B0E282F2072222E806280931B0E67
:10F810008091C00C9091C10CA091C20CB091C30C0E
:10F820008D839E83AF83B8872091C40C3091C50C23
:10F830004091C60C5091C70C29873A874B875C874B
:10F840004090C80C5090C90C6090CA0C7090CB0CC2
:10F85000882009F466C110922404109225041092A5
:10F860002604109227041092DD0C1092DE0C1092E8
:10F87000DF0C1092E00C86E190E00E94983260E08C
:10F880000E94A6C80E9444CAE0902004F09021047F
:10F89000009122041091230480911C0490911D0476
:10F8A000A0911E04B0911F04E81AF90A0A0B1B0B61
:10F8B00088279927DC018E199F09A00BB10B809333
:10F8C000B80C9093B90CA093BA0CB093BB0C809178
:10F8D000200D80648093200DEE0CFF1C001F111F73
:10F8E00031E03F933F933F9380915E028F938091ED
:10F8F0005D028F9380915C028F9380915B028F9366
:10F90000A12CB12C650120E030E0A90160E070E09D
:10F91000CB01DDDD8091200490912104A09122048F
:10F92000B09123048093B80C9093B90CA093BA0CB7
:10F93000B093BB0C609141027091420280914302EE
:10F94000909144029B01AC010E9463EF0E9494F0ED
:10F9500069837A838B839C8341E04F931F924F93FB
:10F9600020E030E040E450E460915B0270915C0282
:10F9700080915D0290915E020E942CF09F938F9384
:10F980007F936F93E980FA800B811C8120E030E047
:10F99000A90160E070E0CB019ADD609141027091B5
:10F9A000420280914302909144029B01AC010E946B
:10F9B00063EF9B01AC010E9463EF90580E9494F0AA
:10F9C00069837A838B839C8351E05F935F935F931A
:10F9D00020E030E040E450E460915B0270915C0212
:10F9E00080915D0290915E020E942CF09F938F9314
:10F9F0007F936F93E980FA800B811C8120E030E0D7
:10FA0000A90160E070E0CB0162DD8091200D8F7B69
:10FA10008093200D2091BF103091C0104091C110F3
:10FA20005091C21060914102709142028091430254
:10FA3000909144020E9420EE20E030E0A9010E9453
:10FA400063EF0E9494F0A1E0AF931F92AF932091D7
:10FA50005E022F9320915D022F9320915C022F93E1
:10FA600020915B022F937B018C0120E030E0A90103
:10FA700060E070E0CB012BDD6091200470912104E7
:10FA800080912204909123040E94C1ED0E9494F081
:10FA90006093B80C7093B90C8093BA0C9093BB0C24
:10FAA000E0911E0DF0911F0D81859285A385B4858F
:10FAB0009C01AD0166277727CB01621B730B840B7A
:10FAC000950B0E94C1ED2091EF0C3091F00C40910C
:10FAD000F10C5091F20C0E9420EE6093320C709366
:10FAE000330C8093340C9093350C81E00E94B62443
:10FAF0008091CC0C982F94609093CC0C982F93709D
:10FB00000FB6F894DEBF0FBECDBF80911B0E9330B1
:10FB100009F0ABC1816080931B0E1092F80C10921B
:10FB2000F70C992009F4ADC180911B0E582F50722B
:10FB3000352E806280931B0E84E190E00E94983203
:10FB400060E00E94A6C80E9444CA70DB8091200D2C
:10FB500080648093200D1092D50C1092D60C1092D8
:10FB6000D70C1092D80C60912C0470912D048091C8
:10FB70002E0490912F0400912804109129042091C3
:10FB80002A0430912B04601B710B820B930B00270E
:10FB900011279801061B170B280B390B0093B00C8B
:10FBA0001093B10C2093B20C3093B30C660F771FF7
:10FBB000881F991FA1E0AF93AF93AF932091560296
:10FBC0002F93209155022F93209154022F9320912F
:10FBD00053022F93A12CB12C6501E12CF12C87014C
:10FBE00020E030E0A90173DC80912C0490912D0479
:10FBF000A0912E04B0912F048093B00C9093B10C7F
:10FC0000A093B20CB093B30C20E030E040EA50E493
:10FC10006091390270913A0280913B0290913C02CE
:10FC20000E9420EE0E9494F069837A838B839C83E8
:10FC3000B1E0BF931F92BF9320E030E040E450E476
:10FC40006091530270915402809155029091560236
:10FC50000E942CF09F938F937F936F9320E030E06E
:10FC6000A90169817A818B819C8131DC60913902A3
:10FC700070913A0280913B0290913C029B01AC0151
:10FC80000E9463EF20E030E040EA50E40E9420EE62
:10FC900090580E9494F069837A838B839C8321E03F
:10FCA0002F932F932F9320E030E040E450E46091B5
:10FCB00053027091540280915502909156020E9415
:10FCC0002CF09F938F937F936F9320E030E0A901F6
:10FCD00069817A818B819C81FADB60913902709114
:10FCE0003A0280913B0290913C020E9494F031E0F4
:10FCF0003F933F933F93209156022F9320915502BB
:10FD00002F93209154022F93209153022F9320E0A0
:10FD100030E0A901DCDB80912C0490912D04A091AE
:10FD20002E04B0912F048093B00C9093B10CA0934B
:10FD3000B20CB093B30C8091CC0C982F916090933F
:10FD4000CC0C982F96700FB6F894DEBF0FBECDBFC7
:10FD500080911B0E963009F08AC08160332009F42F
:10FD600088C0806280931B0E8091200D8F7B8093D2
:10FD7000200D5D85511189C080911A0C90911B0C4A
:10FD8000A0911C0CB0911D0C8D839E83AF83B8870E
:10FD90009D85911196C1882041F04090120C5090A1
:10FDA000130C6090140C7090150C81E00E94B62426
:10FDB00081E08F93809156028F93809155028F93AB
:10FDC000809154028F93809153028F9380EFA82EDD
:10FDD00083E2B82E84E7C82E89E4D82E830172010D
:10FDE00029853A854B855C856D817E818F819885DB
:10FDF0000E94F47481E00E94B6249091CC0C292FCB
:10FE000023700F900F900F900F900F9080911B0E0A
:10FE1000233099F592FF31C0816080931B0E1092C0
:10FE2000A00D0E94754480911B0E222041F180623A
:10FE300080931B0E80E02D960FB6F894DEBF0FBEA8
:10FE4000CDBFDF91CF911F910F91FF90EF90DF9089
:10FE5000CF90BF90AF909F908F907F906F905F906A
:10FE60004F903F902F900C94B6248E7F54CE8E7F6F
:10FE700075CF8F7D77CF8E7F20C18E7FCECF8F7D48
:10FE8000D7CF3D85332309F486CF1092D90C109239
:10FE9000DA0C1092DB0C1092DC0C85E190E00E94F1
:10FEA000983260E00E94A6C80E9444CA209134049F
:10FEB00030913504409136045091370480913004DC
:10FEC00090913104A0913204B0913304281B390B76
:10FED0004A0B5B0B88279927DC01821B930BA40B31
:10FEE000B50B8093B40C9093B50CA093B60CB09363
:10FEF000B70C8091200D80648093200D220F331F5A
:10FF0000441F551FA1E0AF93AF93AF9380915A0266
:10FF10008F93809159028F93809158028F93809193
:10FF200057028F93A12CB12C6501E12CF12C870194
:10FF300060E070E0CB01CBDA80913404909135041D
:10FF4000A0913604B09137048093B40C9093B50C13
:10FF5000A093B60CB093B70C20E030E040EA50E438
:10FF600060913D0270913E0280913F02909140026B
:10FF70000E9420EE0E9494F069837A838B839C8395
:10FF8000B1E0BF931F92BF9320E030E040E450E423
:10FF900060915702709158028091590290915A02D3
:10FFA0000E942CF09F938F937F936F9329813A81C6
:10FFB0004B815C8160E070E0CB0189DA60913D02A9
:10FFC00070913E0280913F02909140029B01AC01F2
:10FFD0000E9463EF20E030E040EA50E40E9420EE0F
:10FFE00090580E9494F069837A838B839C8321E0EC
:10FFF0002F932F932F9320E030E040E450E4609162
:020000021000EC
:100000005702709158028091590290915A020E94B1
:100010002CF09F938F937F936F9329813A814B812B
:100020005C8160E070E0CB0152DA8091200D8F7B23
:100030008093200D60913D0270913E0280913F02BD
:10004000909140020E9494F09B01AC0181E08F935B
:100050001F928F9380915A028F93809159028F93B0
:10006000809158028F93809157028F9360E070E0E7
:10007000CB012DDA8091340490913504A09136049F
:10008000B09137048093B40C9093B50CA093B60C48
:10009000B093B70C8091CC0C982F92609093CC0CBD
:1000A000982F95700FB6F894DEBF0FBECDBF80912C
:1000B0001B0E953009F0DFCE816080931B0E9110EE
:1000C0005BCE2091160C3091170C4091180C50917A
:1000D000190C29873A874B875C875DCEA7D880E0CB
:1000E0000E94B624E0ECFCE080819181A281B38182
:1000F0008093020290930302A0930402B09305023E
:1001000084819581A681B78180930602909307022E
:10011000A0930802B093090280859185A285B385DA
:1001200080930A0290930B02A0930C02B0930D02ED
:100130006091BC0C7091BD0C8091BE0C9091BF0C75
:100140000E94C1ED2091F30C3091F40C4091F50C1C
:100150005091F60C0E9420EE60931E0270931F02D5
:1001600080932002909321028091530C9091540C23
:10017000A091550CB091560C80930E0290930F02F3
:10018000A0931002B093110208954F925F926F9264
:100190007F92AF92BF92CF92DF92EF92FF920F9336
:1001A0001F93CF93DF93CDB7DEB72D970FB6F8949B
:1001B000DEBF0FBECDBF2091C00C3091C10C40916D
:1001C000C20C5091C30C2D833E834F8358874090BF
:1001D000C40C5090C50C6090C60C7090C70C8091F8
:1001E000C80C9091C90CA091CA0CB091CB0C898716
:1001F0009A87AB87BC871AD800911E0D10911F0DEE
:1002000070E060E08CED9AE20E94FA492091530C74
:100210003091540C4091550C5091560C29833A83DF
:100220004B835C838091BC0C9091BD0CA091BE0C63
:10023000B091BF0CF801878F90A3A1A3B2A3F09156
:100240001B0EFD87F0FF61C08091C0029091C1023A
:10025000A091C202B091C302F80141855285638525
:10026000748584179507A607B7070CF04EC09C014C
:10027000AD0166277727CB01621B730B840B950BAF
:100280000E94C1ED2091EF0C3091F00C4091F10CE7
:100290005091F20C0E9420EE6093320C7093330C5C
:1002A0008093340C9093350C3D85306230931B0E57
:1002B00081E08F9380915E028F9380915D028F9396
:1002C00080915C028F9380915B028F9390EFA92EB7
:1002D00093E2B92E94E7C92E99E4D92E86017501CF
:1002E000A6019501C601B5010E94F47480911B0E10
:1002F0008F7D80931B0E0E94167981E00E94B624A8
:100300000F900F900F900F900F9087EB92E09093CB
:100310001F0D80931E0D8091BC0C9091BD0CA0917F
:10032000BE0CB091BF0C80937D0490937E04A0938B
:100330007F04B0938004C090C402D090C502E090C6
:10034000C602F090C702C0924502D0924602E092E7
:100350004702F0924802A701960160E070E080E851
:100360009FE30E942CF06093F30C7093F40C809345
:10037000F50C9093F60C8091CA029091CB02A0915B
:10038000CC02B091CD0280936B0290936C02A0934B
:100390006D02B0936E022091CE023091CF02409157
:1003A000D0025091D10220934003309341034093F7
:1003B00042035093430320935003309351034093DF
:1003C000520350935303C701B6010E9420EE0E94CE
:1003D00099F06093690470936A0480936B0490931E
:1003E0006C046093590470935A0480935B04909357
:1003F0005C0480EE92E00E94B9388091B80290913E
:10040000B902A091BA02B091BB029C01AD0166276E
:100410007727CB01621B730B840B950B0E94C1EDF8
:100420002091E70C3091E80C4091E90C5091EA0CD6
:100430000E9420EE60932A0C70932B0C80932C0C5E
:1004400090932D0C8091BC029091BD02A091BE02B0
:10045000B091BF029C01AD0166277727CB01621BDB
:10046000730B840B950B0E94C1ED2091EB0C309126
:10047000EC0C4091ED0C5091EE0C0E9420EE60933C
:100480002E0C70932F0C8093300C9093310C809134
:10049000C0029091C102A091C202B091C3029C011E
:1004A000AD0166277727CB01621B730B840B950B7D
:1004B0000E94C1ED2091EF0C3091F00C4091F10CB5
:1004C0005091F20C0E9420EE6093320C7093330C2A
:1004D0008093340C9093350C8091FB0C9091FC0C24
:1004E0000E94434A80911B0E80FF21C081E08F93C0
:1004F00082E48F9388EC8F931F921F9280EFA82E37
:1005000083E2B82E84E7C82E89E4D82EE984FA84E1
:100510000B851C85A30192016D817E818F81988559
:100520000E94F4740F900F900F900F900F9089819C
:100530009A81AB81BC818093530C9093540CA0930F
:10054000550CB093560C81E02D960FB6F894DEBF93
:100550000FBECDBFDF91CF911F910F91FF90EF9014
:10056000DF90CF90BF90AF907F906F905F904F9053
:100570000C94B624CF92DF92EF92FF920F931F93C9
:100580000E9435510E940039182F88E690E00E94A1
:10059000E7EE811729F0612F88E690E00E9402EFD4
:1005A00080E092ECA1E0B0E08093490290934A028F
:1005B000A0934B02B0934C021092190D10921A0D99
:1005C00010921B0D10921C0D80E49EE7A5E0B0E098
:1005D00080934F0290935002A0935102B093520225
:1005E00080E090E0A8ECB2E48093390290933A0264
:1005F000A0933B02B0933C0280933D0290933E0255
:10060000A0933F02B093400240E050E06AEF75E4EF
:10061000409341025093420260934302709344021C
:1006200040E050E060E87FE340934502509346028B
:10063000609347027093480240E050E068E473E43E
:1006400040935F0250936002609361027093620274
:100650004093630250936402609365027093660254
:1006600040E050E060EA70E4409367025093680213
:100670006093690270936A028093530290935402CC
:10068000A0935502B093560280935702909358025C
:10069000A0935902B0935A0280E090E0A0E4B0E445
:1006A00080935B0290935C02A0935D02B0935E0224
:1006B00000E010E020EA31E40093270D1093280DAC
:1006C0002093290D30932A0D8AE999E9A9E9BEE31F
:1006D0008093230D9093240DA093250DB093260DA8
:1006E00080E090E0AAE7B4E480934403909345034C
:1006F000A0934603B0934703809348039093490324
:10070000A0934A03B0934B0340E050E068E472E4E6
:1007100040934C0350934D0360934E0370934F03EB
:100720008093340390933503A0933603B09337033B
:100730008093380390933903A0933A03B0933B031B
:1007400040933C0350933D0360933E0370933F03FB
:100750001092720287E390E09093B6028093B50204
:100760008FEF80938D0290E590938E02C12CD12C57
:1007700094E4E92E93E4F92EC0928F02D092900275
:10078000E0929102F0929202C12CD12CE4E0EE2E84
:10079000E2E4FE2EC0929302D0929402E09295027F
:1007A000F0929602C12CD12CF1E9EF2EF3E4FF2E4A
:1007B000C0929702D0929802E0929902F0929A0227
:1007C00080939B02C12CD12CA7E5EA2EA3E4FA2E3C
:1007D000C092260CD092270CE092280CF092290CA3
:1007E000C12CD12CBFE2EB2EB3E4FB2EC092220C25
:1007F000D092230CE092240CF092250CC12CD12C29
:100800009CE0E92E93E4F92EC0921E0CD0921F0CAE
:10081000E092200CF092210C10921A0C10921B0CFA
:1008200010921C0C10921D0C1092160C1092170CAA
:100830001092180C1092190C1092120C1092130CAA
:100840001092140C1092150CE0E6CE2EE5EEDE2E82
:10085000EAEBEE2EE2E4FE2EC092C402D092C50274
:10086000E092C602F092C7024093CA025093CB02B4
:100870006093CC027093CD020093D2021093D30206
:100880002093D4023093D50240E050E46CE975E443
:100890004093CE025093CF026093D0027093D10266
:1008A00093E09093E30222ED30E03093270320930E
:1008B000260396EE9093FE0298E29093FF0240E0AA
:1008C00050E060EE70E440930003509301036093A6
:1008D00002037093030340E050E060E070E4409353
:1008E000040350930503609306037093070340E0ED
:1008F00050E060E272E44093080350930903609370
:100900000A0370930B0380930C031092BC021092A5
:10091000BD021092BE021092BF021092B802109255
:10092000B9021092BA021092BB0221E030E030937B
:10093000DB022093DA0226E930E03093DD022093D7
:10094000DC021092DF021092DE0280932C030E94E0
:1009500035510E94C140E0911E0DF0911F0D808124
:1009600014DC8FE692E00E94B93882E39AE21F918C
:100970000F91FF90EF90DF90CF900C9453508F9297
:100980009F92AF92BF92CF92DF92EF92FF926C0153
:10099000F12CE12C0E94F6DF4B015C01C114D10463
:1009A000E104F104B9F00E94F6DF681979098A09B7
:1009B0009B09683E73408105910580F321E0C21ACE
:1009C000D108E108F10888EE880E83E0981EA11C8A
:1009D000B11CE4CFFF90EF90DF90CF90BF90AF902D
:1009E0009F908F9008950F931F93CF93DF93EC0107
:1009F0008B01BC018BEA9AE20E946E3A80E20E946F
:100A00003124CE010E94E7EE90E00E949A3980E204
:100A10000E943124CE010E94763AC8010E94044B04
:100A200084E090E0DF91CF911F910F91A8CF0F93B9
:100A30001F93CF93DF93EC018B01BC0184EA9AE210
:100A40000E946E3A80E20E943124CE010E94F4EEB0
:100A50000E949A3980E20E943124CE010E94763AA7
:100A6000C8010E94044B84E090E0DF91CF911F9178
:100A70000F9185CF0F931F93CF93DF93EC018B01E1
:100A8000BC018DE99AE20E946E3A80E20E94312414
:100A9000CE010E94EFEE0E94803980E20E94312454
:100AA000CE010E94763AC8010E94044B84E090E097
:100AB000DF91CF911F910F9162CFFF920F931F9300
:100AC000CF93DF93EC018B01F42EBC0186E99AE20F
:100AD0000E946E3A80E20E943124CE010E941D5194
:100AE0004F2D0E94AD3980E20E943124CE010E9438
:100AF000763AC8010E94044B84E090E0DF91CF91E8
:100B00001F910F91FF903BCF2F923F924F925F9298
:100B10006F927F928F929F92AF92BF92CF92DF920D
:100B2000EF92FF920F931F93CF93DF93CDB7DEB772
:100B3000C459D1090FB6F894DEBF0FBECDBF4C012A
:100B4000DC0116968D919C911797893C910511F4C3
:100B50000C94D59708F063C28335910511F40C9479
:100B60000C9308F0F1C08A31910511F40C947E9039
:100B700008F04FC08531910511F40C945E90B0F5EA
:100B80008231910511F40C94119390F4039703971B
:100B900008F4AEC18091330382FFAAC110922202F1
:100BA0008FEF99E20E949F39C4010E948F3AA0C141
:100BB000449781F719821A8280E89CE10E94044BD5
:100BC0008CE19EE00E94F9C96CE17EE0CE010196C5
:100BD0000E94A92E1092570C60E0CE0101960E944F
:100BE00047CF82E79CE10E94044B82C18731910587
:100BF00011F40C94669010F40C9462908831910575
:100C000011F40C947A90499729F680E00E94F9D06B
:100C10006FC18032910511F40C944991B0F58C317B
:100C2000910511F40C94C59010F40C949D908D31A5
:100C3000910509F45DC14E9709F0ACCFF4018081B4
:100C4000918197FF55C18CE19EE00E94F9C9F401A2
:100C5000EE5AFF4F0081118180919D10882309F485
:100C600047C110929C1080E790E10E948E32B8013B
:100C700083E490E10E941BE0882311F40C940C9112
:100C800088E99DE30E94044B33C18035910511F43E
:100C90000C94EC9208F04CC08A9709F07BCFF401D9
:100CA0008081918193FF24C1F2A0CF2CD3A0EEE8E4
:100CB000F9E229EA39E244914C151D0411F40C942F
:100CC000E69231962E173F07B1F7D7FE02C00C947B
:100CD000E69292FD02C00C94D392F401868D978D1A
:100CE000A0A1B1A18F3F9105A105B10519F010F0A8
:100CF0000C94CD9261E08F2D0E94FFD2D4015E96BC
:100D00006C918F2D0E942ED2F401168D078DA12E8D
:100D1000B02E61E08F2D0E94FFD2A114B10411F01A
:100D20000C94E09160E08F2D0E942ED20C940D92D5
:100D30008135910511F40C9401938235910509F0E8
:100D400029CF1092210DD4C08337910511F40C9452
:100D5000F49608F0B6C08836910511F40C94E69329
:100D600008F052C08535910511F40C94619310F48C
:100D70000C9443938C35910511F40C948493833631
:100D8000910509F007CFED91FC91119750E1C52E27
:100D900057E2D52EE12CF12CF2FF0CC05E962D917E
:100DA0003D914D915C919197A8EEB3E00E9449EF7F
:100DB0006B017C01E3FD5F9AF401808184FD8A9AD6
:100DC000D4018C9185FF06C08091080181608093D9
:100DD0000801479A0E943E29C60ED71EE81EF91E3A
:100DE0000E943E29A7019601261B370B480B590B81
:100DF000DA01C901803A9648A140B10510F00C947F
:100E0000D0930E940B78ECCF8D36910511F40C94A1
:100E10007A9588F48936910509F0BCCE10922202A9
:100E20008D919C9143E0969587954A95E1F7817065
:100E30000E9469505DC08F36910511F40C94BD96E7
:100E40008237910509F0A6CE109222020E947544C5
:100E5000F4018081918192FF4BC0868D978DA0A176
:100E6000B1A1892B8A2B8B2B09F442C04091B00C85
:100E70005091B10C6091B20C7091B30C8AEF97E273
:100E80000E94603A4091B40C5091B50C6091B60C40
:100E90007091B70C85EF97E20E94603AC090B80C51
:100EA000D090B90CE090BA0CF090BB0C80EF97E2B8
:100EB0000E949F39C701B6010E9480390E94893A79
:100EC00017C08C38910511F40C94029558F58537AC
:100ED000910511F40C94249710F40C9454908737D6
:100EE000910511F40C944C978837910509F052CE76
:100EF000CC56DF4F0FB6F894DEBF0FBECDBFDF91EB
:100F0000CF911F910F91FF90EF90DF90CF90BF9006
:100F1000AF909F908F907F906F905F904F903F9099
:100F20002F9008958A3A910511F40C94589738F54A
:100F30008B39910509F02ECE8091CC0C2D913C91EE
:100F4000119732FD02C00C94BA965E964D915D9158
:100F50006D917C919197452B462B472B11F00C946A
:100F6000BA968F7E8093CC0C0E943E296093EB034F
:100F70007093EC038093ED039093EE03B9CF8E3B17
:100F8000910511F40C941796883C910509F002CE56
:100F9000A0911E0DB0911F0D8C91F4012081318123
:100FA00031FF06C0EC5AFF4F9081911101C080E0E3
:100FB000F4019281C12CD12C760192FF04C0C6A409
:100FC000D7A4E0A8F1A893FF05C0F401C2A8D3A854
:100FD000E4A8F5A8082F10E02CE7829FF001112467
:100FE000E25DFC4FC082D182E282F3829C91981331
:100FF00006C08091FB0C9091FC0C0E94434A20E0BB
:1010000030E0A901C701B6010E94BBEDB801811112
:101010000C94C8978EEA97E20E94FA4969CF80390A
:10102000B1E09B0711F40C945C9F08F095C78D3DCF
:10103000910511F40C942F9A08F005C28E3C91058D
:1010400011F40C94159908F089C18B3C910511F4A9
:101050000C945B9810F40C9419988C3C910511F445
:101060000C94CE988D3C910509F094CD10922202FB
:1010700066EC72E284E094E0B6DC6DEB72E28BE445
:1010800090E0F8DC43E068EA72E281E890E015DD88
:1010900065E972E28DE790E0EDDC67E772E28FE4EC
:1010A00090E0E8DC6EE472E283E590E0E3DC44E0AB
:1010B0006AE372E283E090E000DD44E066E272E21F
:1010C00087E090E0FADC44E062E172E28BE090E0DD
:1010D000F4DC43E066EF71E28FE090E0EEDC43E0A9
:1010E0006AED71E283E190E0E8DC43E06EEB71E2EF
:1010F00087E190E0E2DC43E060EA71E28BE190E0BE
:10110000DCDC43E062E871E28FE190E0D6DC43E0B2
:1011100064E671E283E290E0D0DC43E063E571E2F3
:1011200087E290E0CADC43E060E471E28FE290E0A5
:10113000C4DC43E061E371E285E890E0BEDC43E0BB
:1011400062E271E289E890E0B8DC43E063E171E2D9
:101150008DE890E0B2DC43E061E071E281E990E08B
:10116000ACDC43E06FEE70E285E990E0A6DC43E0A2
:101170006DED70E289E990E0A0DC43E068EC70E29C
:1011800080E294E09ADC43E063EB70E284E294E076
:1011900094DC43E068E970E288E294E08EDC43E0AE
:1011A0006BE770E283E390E088DC43E06EE570E299
:1011B00087E390E082DC43E061E470E28BE390E05F
:1011C0007CDC43E06DE170E28FE390E076DC43E0AD
:1011D00069EF7FE183E490E070DC43E065ED7FE15F
:1011E00087E490E06ADC43E06EEB7FE180E094E02E
:1011F00064DC67EA7FE188E194E019DC60E97FE183
:101200008AE690E0F0DB6EE77FE18BE690E0EBDBD7
:101210006CE67FE18CE790E0E6DB43E06DE57FE1A3
:101220008CE690E04ADC43E06EE47FE180E790E00A
:1012300044DC43E06FE37FE184E790E03EDC65E27D
:101240007FE188E790E0CFDB62E07FE18CEF93E025
:10125000CADB43E06BEE7EE180EE93E02EDC43E000
:1012600063ED7EE188EE93E028DC43E06CEB7EE109
:101270008CEE93E022DC43E067E97EE180EF93E0CF
:101280001CDC43E061E87EE188EF93E016DC43E09C
:1012900064E77EE188EC90E010DC43E06FE57EE1FE
:1012A0008CEC90E00ADC43E069E47EE180ED90E0C4
:1012B00004DC43E063E37EE184ED90E0FEDB60E28A
:1012C0007EE186E291E0B3DB6DE07EE188ED90E0C7
:1012D0008ADB6FEF7DE189ED90E085DB61EF7DE1F9
:1012E00085EF90E080DB44E06CED7DE18AED90E0FD
:1012F000E4DB44E061ED7DE18EED90E0DEDB44E097
:1013000066EC7DE182EE90E0D8DB60EB7DE186EE7D
:1013100090E069DB6FE97DE187EE90E0ABDB6EE8A2
:101320007DE18BEE90E0A6DB6DE77DE182E291E06E
:10133000A1DB64E67DE18FEE90E079DB6EE37DE199
:101340008AEF90E074DB68E17DE18CEF90E06FDB89
:101350006AEF7CE18EEF90E046DBCACD813D9105DE
:1013600011F40C94919908F054C08F3C910509F048
:1013700011CCF401808183FF0CC0428553856485C4
:1013800075854093270D5093280D6093290D709318
:101390002A0D86FF11C020911E0D30911F0DF40102
:1013A00086899789A08DB18DF901838F948FA58F40
:1013B000B68F80810E94C580D4018C9185FF0EC0BC
:1013C00052968D919D910D90BC91A02D8093230DEF
:1013D0009093240DA093250DB093260D4091270DD9
:1013E0005091280D6091290D70912A0D22E08CE713
:1013F00097E20E944E3A4091230D5091240D609146
:10140000250D7091260D22E084E797E20E94AE4000
:101410006FCD8A3D910511F40C94B5998C3D9105E1
:1014200009F0B8CBD4018D919C91119792FD02C027
:101430000C94299A5E968D919D910D90BC91A02D52
:101440000E94B84A55CD8E32F1E09F0711F40C94FA
:10145000699D08F075C0893131E0930711F40C944F
:10146000419A08F03EC0823E910509F093CBD40129
:101470008D919C919C0122273C7021153C4009F0E4
:1014800037CD11E0F401468D578D60A171A1452B38
:10149000462B472B09F410E083FF15C0D401929628
:1014A0000C91929720E030E0A9011A966D917D9100
:1014B0008D919C911D970E94BBED60E0811162E0CF
:1014C000802F0E94FFD281E00E94DC6083E090E0E8
:1014D0000E94284BF40182A10E9405D21813F3CF79
:1014E00007CD823251E0950711F40C94599A8C3251
:1014F000914009F04FCBD4018D919C911197EE242E
:10150000E394F12C92FF03C05E96ED90FC9028EEE0
:10151000C22E23E0D22E93FF03C0F401C2A0D3A0B9
:1015200080911202853211F40C94BF9A8F3F11F40E
:101530000C94889BC60123DA85E20E945CD2D8CC49
:101540008E35B1E09B0709F4D3CC08F054C28F323A
:10155000914009F01FCBF4010190F081E02DCD57AF
:10156000DF4FF983E883C358D04076E9A72EB12C2A
:10157000F2FF04C0D4015E96AD90BC90CD57DF4F12
:10158000E881F981C358D040F12CE12CF3FF04C06D
:10159000D4019296ED90FC90F401128165E0D62E74
:1015A00000E012FF08C066A577A580A991A90E9456
:1015B00094F0D62E072F14FD02C00C94909DD401F8
:1015C000D6966D917D918D919C91D9970E9494F0C2
:1015D000E0967FAF6EAFE09711E01E141F040CF091
:1015E00010E0E12FF0E0EE0FFF1FE65AFC4F2080E5
:1015F0003180B501BB0C880B990B0E94C1EDE596BB
:101600006FAFE597E6967FAFE697E7968FAFE797E0
:10161000E8969FAFE8970E943E29E4966CAF7DAFB5
:101620008EAF9FAFE497F10184A590E095958795E3
:101630002C01990F66087708A996DFAEA997AA969C
:101640000FAFAA97AA962EAD3FADAA9725313105C7
:1016500034F044E150E0AA965FAF4EAFAA97AA9645
:101660008EAD9FADAA97059734F4A5E0B0E0AA9699
:10167000BFAFAEAFAA978EEA93E20E945350109389
:101680000102D101EC91F0E0EF51F34F9C968C9167
:1016900080831E141F0424F080912C0380932D035B
:1016A0001E141F0414F40C94969D24EC39E040E0C1
:1016B00050E0C357DF4F288339834A835B83CD587B
:1016C000D0401E141F0414F40C94A49D28E833E1A8
:1016D00040E050E0CF56DF4F288339834A835B8355
:1016E000C159D040A0964CAE5DAE6EAE7FAEA09715
:1016F000E4968CAC9DACAEACBFACE497C757DF4F63
:1017000088829982AA82BB82C958D04065961FAE52
:101710006597E9961FAEE99790EAEA969FAFEA9738
:10172000A1E4EB96AFAFEB97EC961FAEEC97ED967E
:101730001FAEED97B0EAEE96BFAFEE97E1E4EF96FD
:10174000EFAFEF97A8961CAE1DAE1EAE1FAEA897CA
:10175000A4961CAE1DAE1EAE1FAEA497C12CD12CFC
:101760007601CB57DF4F188219821A821B82C55827
:10177000D040F1E0C158DF4FF883CF57D04010E0A0
:1017800000E021E02093AE0C81E00E94DC6083E069
:1017900090E00E94284BC1010E94DF26D1011696DD
:1017A000BC91AB96BFAFAB97F101F781AC96FFAFA1
:1017B000AC97D1011896BC91AD96BFAFAD97F10132
:1017C000F185AE96FFAFAE970E943E296C966CAF46
:1017D0007DAF8EAF9FAF6C97EC962FADEC97ED96EB
:1017E0003FADED97EE964FADEE97EF965FADEF976D
:1017F000AB966FADAB97AC967FADAC97AD968FAD1A
:10180000AD97AE969FADAE970E9476F11816C4F4D0
:10181000AB962FADAB97EC962FAFEC97AC963FAD58
:10182000AC97ED963FAFED97AD964FADAD97EE9679
:101830004FAFEE97AE965FADAE97EF965FAFEF9777
:1018400065962FAD6597E9963FADE997EA964FAD5E
:10185000EA97EB965FADEB97AB966FADAB97AC9617
:101860007FADAC97AD968FADAD97AE969FADAE9771
:101870000E9476F11816C4F0AB968FADAB976596C3
:101880008FAF6597AC969FADAC97E9969FAFE99700
:10189000AD96AFADAD97EA96AFAFEA97AE96BFAD56
:1018A000AE97EB96BFAFEB97C158DF4FE881CF57AC
:1018B000D040AB962FADAB97AC963FADAC97AD9605
:1018C0004FADAD97AE965FADAE97E5966FADE59730
:1018D000E6967FADE697E7968FADE797E8969FADE2
:1018E000E897EE2311F40C947EA10E94BBED87FFD4
:1018F00054C06C968CAD9DADAEADBFAD6C978819E4
:101900009909AA09BB09C357DF4F288139814A8148
:101910005B81CD58D040281739074A075B07E8F5A7
:10192000F1012081E22FF0E0EF51F34F242D6D966D
:101930003FAD6D97231B2083CB57DF4F888399835F
:10194000AA83BB83C558D040E5964FADE597EC968A
:101950004FAFEC97E6965FADE697ED965FAFED97EC
:10196000E7968FADE797EE968FAFEE97E8969FAD2F
:10197000E897EF969FAFEF976C962CAD3DAD4EADCF
:101980005FAD6C97E4962CAF3DAF4EAF5FAFE49781
:10199000C158DF4F1882CF57D04020E030E040E2FE
:1019A00052E4E5966FADE597E6967FADE697E7964C
:1019B0008FADE797E8969FADE8970E9463EF9B0194
:1019C000AC01AB966FADAB97AC967FADAC97AD96D7
:1019D0008FADAD97AE969FADAE970E9476F118167B
:1019E00014F00C94BE9E8CEE92E20E94B34C8FEFEA
:1019F000809301027DCA833621E0920711F40C9492
:101A00004F9F8836914009F0C5C810922202C090BD
:101A10004902D0904A02E0904B02F0904C0285E1DE
:101A20009AE20E949F3989E696E20E949F39C70197
:101A3000B6010E9480390E94893A6FE770E08CE518
:101A400096E20E94324A61E070E08FE496E20E94E2
:101A5000324A70E060E08FE396E20E94324A61E031
:101A600070E084E396E20E94324A61E070E08CE22A
:101A700096E20E94324A70E060E087E296E20E94BD
:101A8000324A85E19AE20E949F3980E296E20E9402
:101A9000044B61E070E08BE196E20E94324A61E023
:101AA00070E086E096E20E94324A6FEF7FEF8CEFA3
:101AB00095E20E94324A6FEF7FEF82EF95E20E943B
:101AC000324A6FEF7FEF88EE95E20E94324A20E0C3
:101AD00030E0A90160911A0C70911B0C80911C0CD4
:101AE00090911D0C0E9463EFAB01BC0122E08EEDD2
:101AF00095E20E945A4420E030E0A9016091160C62
:101B00007091170C8091180C9091190C0E9463EF42
:101B1000AB01BC0122E084ED95E20E945A4420E032
:101B200030E0A9016091120C7091130C8091140C9B
:101B30009091150C0E9463EFAB01BC0123E08AEC8D
:101B400095E20E945A4461E070E08BEB95E20E94BE
:101B5000324A61E070E08FE995E20E94324A70E01B
:101B600060E083E995E20E94324A70E060E08BE831
:101B700095E20E94324A70E060E080E895E20E94BF
:101B8000324A61E070E088E795E20E94324A60E103
:101B900070E088E695E20E94324A4091270D50910C
:101BA000280D6091290D70912A0D22E080E695E2C2
:101BB0000E945A4460ED77E08DE495E20E94324A3B
:101BC0004091230D5091240D6091250D7091260DAB
:101BD00022E086E495E20E945A4480EE93E00E945F
:101BE0001D51AB01BC0122E084E395E20E945A44FE
:101BF00084EE93E00E941D51AB01BC0122E08EE116
:101C000095E20E945A4488EE93E00E941D51AB0178
